:020000040800F2
:1000000000500020D94A0108854B010879350108C4
:10001000854B0108854B0108854B01080000000055
:10002000000000000000000000000000854B0108F7
:10003000854B010800000000854B01084935010887
:10004000854B0108854B0108854B0108854B01084C
:10005000854B0108854B0108993401089534010846
:10006000854B0108854B0108854B0108854B01082C
:10007000353501082135010855340108854B010843
:100080000D350108F9340108854B0108854B01083D
:10009000854B0108854B0108854B01089134010807
:1000A000854B010811340108854B010821340108F2
:1000B00001340108F1330108E1330108A9340108D2
:1000C000A1340108A53401089D340108854B0108BD
:1000D000854B0108493401083D34010831340108D9
:1000E00059350108854B0108854B010800000000C7
:1000F0000000000000000000000000000000000000
:0C01000000000000000000005FF808F1A3
:100110002DE9F04FB54BDBB01F78002F00F0C38006
:10012000B34C6068002801F07A870AF063FAA0688F
:10013000AF4D0AF027FB002801F07187A8680AF08C
:100140001CFB092801D03F2848D14FF00008E66881
:10015000A84F45462EB1A8483968324616F09EFD94
:1001600010B9B84605B93D46A44B10379F42F1D3AC
:10017000BDB1E3682A689E48D75CD8F80020D15CFE
:10018000B9420ED15A1C41B92D2B06D8C260034486
:10019000202702441F74117403E023441F74E2609B
:1001A000E7E7E3680BB145450FD095480AF043FAFD
:1001B000454507D855F8100B0AF03DFA09200AF01A
:1001C00033FAF5E70AF044FA0026E3689E42AED21D
:1001D000894B985D0AF028FA0136F6E7EB68002BA8
:1001E00041F09986042841F0F38605F1100006F0ED
:1001F0001DFC01F014BF052A00F0A680266C96F8BD
:1002000048A0BAF1060F64D196F849004D2800F0D5
:10021000338500F29081322800F04F8500F22B8167
:10022000242800F0E08400F2C380032800F0338229
:1002300040F29D80052840F0AF801A2006F0C8FAF1
:100240000024704B185D013406F07CFA0B2CF8D1B9
:1002500000246D4B185D013406F074FA082CF8D1B7
:1002600000246A4B185D013406F06CFA072CF8D1B3
:1002700006F07AFA2B6C002283F84820A86C0AF06A
:10028000B9F995F8C83053B1614BD8590AF06AFAF8
:100290000CF032FF0AF01FFA5E4A5F4BDA604C370F
:1002A000982F01F0BC865A49594B7A583B44002A92
:1002B000F5D04F4D59496A64139200222B648DF892
:1002C000512012AB142212918DF85020AB642C46B1
:1002D0008846606CDFF818A10AF054FA0028CDD0E7
:1002E000DAF844000AF049FADAF84030064693F8A2
:1002F000482022B9242840F0F285012234E0012A66
:1003000004D14D280CBF022200222DE0022A04D184
:100310003C280CBF0322002226E0032A09D14028F2
:100320004FF0000220D81A71DA71587198710422C6
:100330001AE0042A7FF45FAF9A7983F8490080EAD3
:1003400002069E7105220FE059791A799142997936
:1003500006D941409971511C1971134418724DE727
:1003600081420CBF0622002283F8482046E701287C
:1003700000F08581022840F00286042006F028FA69
:10038000422006F0DFF9542006F0DCF9462006F0A2
:10039000D9F94C2000F09FBDC0F08881222840F0A0
:1003A000EE851F4C502006F013FA04F150061EE3B0
:1003B0002A2800F0408435D8262800F01A842828FE
:1003C00040F0DD85164C072006F002FAB4F81A0258
:1003D00006F001FAB4F81C0206F0FDF994F81E02CA
:1003E00006F0B0F9B4F8200200F03ABDDC3200208B
:1003F000DC14002070A50108EC14002060A701089F
:10040000E0BE010848BF010854BF01085DBF0108F4
:10041000640E00200400FA0500ED00E07D7D000878
:10042000500400202E2800F08F84302800F0A38490
:100430002C2840F0A485D84C0C2006F0C9F994F87B
:100440003C0206F07FF9B4F8480206F0C4F9B4F8AB
:10045000440206F0C0F9B4F8460206F0BCF994F87C
:100460003E0206F06FF9B4F84E0206F0B4F9B4F8A3
:10047000500200F0F5BC402800F0268423D838282C
:1004800000F0C68311D8342800F0CA82362840F024
:100490007685C24BC04C187804F12806C0EBC0002A
:1004A000C0B206F095F900F04BBC3B2800F09882F2
:1004B0003D2800F039823A2840F06185042006F09A
:1004C00087F9B74B8DE3462800F07B840BD8422890
:1004D00000F00984452840F05285132006F078F991
:1004E000002400F09CBC492800F029824B2800F031
:1004F000A883472840F0438506F040FA044684204C
:1005000006F066F9204606F06FF9A64B04F180026A
:10051000DB681AAE9A428CBFC4EB03084FF0800828
:100520000FF032FC20464246314606F0B5FE00246C
:10053000804600F05ABC702800F032825BD86728F1
:1005400000F01D8134D8522800F0648418D84F2858
:1005500000F05384502840F012858F4C042006F0A0
:1005600037F9012006F0EEF894F8050506F0EAF8F0
:1005700094F8030506F0E6F894F8040500F0ABBC27
:10058000652800F0A58000F2CC80642840F0F78454
:10059000072006F01DF9E72006F0D4F87E4B5879C5
:1005A00006F0D0F8002006F0CDF8042000F042BCA0
:1005B0006C2800F079810ED8682800F05E816928E7
:1005C00040F0DD84784E00243078400000F0FE00DA
:1005D00006F0FEF85DE16E2800F0768100F2B5814C
:1005E000062006F0F5F8714B186806F0FDF8B5F82E
:1005F000880000F035BC7C2800F020841CD87428CA
:1006000000F030820AD8722800F09582732840F0FA
:10061000B684082006F0DCF80124C1E2772800F057
:100620006F82782800F0D480752840F0A8842F20AD
:1006300006F0CEF85E4CCBE1A02800F0C6820AD8C6
:100640007E2800F03A84C0F02984962808BF0C2048
:100650003FD000F094BCF12800F0E980FE2800F0C3
:10066000A782F02840F08B844B4C042006F0B0F8B1
:10067000B4F8F20106F0AFF8B4F8F001F0E30320AB
:1006800006F0A6F8002006F05DF8012006F05AF802
:10069000102000F020BC06F09BF8022006F052F873
:1006A000504606F04FF8012000F015BC062006F079
:1006B0008FF8412006F046F8462006F043F84E2019
:1006C00006F040F8412006F03DF83A4B1878C7E3B1
:1006D0000B2006F07DF8384B188806F07CF8B5F84A
:1006E0006C0080B206F077F8344B1B68C3F3C0008F
:1006F000C3F38002800040EA4200C3F3400210438B
:10070000C3F3401240EAC20003F01003184306F09E
:1007100062F806F072F806F067F81F4B93F8580479
:10072000D9E3122006F054F8254B00261B88B3F5B8
:10073000806F94BF4FF001084FF00808214C04F17E
:100740007003F058043690FBF8F080B206F043F8DE
:100750000C2EF3D11C4E308806F03DF8B08806F020
:100760003AF8308906F037F8B4F87C0006F033F830
:10077000B4F8800006F02FF8B4F8840070E310207D
:1007800006F026F80024114B185D013405F0DAFF5D
:10079000102CF8D16CE500BF50040020440A002062
:1007A000141000200C000020E80F00205C1800202E
:1007B0005FA70108DB320020D8320020100E002095
:1007C00006000020DC140020B0180020940A00204D
:1007D000702005F0FDFFBE4C0026A046B4F856017F
:1007E00005F0F9FFB4F8580105F0F5FFB4F85A0127
:1007F00005F0F1FF94F85C0105F0A4FF94F85D01A9
:1008000005F0A0FF94F85E0105F09CFF94F85F01ED
:1008100005F098FF0E2303FB06830136D3F8600131
:1008200005F0E2FF082E04F10E04D7D120E5702078
:1008300005F0CEFFA64C04F1700694F8E60005F032
:1008400081FF94F8E70005F07DFF94F8E80005F0DB
:1008500079FF94F8E90005F075FF94F8EA0005F0D7
:1008600071FF94F8EB0005F06DFF073494F8E50094
:1008700005F068FFB442E0D1FAE4102005F0A8FFCB
:100880000024944B185D013405F05CFF102CF8D166
:10089000EEE433789C42BFF4EBAC8F4B33F814009A
:1008A00005F099FF0134F4E78C4C504605F090FFB9
:1008B000208805F090FF608805F08DFFB4F90400F2
:1008C0000A2390FBF3F028E0072005F081FF844B1A
:1008D0004FF6FF761888834CFF28A8BFFF20C0B2D0
:1008E00005F030FFD5F88C00B042A8BF304620EAB2
:1008F000E07080B205F06FFFB5F8900005F06BFF77
:10090000734B93F81F3253B1D4F894300A205843F4
:10091000B042A8BF304620EAE07080B2A0E2D4F82E
:10092000940000F30F00F8E7694C022005F050FF37
:1009300094F8890205F006FF94F88802CBE20220C1
:1009400005F046FF684B18888AE2684C0B2005F0DA
:100950003FFF23680026187805F0F4FE2368A046C0
:10096000587805F0EFFED8F80030604C3344187921
:10097000013605F0E7FE032EF5D12368D87905F09E
:10098000E1FE2368987805F0DDFE2368D87805F04D
:10099000D9FE2368588905F01EFF2368187A9AE269
:1009A0001E2005F015FF0024514E3368234458786B
:1009B00005F0C8FE33682344D87A05F0C3FE3368D7
:1009C0002344587D013405F0BDFE0A2CECD14FE4E0
:1009D00014F8010F00283FF44BAC05F0B3FEF7E725
:1009E000012005F0F5FE424B1B68187873E2414A7E
:1009F00094F859340C2101FB0323187A05F0A2FE68
:100A000094F85A0405F09EFE94F85B0405F09AFEF3
:100A1000043494F8580405F095FEB442E7D127E475
:100A20005A2005F0D5FE2A4C04F15A0694F8AE047B
:100A300005F088FE94F8A90405F084FE94F8AA0451
:100A400005F080FE94F8AB0405F07CFE94F8AC044D
:100A500005F078FE063494F8A70405F073FEB4425E
:100A6000E4D105E44FF0000801240026224B1B7856
:100A70009E4224DA214BF15C00231E4A03EB020B59
:100A80009A5C8A4204D00C33B3F5BA7FF5D114E0F6
:100A9000DBF8040016F0FAF881460CB9A24601E032
:100AA00080440AE0CA4508DADBF8042012F80A009C
:100AB00005F048FE0AF1010AF4E70136D6E7002CFA
:100AC0003FF4D6AB5FFA88F005F082FE0024CCE755
:100AD00050040020B81900202E0F002036180020E6
:100AE0009E190020DC1400205814002090190020CA
:100AF0004018002090A70108620E0020440E00203C
:100B0000D94E0024307805F063FE33789C42BFF460
:100B1000AFABD64BE05C0023D54A99189A5C824271
:100B200004D00C33B3F5BA7FF6D102E0087A05F0B1
:100B300009FE0134E9E7CF4C162005F049FEB4F870
:100B4000440205F048FEB4F8D00005F044FEB4F8C5
:100B5000D20005F040FEB4F8D40005F03CFEB4F835
:100B60009A0205F038FE002005F0ECFD002005F0AB
:100B7000E9FD002005F0E6FD94F81F0205F0E2FD16
:100B800094F8400205F0DEFD002005F0DBFDB4F92D
:100B9000EE010A2390FBF3F080B205F01CFE3BE06F
:100BA000E0B2013405F0CEFD092CF9D1FFF760BBAE
:100BB000082005F00DFE0024AF4B185B023405F051
:100BC0000AFE082CF8D1FFF753BB0C2005F000FEFD
:100BD000AA4B186805F008FEA94B186805F004FE3A
:100BE000A84B186826E1042005F0F2FDA14B986897
:100BF00020E1A04C062005F0EBFDB4F8CC0105F097
:100C0000EAFDB4F8D00105F0E6FDB4F8D40127E11F
:100C1000042005F0DDFD974C94F8120205F092FDDA
:100C200094F8160205F08EFD94F8150205F08AFD81
:100C300094F817024FE1012005F0CAFD8D4B587959
:100C400049E18C4C082005F0C3FD94F8980205F0AA
:100C500079FD94F8990205F075FDB4F89A0205F053
:100C6000BAFD94F89C0205F06DFDB4F89E0205F003
:100C7000B2FD94F8A0022EE1DFF81C82824C98F8B5
:100C80000000002600EB4000C0B205F0A1FD98F87E
:100C9000003002349E42BFF4EBAA14F8020C05F0B7
:100CA00051FD14F8010C013600EB800000EB8000D0
:100CB00000F2EE2005F08FFDE9E7012005F088FD48
:100CC0006C4B93F8400206E1082005F081FD0024FA
:100CD000684B234493F83402013405F033FD082CAB
:100CE000F6D1FFF7C5BA634C102005F071FD6079AD
:100CF00005F028FDA06805F077FD94F83C0205F0AA
:100D000021FDB4F8CC0105F066FDB4F8D00105F082
:100D100062FDB4F8D40105F05EFDB4F81A0205F0E6
:100D20005AFDB4F81C029BE0584AD25C904200F095
:100D30000F810C333C2BF7D10834B4423FF498AA0E
:100D400094F8A4020023EFE7402005F041FD494C50
:100D500004F14006B4F8600305F03DFD94F8620329
:100D600005F0F0FC043494F85F0305F0EBFCB442AA
:100D7000F0D1FFF77DBAE02005F02AFD3D4C04F1EB
:100D80008006B4F8E202043400F03F0005F023FDD1
:100D9000B4F8DE02C0F3861005F01DFD94F8DC0205
:100DA000000905F0CFFC94F8DC0200F00F0005F01C
:100DB000C9FC94F8DD0205F0C5FCB442E1D1FFF7AF
:100DC00057BA0D2005F004FD06F032FA304C40F021
:100DD0000200C0B205F0B6FC208805F005FDE06811
:100DE00005F002FD10F0B2FD24E04445BFF640AA34
:100DF000305D05F0A7FC0134F7E70B2005F0E8FCB7
:100E0000002005F09FFC002005F09CFC002005F070
:100E100099FC0BE0012005F0DBFC00205BE01D4BA2
:100E2000185D013405F08EFC0B2CF8D1002005F084
:100E3000DBFC002005F0D8FCFFF71ABA0D4C0820A7
:100E400005F0C6FCB4F8D80005F0C5FCB4F8DA002B
:100E500005F0C1FCB4F8DC0005F0BDFCB4F8DE0020
:100E600005F0B9FCFFF704BA620E0020440E002022
:100E700090A701085004002008180020E8F7FF1F81
:100E8000ECF7FF1FF0F7FF1FA2060020480A002022
:100E90000C00002048BF0108E80F0020D04C0320C0
:100EA00005F096FC94F8220205F04CFC94F823021D
:100EB00005F048FC94F824020DE0C94C032005F02D
:100EC00087FC94F8C70105F03DFC94F8C80105F0D3
:100ED00039FC94F8C90105F035FCFFF7C9B9DFF812
:100EE00020B39BF8003013F004027FF487A9232E6F
:100EF000DAF844301ED1BB480121CAF80830CAF8DC
:100F00004C30CAF85430102301708AF859208AF8FE
:100F10005830B5480AF15003CAF85080CAF8043076
:100F200009F089FB09F094FB9BF8003043F00203C1
:100F30008BF80030AD4B1B681B78B3427FF45EA981
:100F4000AB4AAC4B1A60AC4AAC4BDA60FFF756B90F
:100F500005F0F8FBB4F8A60205F03DFC94F8A802F1
:100F600005F0F0FB94F8A90205F0ECFB94F8AB0255
:100F700005F0E8FB94F8AA0205F0E4FBDCE64E2855
:100F80003CD109F08EFA1128044602D90BF06EFA12
:100F90002FE009F086FA924E04F5927406EB4403B2
:100FA000987205F0E1FC40F2ED23984205DD40F631
:100FB000CA039842A8BF184601E040F2EE20A0F212
:100FC000EE20192306EB440490FBF3F0E07210E0EE
:100FD000C0F0C482D02800F0DF82D22840F097878A
:100FE000874B1B7803F0040303F0FF04002B00F091
:100FF000DF82002005F0ECFBFFF73AB900F2CF8169
:1010000035281CD109F04DFA0E28BFD87D4B062695
:1010100006FB003609F045FA0328B7D8B07109F08D
:1010200040FA707009F03DFAB07009F03AFAF070C9
:1010300009F037FA307109F034FA7071D9E700F22B
:10104000EB802B2804D109F02CFA654B5871D0E7BE
:1010500062D8252807D1624B00229A6005F08EFCE9
:101060000AF0ACF8C5E732D8232840F0508709F0E1
:1010700018FA13288AD85A4B00F58B7603EB8606AC
:1010800009F00FFA604B741C03F5BA72197A8142A9
:1010900003D00C339342F9D178E71B78737009F0D1
:1010A00000FA607009F0FDF9A07009F0FAF9574BE9
:1010B000574A1B68E0700020C5F8C430C5F8C0204E
:1010C0000BF0EAF8534B80F00100187091E72728E5
:1010D0000DD105F049FC424CC4F8CC0105F044FCAC
:1010E000C4F8D00105F040FCC4F8D40181E72928F8
:1010F00040F00D8705F038FC394CA4F81A0205F0D1
:1011000033FCA4F81C0209F0CCF984F81E0205F0A7
:101110002BFCA4F820026CE72F2800F0858424D84B
:101120002D2840F0F48609F0BCF92D4C84F83C02DF
:1011300005F01AFCA4F8480205F016FCA4F84402D5
:1011400005F012FCA4F8460209F0ABF984F83E025F
:101150007379082B7FF64DAF05F006FCA4F84E021C
:1011600005F002FCA4F8500243E731282ED109F023
:1011700098F91F283FF60AAF7379082B7FF406AF62
:1011800000F1B80805F0F0FB154E00F03F0006EB4B
:101190008804608005F0E8FB6288800100F4FE535B
:1011A0001343638009F07DF9000106F8280009F077
:1011B00078F916F8283000F00F00184306F82800D8
:1011C00009F06FF9607010F04BFB12E7332840F024
:1011D0009E8609F066F9024B83F8400209E700BFDA
:1011E00050040020DC32002010BF0108400A00201B
:1011F000EFBEADDEF04F00200400FA0500ED00E088
:10120000DA320020F808002090A7010840180020DA
:101210002005002028000020412800F0F9836AD82A
:10122000392811D109F03DF9D24C84F8120209F0A5
:1012300038F984F8160209F034F984F8150209F037
:1012400030F984F81702D4E632D8372840F05F86A8
:1012500073790726B3FBF6F2C2EBC2029A1A12F0B8
:10126000FF0F7FF493AEB3FBF6F6002E3FF4C1AE52
:1012700009F017F95FFA80F84FFA88F009F060F981
:10128000013EF6B2044600283FF480AE80F80080AC
:1012900005F06AFB608009F004F9207109F001F99A
:1012A000607109F0FEF8E07109F0FBF8A071DCE76D
:1012B0003C2813D1B04C266896F8008009F0F1F86C
:1012C00030702368187809F023FC23681B784345A5
:1012D0003FF48FAE00200DF025FE8AE63E2840F058
:1012E000168609F0DEF8A34C84F8890209F0D9F8D3
:1012F00084F888027DE6482802D10EF0B7FC78E633
:101300002BD8432822D109F0CCF89A4C0023A360B3
:10131000607105F033FB09F051FF09F0C2F884F861
:101320003C0205F021FBC4F8CC0105F01DFBC4F81C
:10133000D00105F019FBC4F8D40105F015FBA4F8A1
:101340001A0205F011FBA4F81C0252E6442840F0F2
:10135000DE85012385F8C8304BE64A2802D105F026
:1013600003FBB8E74C2840F0D28509F09AF8814C8D
:1013700084F8980209F095F884F8990205F0F4FAD7
:10138000A4F89A0209F08DF884F89C0205F0ECFAB2
:10139000A4F89E0209F085F884F8A00229E6D32873
:1013A00004D105F0E1FA754B188022E600F20A81BB
:1013B000CD2809D1724B1B785C073FF51AAE714BF3
:1013C0004FF4C8721A8014E600F28F80C82827D123
:1013D00074796408122C3FF6D9AD0026A64206D2D5
:1013E00005F0C2FA1AAB23F816000136F6E700231F
:1013F000A342654A06DA1AA931F8131022F813102D
:101400000133F5E7013C02EB44042232944203D05D
:10141000002324F8023FF9E7012385F8BC30E8E512
:1014200015D8512840F07385584B1B78012B3FF697
:10143000E0AD09F036F84F4C84F8050509F031F8B5
:1014400084F8030509F02DF884F80405D1E5CA28CD
:1014500000F0C482CC2840F05A857379092B7FF6BE
:1014600095AD4B4CD4F8008009F01BF888F80000CB
:10147000D4F8008009F015F888F8010009F011F897
:1014800023686428A8BF6420187109F00AF823684B
:101490006428A8BF6420587109F003F82368FF2866
:1014A000A8BFFF20987108F0FCFFD4F800806428E2
:1014B00028BF642088F8070008F0F3FF88F80200CE
:1014C000D4F8008008F0EDFF88F80300D4F800801D
:1014D00005F04AFAA8F80A0073790A2B7FF689AD5D
:1014E000246808F0DEFF207283E5CF287FF470AD1A
:1014F00005F03AFA6FF4AF6E00EB0E039BB21D4C91
:10150000C62B98BFA4F8440205F02EFAA4F8D00028
:1015100005F02AFAA4F8D20005F026FAA4F8D400BF
:1015200005F022FAA4F89A0208F0BBFF08F0B9FF10
:1015300008F0B7FF08F0B5FF84F81F0208F0B1FF0C
:1015400084F8400208F0ADFF05F00EFA00EB8000D1
:101550004000A4F8EE0108F0A4FF66E6084B1B78F3
:1015600058073FF546AD0B4B1A7842F004021A704B
:101570003FE500BF50040020401800203C18002028
:10158000DA3200206214002074150020601400205C
:1015900090190020B90D0020C04B1B785E073FF565
:1015A00028AD0DF05BFA04F0F1F807F0B7FD20E587
:1015B00008F077FFBA4B012883F85804F3D983F871
:1015C0005844F0E7DB283FF414AD5AD8D62800F091
:1015D000FB8131D8D42840F09A8473790F2B7FF4A3
:1015E000D5AC08F05EFF072880463FF6CFAC05F08B
:1015F000BBF9AB4B0E2606FB0836A6F8560105F0E4
:10160000B3F9A6F8580105F0AFF9A6F85A0108F0A9
:1016100048FF86F85C0108F044FF86F85D0108F099
:1016200040FF86F85E0108F03CFF86F85F0105F098
:10163000A5F9C6F86001DCE4D92811D105F094F9C8
:10164000974CA4F8D80005F08FF9A4F8DA0005F05B
:101650008BF9A4F8DC0005F087F9A4F8DE00C8E4F3
:10166000DA2840F0548408F01CFF8D4C84F82202E4
:1016700008F017FF84F8230208F013FF84F824020F
:10168000B7E4F22821D108F00CFF0F2804463FF6FA
:101690007DAC08F006FF834BC4EBC4041C44A0716E
:1016A00008F0FFFEE07108F0FCFE207208F0F9FE81
:1016B000607208F0F6FEA07208F0F3FEE07208F027
:1016C000F0FE207309F04DF993E41CD8DC280DD10D
:1016D00008F0E7FE724C84F8C70108F0E2FE84F8D7
:1016E000C80108F0DEFE84F8C90182E4EF2840F06A
:1016F0000E8405F039F96A4CA4F8F20105F034F9CA
:10170000A4F8F00175E4F52840F05581012005F0BA
:101710005FF8654900260E7064483146C02285F89E
:10172000C96015F072FA8DF80F60614B9DF80F20BB
:101730009978914259D99DF80F2003EBC202527952
:10174000D2074BD59DF80F2003EBC2021179594AFD
:1017500032F91120002A41DD9DF80F1094F8C9A03C
:1017600003EBC10189684FEA0A124968A618C6F856
:10177000CC109DF80F1003EBC1039B681889002360
:10178000A6F8D20001219940014003D10133102B6A
:10179000F8D100E01946A618B6F8D230A6F8D01055
:1017A000A6F8D430022386F8D730482386F8D630FE
:1017B000D6F8D4304049C6F8D830102386F8DA304D
:1017C0001144D6F8CC0010F090F9D6F8CC30B6F829
:1017D000D2200AF1010A1A6184F8C9A09DF80F30DD
:1017E0000133DBB28DF80F309FE795F8C90004F0A4
:1017F000A9FF04F0B9FFA86C08F0FCFE2B6C186878
:1018000008F0B0FFAB6C2A6CC5F89031C5F88C219C
:101810000DF058FF4FF0000884F8948184F895810A
:1018200007F04FFE2F28F5D1244EADF81480336811
:10183000B2885A6107F045FE824607F042FE8DF8F5
:101840001D0007F03EFE8DF81E0007F03AFE8346AD
:1018500007F037FE0DF1680909F8080008F10108E2
:101860005FFA88F29345F3D108F091FF8DF81100EB
:1018700008F08DFF3268B1888DF810001161BDF855
:101880001010B4F89421914200F0E2804FF000086B
:1018900005AA4FF001094FF0030B20E0DA320020D7
:1018A00050040020300500201C000020A815002056
:1018B000A80A0020B8190020B015002074090020E3
:1018C0009DF8682094F8C910BC4B914200F22B811E
:1018D0004FF0000805AA4FF001094FF0080BB3893B
:1018E000B06800214361D4F88C0184F8A91184F810
:1018F000AA1100680191009208F024FF2E2006F042
:101900003DFD504606F03AFD9DF81D0006F036FDFF
:101910009DF81E0006F032FD484606F02FFD0199A5
:10192000009A8A4612F80A000AF1010A009206F0AB
:1019300025FD5FFA8AF18945009AF3D1584606F0F1
:101940001DFDD4F8900194F8AA1108F05FFE94F8F8
:10195000A911D4F8900108F059FED4F88C31186818
:1019600008F0EAFED4F8900108F044FEB368B289AA
:101970001A61B8F1000F3FF44DAF94F8C9208F4BB6
:10198000A2B1013AD2B283F8C92012019E181821DF
:1019900086F8DA10D6F8CC0006F1D80110F0A5F8D8
:1019A000D6F8CC30B6F8D2205A61E6E7844A012353
:1019B0001370FFF71EBBFA2840F0A982814B1B78F9
:1019C00059077FF5F0ADA2E2002404F0CDFF7E4B75
:1019D00018530234102CF8D1FFF70BBB00247B4EB8
:1019E000D6F8008008F05DFD08EB04035870D6F8C7
:1019F000008008F056FD08EB0403D872366808F042
:101A000050FD264401340A2C7075E8D1FFF7F1BA75
:101A1000002408F046FD6E4B23440134082C83F863
:101A20003402F6D1FFF7E5BA694C04F1400604F040
:101A30009BFFA4F8600308F034FD84F8620308F00B
:101A400030FD043484F85F03B442F0D1FFF7D1BA1B
:101A5000AAF13003CDF8209000220F2B00F215825E
:101A600001A050F823F000BFA91A0008F51A0008D9
:101A70009B1E0008FD1A0008A71E0008C1180008D8
:101A80008B1E0008591B0008BF1C0008231D0008FE
:101A9000671D0008DB1D00088B1E0008971D00084D
:101AA0000D1E0008151B00082378002B00F0E781AD
:101AB000424B93F89631002B00F0FC81022B02D9A7
:101AC000032B11D0F6E1FD238DF830300CA8002354
:101AD00002218DF8313003F05FFF012003F006FF93
:101AE000C12800F0CC81E5E106F0D6F9002800F02D
:101AF000E181C4E16A238DF81430C0E190238DF8B0
:101B0000143004238DF815304FF0000805AA4FF06B
:101B10000209FAE19DF868305A1E022A00F2A781F4
:101B200084F89631ABE183F8972193F89621013A36
:101B3000012A0AD800228DF830208DF831200CA817
:101B4000012202211A7003F027FF4FF0000884F8E9
:101B5000008084F8018094E1227062709DF8683002
:101B600094F8C9209A427FF6B3AE144A4FF00308A6
:101B700082F8973106F090F960B3DFF840B00121A8
:101B80000BF1010006F046F920B35846022106F099
:101B900041F9F8B1BBF8003049F2073223F00801EF
:101BA000914207D049F20A32934203D049F20B42E4
:101BB00093420FD1032384F8963185E1DC14002091
:101BC0001C000020DA320020D0190020401800202C
:101BD00050040020C2490DF1180B0A888B78ABF82D
:101BE00000208BF802300CAA0B1D01F1140C1868B0
:101BF00059689646AEE80300083363457246F6D14D
:101C000018681B79106015210CA813710DF12409B7
:101C100003F0C2FE4846082103F079FE002840D0B8
:101C2000002219F802001BF80210884239D1013253
:101C3000032AF6D1AB4A99F8031099F80530917050
:101C400099F804101370517013884FF2103123F07B
:101C50002000884211D04FF210418B420DD04FF23C
:101C600090318B4209D04FF650018B4205D003F5DD
:101C7000BA510F3189B2012901D801230EE023F0B6
:101C8000080049F20731884207D049F20A318B42F5
:101C900003D049F20B418B4203D1022382F89631E3
:101CA00012E108F1FF3818F0FF087FF463AF8D4AA6
:101CB0004FF0040982F8008082F801800DE194F869
:101CC0009631DFF82082032B40F0DF804FF0120BBB
:101CD00088F898B103F076FF002003F029FF072071
:101CE00003F026FF0E2003F023FF584603F020FFE9
:101CF000142003F01DFF002003F01AFFAC2003F0B6
:101D000017FF882003F014FF132003F011FF762043
:101D100003F00EFF06F05CF808F2991003F080FC67
:101D200095E094F89631012B40F0AF809DF8683033
:101D300007A88DF814305B008DF81D3000238DF856
:101D40001E3003F0A3FE002878D0674B0CA81B8838
:101D50000221ADF8303003F01FFE142003F0C6FD61
:101D600030286BD18BE09DF868308DF81C3094F8EA
:101D70009631002B00F0BC80022B02D9032B04D03B
:101D8000B6E00CBF0720032011E007A806F0A2F878
:101D900098B114221AE09DF868308DF81C3094F840
:101DA0009631022B02D0032B0AD0A1E0042007A910
:101DB00003F094FE002840F0A3804FF00F0B99E051
:101DC00007A806F087F80028F7D01622454B07A889
:101DD00083F8982106F008F9ECE794F896318DF82D
:101DE0001CB0002B4BD0022B02D9032B08D046E0AD
:101DF00007A803F04BFE08B3012007A9142224E032
:101E000007A806F067F8C8B1132229E094F89631C4
:101E10008DF81CB0022B0DD0032B1BD0012B4FF0E3
:101E2000000805AA4FF001090CBF4FF0020B4FF05C
:101E30000F0B54E507A803F029FE10B94FF0000876
:101E40003EE0052007A940F2DC5203F0E3FD002844
:101E5000F4D014E007A806F03DF80028EED01522D3
:101E6000204B07A883F8982106F06AF8EFE74FF0B7
:101E7000000805AA4FF001094FF0090B2FE54FF0BC
:101E8000000805AA4FF001093FE04FF0000805AA3D
:101E90004FF001094FF0020B21E54FF00008134A03
:101EA0004FF0090931E04FF0010805AAC1464FF093
:101EB000000B14E54FF0000884F8008084F80180DE
:101EC00005AA4FF0010908E094F896314FF0000898
:101ED000E370044A4FF0040917E04FF00F0BFEE4E3
:101EE00004A90108DC1400201DA90108D6BE0108C0
:101EF0004FF0020B4FF0000805AA4FF00109EEE485
:101F00009DF81C904FF000081AAAC346E7E40AF0B7
:101F1000ADFAFEF7ADB90C2803D1424808F08BFBAF
:101F200052E00A2801D00D286DD13F4D3F4805F100
:101F3000100608F080FB3046232114F09AFE08B109
:101F4000801BE860E368002B35D0591E705C364A70
:101F5000202801D10B46F6E7D360134400221A74FF
:101F6000334B344DD3F800A0D5F80090DFF8B8809B
:101F7000484614F08BFE08F11007064649463846DD
:101F8000324614F08BFE2C4B30B908EB0602127C63
:101F900052445278520703D010359D42E4D306E0F4
:101FA0009D4204D2701CEB683844984702E02348F5
:101FB00008F041FB0023224800213022E36014F0A6
:101FC00024FE2048037853B308F042FBFEF7AFB875
:101FD0000C28A2D07F2804D1FEF7A9B82F2B3EF6FB
:101FE000A6A8A0F12002D2B25E2A3EF6A0A813B99C
:101FF00020283EF49CA85A1C2344E260187408F080
:1020000013FBFEF794B87F28E8D1013BEB60002278
:102010002B440D481A7408F00EFBFEF788B85BB02D
:10202000BDE8F08FE5BE0108DC140020EAD001080D
:10203000DC03002070A5010860A70108F0BE0108BC
:10204000EC140020DC3200200CBF01082DE9F04F19
:102050009E4F9F4C3A68267902F59C4320338DB001
:102060002360C6B1A3689A4240F20581013E267101
:1020700001E1DFF87882072DD8F800308CBF2946BF
:10208000595D944B94481B689847032D09D904EB7C
:102090004505A881013604F0F3FAF5B28542E8D38C
:1020A0001FE0D8F8003005F1100203EB82025388DC
:1020B00092880028EBD0C01A4FF47A714843D31AA3
:1020C00090FBF3F0084440F6C903984205DC40F267
:1020D000EE239842B8BF184601E040F6CA0080B22D
:1020E000D5E77E4B42F201091B6803EA0909D9F1E1
:1020F00001097B4B38BF4FF00009D3F800A0984688
:10210000B9F1000F06D194F8313084F83030754BB6
:102110005A781A7094F830302BB1724B93F800B0A3
:102120008BF0010B00E09B460F23002684F8323031
:10213000354604F0A5FA854263DABBF1000F02D000
:10214000694BF05A00E05846684B1B685A8B824234
:1021500005D8998B814234BF0021012100E0002184
:10216000634A644BC1B952F82520924501D2985B6D
:1021700016E0EAB210460392029304F057FA039A6B
:10218000029B032A0CD80122AA4094F8321021EABB
:10219000020284F8322003E00AF5967142F8251015
:1021A000B9F1000F29D1544A0321127805EB450EED
:1021B000B2FBF1F101EB4101511AC9B2714404EBD8
:1021C0004101888694F87C1029B9022A15D9404A21
:1021D000012182F87C1006206843484A111830F823
:1021E00002E0488889887044084480B24A32B0527C
:1021F00000B2032290FBF2F080B298530135023610
:1022000097E794F832203E4BB2F10F056A426A41DB
:1022100084F8962072B13B4A126850010AD4D8F86B
:102220000020D9689A60521AC82A20D9012283F85E
:1022300021201CE02B4A012151701170D8F8002098
:102240009968DA605B68521A9A4203D92C4B0022D3
:1022500083F82120002504F013FA854207DAE8B25A
:1022600004F0E4F9234B23F815000135F3E7224B82
:102270001A7801321A70194B1A689A4612F4805F64
:1022800005D0204B1B68D90701D40DF094FF174BE4
:102290003D6819680B7B002B38D0164A013B32F899
:1022A00013008B7B1BB1C0F53B60083080B200B2DD
:1022B000A0F57A70B0F57A7FA8BF4FF47A7020EA63
:1022C000E07011F021FA104956E000BFB83200204A
:1022D0008816002008000020E80F00207009002068
:1022E000943200202000002094160020280F0020A7
:1022F000540F00202E0F00202C0F0020BC160020B1
:10230000040F0020A018002000007A44DAF8002012
:1023100012043AD5D4F89800A64A281A002834DBCB
:1023200005F59C402030C2F89800A348497B4679C7
:10233000A24830F8160080B290FBF1F092F89C10A1
:10234000013101F00F0182F89C100A4482F89D00CF
:1023500018469B4A9A5C01331044102B80B2F8D186
:1023600000B290FBF3F000B26428A8BF642020EA1A
:10237000E07011F0C9F9934911F0CEFA924911F0C9
:1023800017FA11F001FC914B1880DAF80030904EEA
:1023900013F4807F00F0F0808E4B8F4F9D4203D965
:1023A000BA780AB90122BA70BA78002A00F0E4803B
:1023B000894A8A4992F821500868B5F1010EDEF188
:1023C0000005327855EB0E05C2F38008C0F3806932
:1023D0008B4635B912F0080F0CBF0022022204927E
:1023E00001E00023049397F82020052A00F2BF8023
:1023F000DFE802F0034B5E828FA8B8F1000F37D000
:10240000774A1068774A11880AF03AFD012808D106
:10241000754A64201168D4F8B020D28800FB0212FB
:102420003A61B9F1000F0BD0D4F8B02012793AB16B
:102430000DF038FB032287F820204FF47A7235E044
:10244000002D40F09480684A39691068624A8842D9
:102450000AD903920DF026FB039A032182F820107B
:1024600040F6B831D161BEE7012182F82010BAE709
:102470004FF48060B9F1000F02D00DF003FB01E0D2
:102480000DF02EFB00223A6171E0002D52D1D4F8FC
:10249000B020127A012A02D00DF004FBA3E70DF060
:1024A00001FB032287F8202040F6B832FA619AE750
:1024B00025B1052287F82020012000E02846B8F148
:1024C000000F0CD0464A1268118A484A1180518088
:1024D0009180D4F8B0104988D18003220492424AF6
:1024E00011687A69914202D8B8F1000F3CD147F2E5
:1024F0003052FA6103221EE0327842F0020232705A
:102500000DF059FE384A1168FA690A44BA6104228A
:1025100011E0354A11688DB1BA69914227D9344A20
:1025200012781AB9DBF80020D00720D4327822F0D4
:1025300002023270052287F8202054E7FA690A4423
:10254000BA6114E0284A64201168D4F8B020D28817
:1025500000FB02124FF480603A61002287F82020CD
:10256000FA700DF0BDFA3EE700287FF43CAF049B03
:1025700013B118460DF0BAF81E4FB7F8DE1007F584
:102580000D700AF07DFC05461848B7F84432B0F9E2
:10259000022003F10B01914280462DDB0B3B93425D
:1025A0002ADCB0F90020914226DB9342CCBF002305
:1025B000012322E088160020BE0D0020CE0D002051
:1025C000251700200000C84200C07F446C15002081
:1025D000DA320020404B4C00040F0020A0180020ED
:1025E000FC0E0020000F0020943200202E0F00204F
:1025F000280000205004002000239DBBA24A12683E
:10260000110114D5A14AD27812B9327852072CD4CC
:1026100000230022C4F8B830C4F8C420C4F8BC3089
:10262000C4F8C820C4F8C030C4F8CC200DE00023A2
:10263000C4F8C430C4F8C830C4F8CC30C4F8B850BA
:10264000C4F8BC50C4F8C050012384F8D030002333
:10265000C4F8D430C4F8D8300023C4F8DC30C4F84F
:10266000E03004E0002384F8D03084F8B4303378CC
:10267000580741D5DAF80030D9063DD5844B1B7890
:10268000DA0639D4834B93F80090B9F1000F10D0DB
:1026900097F88932ADB96BB17F4B1A68D4F8E43042
:1026A0009B1A002B06DA0DF086FD7C4B83F8E85070
:1026B00022E0CDB910200DF019F8012384F8E8309C
:1026C0001AE03BB1744A4FF47A71126801FB03239C
:1026D000C4F8E43094F8E83073B10CF0F3FF6F4BBA
:1026E000002283F8E82007E094F8E83023B10CF0EA
:1026F000E9FF6A4B83F8E890002297F88812B7F850
:1027000046E2B7F848C2134638F902009B08704504
:10271000C4BF63F07F03DBB202326045B8BF43F051
:102720004003082AF0D194F8E9005C4A984205D1A8
:1027300092F8EA00F92804D8013000E0002082F87D
:10274000EA0084F8E930534B544A1878DFF838919E
:102750009B4618BBD9F80030DB0708D582F8EB00A0
:10276000E5B93378DD0719D510F07CFC16E0337835
:10277000580713D592F8303083B1444BDB786BB9EE
:1027800092F8EB300133DBB2032B82F8EB3005D942
:1027900011B10DF010FD01E0002DFAD094F8EA30EF
:1027A0003E4D142B40F08C809BF800309BB195F887
:1027B000E9305F2B0FD1337803F0040303F0FF02FD
:1027C00013B10DF0F8FC06E00B2003920CF08EFF25
:1027D000039A85F8EA20337803F0040303F0FF003E
:1027E000002B6DD194F8E9302C4A572B13D12C4B88
:1027F0004FF47A721B68B2FBF3F3C3EB431203EBA3
:102800008203284ADB001380274B1B685B0757D5E0
:102810000A22264B35E0DAF800104D0717D55A2B5F
:1028200015D192F8EC302BB1012382F8EC0082F83C
:10283000ED3045E092F8EE3083F0010382F8EE309F
:102840000BB10C2000E00D200CF050FF38E05D2BA8
:1028500000F0DC855B2B00F0DB855E2B02D10320D2
:1028600000F0D7BD562B01D10EF0E6F99BF80030F1
:1028700003BB94F8E930972B40F0D1850C4B4FF413
:10288000C8721A801CE000BFA0180020040F0020AE
:10289000B90D002028000020943200208816002066
:1028A00058140020D4320020100E0020D632002010
:1028B0006214002094F8E9306F2BDAD110F0D2FBCB
:1028C000DAF80030580737D594F8EE30B74A93B1AC
:1028D000337859070FD5B8F90610B7F84632994240
:1028E00009DDD9F8003013F0010304D13221A2F838
:1028F000F01082F8EE30D9F8003013F4803FAB4B83
:102900000CD094F8F2202AB993F8EC2012B93222B4
:10291000A3F8F020012384F8F2300DE094F8EC20C5
:1029200052B1327802F0040202F0FF0122B9012212
:1029300083F8EC1083F8ED209D4D0023C9F800309A
:1029400005F1500B2A786B7815F8010C9A420CD2DD
:1029500029460CF03DFB40B115F8023C01229A409B
:10296000D9F800301343C9F8003004355D45E9D18A
:10297000904B1B7853B1904DDFF858B22B68DFF8BD
:10298000589213F0020F40F0F581ECE1DFF84C9221
:10299000A9F15A0595F8AA2495F8AB3495F8A9043D
:1029A0009A422ED205F2AA410CF012FB48B395F8D8
:1029B000ACE495F8AE040EF1FF3E804B0EEB4E0EEC
:1029C0004FF00C0C73440CFB00FC0493774B059008
:1029D00003F1F40B0BEB0C025168049895F8ADE48D
:1029E00081420ED000210BF80CE0916005995060F7
:1029F000012202FA01F093F8242122EA000083F870
:102A0000240106354D45C5D16D4B94F830201D6825
:102A10006C4B4FF000091B68079206936A4BCDF888
:102A200014900493049A1368002B00F0928193F899
:102A30000090B9F1000F00F08C8152680698821A5C
:102A4000002A0CDB049900F5FA7205984A6001220D
:102A5000824094F8241121EA020284F82421079A82
:102A6000002A00F076810498597810F8042C04327A
:102A7000D2B2002940F03681544938F91220B1F819
:102A8000441201F1C800824202DD93F802B015E061
:102A9000C8398A4203DA9B78C3F1000B0EE0059A2D
:102AA0000123934094F8242122EA0303069A84F830
:102AB000243102F5FA73049A53604AE1059B94F8B5
:102AC00024211A41D30700F14481BBF1000FCCBF90
:102AD000022001200CF0BEFF09F1FF32132A00F2A0
:102AE0003081DFE812F01400250036004A007D0036
:102AF0008400A100BD00D900E500F3002E014A00CA
:102B000059008400A100BD009500B100CD0095F8EA
:102B100000902846D944B9F1FA0FA8BF4FF0FA093E
:102B200029EAE97985F8009007F04AFD012022E0C2
:102B300095F801902846D944B9F1640FA8BF4FF029
:102B4000640929EAE97985F8019007F039FD022046
:102B500011E095F803901E4BD944B9F1640FA8BF5A
:102B60004FF0640929EAE97985F803902846196845
:102B70000AF0F8F803204946A5E069790D20594488
:102B80006429A8BF642121EAE17169710AF028FE75
:102B9000B9F10D0F00F0D58029790E205944642930
:102BA000A8BF642121EAE17129718CE08816002018
:102BB000AB080020DC320020A018002020A901086A
:102BC000901900209432002080170020500400202B
:102BD0009C150020100E002014180020AA040020CC
:102BE000A9790520594481F30801A9716BE0AA4A2B
:102BF0000F20126891785944C829A8BFC82121EA3A
:102C0000E17191700AF0ECFDB9F10F0F00F09980BD
:102C1000A14A1220126851785944C829A8BFC82176
:102C200021EAE17151704EE09B4A10201268117B3D
:102C30005944C829A8BFC82121EAE17111730AF0DB
:102C4000CFFDB9F1100F7CD0934A13201268D17ACE
:102C50005944C829A8BFC82121EAE171D17232E0E4
:102C60008D4A11201268917D5944C829A8BFC821F6
:102C700021EAE17191750AF0B3FDB9F1110F60D04D
:102C8000854A14201268517D5944C829A8BFC8211B
:102C900021EAE171517516E07F4A09201268D17866
:102CA0005944C829A8BFC82121EAE171D1700AE0BE
:102CB000794A0A201268517B5944C829A8BFC82103
:102CC00021EAE17151730AF08BFD3AE0724A0B2060
:102CD0001268D17D5944C829A8BFC82121EAE171F1
:102CE000D175F0E701292CD138F912209978B2F585
:102CF000617F05DB40F633039A42B8BF134601E01B
:102D00004FF46173B9F10C0F1BD14FF4966292FB33
:102D1000F1F2A3F5617393FBF2F3604ADBB292F830
:102D200025219A420DD0184602930AF08DF8029B95
:102D3000484619460AF054FD029B581CC0B20CF0DC
:102D400089FE059A0123934094F82421134384F8C3
:102D50002431059B049A01330C32042B0593049211
:102D60007FF460AE07E6DAF80030D80511D54C4B99
:102D7000DB7873B1DBF8003099070AD5B9F8003079
:102D800013F001030AD1012002930CF07BFE029B99
:102D900005E001200CF0A4FE012300E000232A68D6
:102DA00052070BD553B101200CF09AFEB9F8003050
:102DB000980706D402200CF065FE02E002200CF019
:102DC0008FFE384BB9F8002099689B8912F0030FE9
:102DD00014BF4B610B61DBF8003013F00A0F2CD0ED
:102DE0002B68D9060DD552070ED404200CF04AFEEC
:102DF0002D4BB3F904200A2392FBF3F22B4B1A80DC
:102E000002E004200CF06CFE2B689B0607D5B9F895
:102E10000030580606D440200CF034FE02E040207A
:102E20000CF05EFE2B68590607D51F4BB3F9042042
:102E30000A2392FBF3F3A4F826312B684FF4807039
:102E40001A0502D50CF01EFE01E00CF049FE184AEE
:102E50005379082B01D00E2B04D1402003920CF0A3
:102E60003FFE039ADAF800305B0527D592F8CC32A2
:102E70001BB9337813F0040F02E02B6813F4002F12
:102E800018D0002384F828313C200FF03BFBA8B178
:102E900003F038FCF8E700BFA015002088160020DA
:102EA000040F002074090020361800203C18002070
:102EB000500400200AF04CFB10F05AF8A64B0122F7
:102EC0001A70A64B1A781E46FAB1DBF80030580784
:102ED0001BD52B68190703D408200CF001FE14E061
:102EE000B9F8004004F00804A4B274B908200CF04A
:102EF000C9FD9B4B1A689B4B1A609B4BB8F8062088
:102F00001A809A4B1C609A4B1C6033780BB3DBF829
:102F10000030DA061DD52B689B0204D44FF40070F4
:102F20000CF0DEFD15E0B9F8004004F40074A4B222
:102F30007CB94FF400700CF0A5FD894B1A68894BE1
:102F40001A60894BB8F806201A80884B1C60884BA1
:102F50001C60884BB8F90600D3F800C0BCF80A30F2
:102F6000984211DBB0F5FA6F9CF8078009DAC21AB3
:102F700002FB08F8A3F5FA6398FBF3F808F164087C
:102F800004E0C8F1640801E04FF0640897F82232C9
:102F900097F82342049397F9D83100219BB2089304
:102FA000754BB7F844B21B68059407931E460A4652
:102FB000724B40F2E634CB5E0693CBEB030303F295
:102FC000F315A54203D8002BB8BF5B4201E04FF4D4
:102FD000FA73022A6A4D4FF0640436D0049F27B179
:102FE000BB42CCBFC7EB0303002393FBF4FA6FF0A3
:102FF000630909FB0A3905EB4A0705EB4A0ABAF9E6
:103000002CA1B7F82A71CDF824A0CDF80490DDF8F2
:1030100024900FFA87FACAEB090ADDF804900AFB3C
:1030200009FA9AFBF4FABA44564F21F807A00CEBC0
:1030300002073F797B43544F93FBF7F364339BB212
:1030400008FB03F393FBF4F42BE0059F27B1BB428D
:10305000CCBFC7EB0303002393FBF4F46FF06309C9
:1030600009FB043A05EB440705EB4404B7F9387152
:10307000B4F93A41002BB8BF5B42E41B04FB0AFAE7
:103080009AFBF9FADDF82090C7EB0A0707FB09F76E
:103090003C4CA7809CF806403B4F5C4394FBF7F404
:1030A0006434DDF81C90364B914499F801A04FF040
:1030B000640904FB0AFA03F5A3779AFBF9FA02F80C
:1030C00007A096F80BA003F2491704FB0AFA9AFB33
:1030D000F9FA02F807A096F815A003F5A67704FB05
:1030E0000AF4022A94FBF9F4D4551F4616BF03F2E2
:1030F0004F1383F8519102F80380069B214C5B45E6
:1031000002DA635A5B4263520231062902F101027C
:1031100006F101067FF44CAF1C4BDFF874801B688E
:1031200013F4805C0ED0B0F57A7F06DBB0F5FA6F51
:10313000B4BF03464FF4FA6301E04FF47A73A3F58A
:103140007A7330E0B8F84632984223DBB0F5FA6F74
:10315000A8BF4FF4FA601EE01818002034180020B1
:103160005C180020581800204C180020501800202F
:103170004418002090190020401800202E0F002035
:10318000881600201C1800200CFEFFFF700900208C
:10319000500400201846C01A4FF47A725043C3F509
:1031A000FA63B0FBF3F3642693FBF6F207EB4201FC
:1031B0006FF0630000FB0233B1F8521107EB4202DB
:1031C000B2F954010AB2821A534393FBF6F30B444B
:1031D0009BB2E380BCF1000F16D0AF4A1268960094
:1031E00012D5AE4AD2787AB9A3F57A7212B2CBF57B
:1031F000FA6112034FF47A7009B292FBF0F24A437B
:10320000A74B0BEB2232DA80A64BB3F800A00AF0F2
:10321000400A1FFA8AFABAF1000F44D0A24BB3F960
:1032200004000A2390FBF3F0B5F82631C01A00B26F
:1032300010F06AFA9D4910F0BBFA9D49054610F05E
:10324000AFF907F042FF0646284607F03EFF054665
:10325000B4F9020010F058FA8146B4F9000010F0F9
:1032600053FA3146834610F0A3FA294603464846EE
:10327000029310F09DFA029B0146184610F08EF959
:1032800010F05CFC31462080484610F091FA294647
:103290000646584610F08CFA0146304610F080F988
:1032A00010F04CFC608098F84B0200285BD0BAF11B
:1032B000000F58D197F86A317E4E83427E4D12D06E
:1032C00086F86A0110F020FA784910F071FA78490E
:1032D000804610F065F907F0F8FE6860404607F098
:1032E000F4FEC6F86C01B4F9000010F00DFA0646C1
:1032F000B4F9040010F008FAD5F80480814641467C
:10330000304610F055FAD7F86C51824629464846A7
:1033100010F04EFA0146504610F040F910F00EFC45
:10332000DFF8C4A1B0F5FA7FA8BF4FF4FA7050459A
:10333000B8BF504641462080484610F039FA294629
:103340008046304610F034FA0146404610F028F925
:1033500010F0F4FBB0F5FA7FA8BF4FF4FA705045B7
:10336000B8BF5046A080554B1A78550704D5544B2A
:103370001A689B88536142E047490968CC0702D527
:1033800097F8701111B142F001021A704D4A12788B
:10339000100703D41A7822F001021A704A4A126800
:1033A000510702D54949098881B94949098809B1B4
:1033B000920705D4474A1288003218BF012200E064
:1033C00001221AB944490988642907D9022287F8D9
:1033D00071211A7822F001021A7007E01B78DB07CE
:1033E00056BF022387F8712187F8713107F042F93F
:1033F000D7F87431C01A002801DB03F05BF9374BB2
:103400009B68002B7CD03648984779E0012000E08B
:1034100002200138C0B20DF0D7FBFFF751BAA72B3D
:1034200006D1284B1A7842F004021A70FFF748BA06
:103430000022BB2B0B9201D1022303E0B72B04D156
:103440004FF6FE73ADF82E3009E0BE2B01D10223FA
:1034500003E0BD2B18D14FF6FE73ADF82C30BDF84C
:103460002C20B7F8F0311344A7F8F031BDF82E2026
:10347000B7F8F2311344A7F8F2310DF0DDFB002369
:1034800084F8EA30FFF71CBA792B2FD1154BDA7884
:1034900022F0010231E000BFA0180020040F00203C
:1034A0001C180020141800203618002035FA8E3C15
:1034B000DB0FC93F8816002020000020DA320020F0
:1034C00074090020B90D0020100E0020D632002013
:1034D00062140020D4320020101800202C0E00208E
:1034E00000180020040E00200CFEFFFF7A2B7FF452
:1034F000E7A9054BDA7842F00102DA70FFF7E0B98C
:103500000DB0BDE8F08F00BF040E00202DE9F04F94
:10351000934BA1B01B68934C9F6A07F0ABF82568EA
:10352000914B401B85B21D8007F0A4F88F4B2060A3
:103530001A78012A02D1A389A580E3808C4E19A8AC
:10354000F36898479DF8643023B1A37B002B00F00B
:103550002E830AE007F08EF8864A23681268FB1A69
:10356000184450329042E9D3EFE709F0EBFD08B977
:1035700009F0C6FC804D95F84A3213B9238A002B16
:103580004DD07E4B227D19887D4B1B68B1FBF3F13A
:1035900001F1010C1FFA8CFC724BA4F812C00AB3A3
:1035A000B3F916B000236F4A0FFA8CF902F1200E1E
:1035B00033F90EA002F118000BFB0AFA1F5A02F1B0
:1035C000280033F800809AFBF9F9C8EB0708C144DA
:1035D00023F80E901F520233082BE4D100231375F9
:1035E000D18202E0DA8A013ADA82B4F916105D4A31
:1035F00000294FF0000311DDB2F912E0614A02F137
:103600000800185E02F110074843DF5B90FBFEF0F4
:10361000381A98520233082BF0D100E0D3820123EC
:1036200084F83030584B4F4A1968534E11F0080F48
:1036300037D0908B00F10E039BB21C2B2BD8138A32
:103640005B0728D5B2F936700A2397FBF3F7138F7F
:10365000FA1A92B293B21FB2B337BCBF02F5B47379
:103660009BB24A4F1AB2B32A3F78C4BFA3F5B473D2
:103670009BB23F0796F8D82113D552B2524253431A
:10368000E26B1BB2527A53436FF01D0293FBF2F3CD
:103690001844A08305E0B4F936200A2392FBF3F323
:1036A000238711F0140F00F08C80228A2D4B02F436
:1036B0000272002A00F08580344A127802F010026B
:1036C00002F0FF073AB1598B96F996021A6C00FB8B
:1036D00002125A8375E05A6C2D48D178927841B322
:1036E000B3F94810B0F90600C1EB000EBEF1000FAF
:1036F000B8BFCEF1000E96450DDDDF6488424FF075
:103700000107C8BF524283F85070DB8BC8BF92B22A
:103710001A44E28355E093F850201AB19A6D83F869
:1037200050705A65236CE26D19441388528899428F
:1037300041E0B3F94870B0F90600C01B80EAE07EB2
:10374000AEEBE07E964527DD022290FBF2F0114AB7
:103750001060012283F8602083F8502025E000BF2C
:10376000C414002004180020D83200206C09002066
:103770002C0E002058140020500400209C0F002024
:103780005C1400201C180020100E0020B90D002031
:103790002E0F0020BC32002093F850202AB1986DE3
:1037A00083F86010586583F85010E16D226C0B8827
:1037B0003A4449889A4203DB8A42B4BF13460B4617
:1037C000E383A34B1B78ABB1A24BB3F90620B6F849
:1037D00046329A420EDCA04B5B79012B01D0192BAB
:1037E00002D196F890222AB90E2B03D0082B1CBFC9
:1037F0000023A38396F810728FB3238ADFF8C49254
:103800009A072CD0D9F884B094495846B9F81E804C
:1038100010F076F9F8B9584613F0BAFCD9F88810C8
:103820000FF0C6FF13F038FCB0F5617FA8BF4FF46E
:1038300061700FF069FF8A4910F06EF807F045FCDF
:10384000814638460FF060FF49460FF0B1FF13F094
:1038500023FC80B200E000208044A4F81E80814B4D
:103860001878002840F0A1817F4B1A68994612F41D
:10387000002F00F09A817D4F3B78033B052B1CD82D
:1038800096F8053533B1012B09D10EF06FF8C0F170
:103890007F0004E0D4F88C0003689B689847744A62
:1038A00094F8901013680B44B3F5807FA8BF4FF4D1
:1038B00080738342D4BF136010603B78023B092BB6
:1038C00000F26E81DFE813F00A00140047006C017B
:1038D0006C015F0071001F0142014E01644B002228
:1038E0001A60644B1A60644A12685A60032356E1F6
:1038F000614B19685F4B5A681E466432914240F230
:103900004F8140200CF078FA002840F04981402592
:103910005A4A3368DFF85C91D05C924670B10CF083
:10392000ADFA534A013D136803F1FF331360D9F830
:10393000003003F10103C9F80030E9D132684D4B82
:103940001AF80220002A40F02B811A604FF0FF3253
:103950005A60042323E12A230093494B492003F1B1
:103960000C02019302925021A3F10A0202330CF0DF
:10397000ADFA002840F014813E4B4FF0FF32186042
:103980005A6007230BE13F4A052300210093019170
:103990000291532002F108030CF098FA002840F03D
:1039A000FF80344B18600823F9E040200CF024FA23
:1039B000002840F0F5802F4A136890460C2B00F247
:1039C000DE85DFE803F0070B0E1218292D3135399B
:1039D000818B8F002C480CF06EFC8EE02B482C491C
:1039E00017E02C482C492D4A85E02D4896F8031500
:1039F00096F804257FE095F858345C225343EA1882
:103A000092F8D4230C2101FB02331D44254895F87C
:103A1000D6130CF050FC70E02348B6F8D010F8E74D
:103A20002248B6F8D210F4E7214A22481169F0E79B
:103A3000214B22481988ECE7D4F89430DB0403D5F5
:103A40001F4896F81212E4E70B23136055E000BFFD
:103A5000280000202E0F0020500400208FC2753C4B
:103A6000EFB6B044DC320020700900206014002062
:103A7000D4140020CC140020943200205CA901084A
:103A8000C6A90108B4AB010833C401084DC401083C
:103A90005DBF010862C4010848BF010854BF0108A6
:103AA00076C4010887C4010891C40108A0C40108B4
:103AB0002C0E0020AFC4010806000020BFC401087E
:103AC000C9C4010804180020AD4896F8161296F8EB
:103AD000172296F815320CF0EEFB0EE0A948B4F868
:103AE000981096E7D9F800301D0506D5A648B6F817
:103AF0001C12B6F91A220CF0DEFBD8F800300133A4
:103B0000C8F800304CE0D4F89C20A04B90011AD5A6
:103B1000B3F8A020BAB9D3F8A4609D4B45201D6826
:103B20000CF0ACF90E200CF0A9F930460CF030FB8B
:103B300028460CF02DFB974B4FF480521A800A2335
:103B40003B7004F029FF07F041FB29E094F8A8300E
:103B5000002BF6D08D4BD3F89C309901F1D409237A
:103B60003B70F0E78C4B1A688C4B5B68C8339A4209
:103B700003D996F805558DB904E00CF06DF90028CD
:103B8000F7D10DE0D4F88C0006F0C8FC94F8A93009
:103B9000C4F88C50022B01D10FF0EAF901233B70DD
:103BA00004F01CFC08B101233B700023A3737C4884
:103BB00011AD436828469847002800F02A817949CA
:103BC000794A08780023032802D15168774E995327
:103BD000E95E0233062B42F8041FF4D16B4D94F8D2
:103BE000B82005F1AC00014602F04EFCD4F8BC60F0
:103BF000002130460FF070FF80B16D4B6D4F1A8879
:103C0000984607F1D009002A00F0FA80D4F8303144
:103C100007F188051B780026099348E095F8C05005
:103C200095B9654B1A68984672B1584F304607F1FE
:103C3000C4012944D8F80020243507F027F86C2D5A
:103C4000F3D1012387F8C03094F8C030002BD4D0D2
:103C50000025584EA8590FF057FD05EBC50306F196
:103C60001801194407F09CF813F016FA7051043546
:103C70000C2DEED1C1E79A59B85902449A510FF070
:103C800043FD2A690132012A2A6125D10023686097
:103C90002860AB600023BAF1010FBB5149F8063030
:103CA00046D004360C2E05F1140500F09E80424BE0
:103CB0004FF47A721B68B8F800A0B2FBF3F3C3EBC1
:103CC000431203EB8203DB009BB29A453B4BD2D1FC
:103CD00000229A512A61CEE7D5F800C007926146CA
:103CE000CDF814C006900FF059FC079A8346104691
:103CF0000FF00AFD014658460FF00EFEDDF814C025
:103D0000014660460FF04CFC069B02461146686077
:103D1000184607920FF042FC014658460FF048FD46
:103D2000A9680FF03DFC079AE8602A60A860B1E737
:103D30002869012807DD01380FF0E6FC0146E86834
:103D40000FF0EAFD00E0002013F0FCFB099A834627
:103D5000DFF864A0A2B310460FF0D6FC0146584627
:103D60000FF0E2FE60B3DAF800304FF47A72B2FB83
:103D7000F3F3C3EB431203EB8203DB003EE000BF2F
:103D8000D6C40108EFC40108FAC4010804180020D1
:103D9000B8320020C814002094320020CC14002037
:103DA0002C0E00206C090020AC1800200818002000
:103DB000D4320020B01800205814002074190020BC
:103DC000DAF800304FF47A72B2FBF3F3C3EB43122C
:103DD00003EB8203B34ADB00B2589BB202EB5302FF
:103DE00092FBF3F349F806305BE7B8F800000128CE
:103DF00001D10BF07BFCB8F80030013BA8F8003093
:103E00000023F95859F803208A1AFA5004330C2B6E
:103E1000F7D194F8883123B1A34A013B82F8883165
:103E2000B9E3A24D0021D5F8E0010FF055FE20B90D
:103E300095F8E831013BDBB200E0012384F88831DA
:103E40009B4B9C49B5F8262200930D68443BE06BE0
:103E5000D4F88C11A847984B934EDB780D93974B71
:103E60001D78032D16D9D6F890315A88B2F5FA7F0D
:103E700010D2B6F91C00B6F998110028B8BF40421C
:103E800053421B1A994203DB13188B42A8BF0B46FF
:103E9000A4F898318A4B1B6893F807B0BBF1000F68
:103EA00021D0884A1268920719D5874A1278012AC8
:103EB00011D9DB78B4F89A115A43D31A994290B2C7
:103EC00003DB8A42B4BF13460B4602B212031BB295
:103ED00092FBF3F301E04FF48053089303E04FF4B7
:103EE000805ECDF820E0D4F89031B4F89421B4F895
:103EF00096C1B4F99891754C0A93754E23780024B5
:103F000009920DF14A08A2462746AF4251D20FFA54
:103F10008CF00693CDF814C00FF0F6FBB1680FF0EB
:103F200047FCDDF824E002460FFA8EF007920FF00E
:103F3000EBFB71680FF03CFC079A014610460FF04E
:103F40002FFB0A99024691F900000792404209FBB3
:103F500000F00FF0D9FBF1680FF02AFC079A014638
:103F600010460FF01DFB0FF0E9FD069B80B2DDF857
:103F700014C0BBF1000F03D0089A00B250430013E5
:103F8000A8F8020038F8022F0FFA8AF011B2814225
:103F900004DC20B28142B8BF144600E09246052BF3
:103FA00004D1042F9CBF4B4921F81720013710364C
:103FB000ABE74448C4EB0A040368A4B213F4805F7F
:103FC000394E3BD0444B1B785F0704D4D6F8A03160
:103FD0001B8AA6F89C31D6F8A021D6F8A411F78B3D
:103FE000B2F81080B1F806C00FFA87FECCEB0802D9
:103FF00096452D4B05DC0A88D3F8A811B1F800903E
:1040000007E0C444E64507DBD3F8A821B1F80290E5
:104010005288A3F89C7117E0B3F99C71974206DCB3
:104020000A88D3F8A8311746B3F800900CE0D3F80B
:10403000A831B1F802905A884F4605E0D6F8A83169
:10404000F78BB3F800905A8892B21FFA89F9C9EB3E
:10405000020123B209B28B4240DD012286F8AC2175
:104060000A0392FBF3F20DF14A03C6F8B02103EB09
:10407000450E734508D0B3F902C002FB0CFCCCF32B
:104080000F3C23F802CFF4E7022391FBF3F10F4B2F
:1040900089441B781FFA89F9062B2DD1022D2BD8C4
:1040A000F48029E074190020041800205004002036
:1040B00084060020D4030020040F0020840C00207C
:1040C0006414002070090020C00000206C0900204A
:1040D000880C002008180020DA3200204FF0020A75
:1040E00093FBFAF399440021D31A86F8AC111FFA16
:1040F00089F91FFA83FA00E0CA460368B6F99C41C1
:1041000003F4805C03F010030E93AF4BD6F8A88144
:104110001B78D6F8A02103F00403DBB20A93D6F88B
:104120009C30D6F8A4B103F000630B93A74B09941D
:10413000B3F9063000240C936B000F930F9B9C4245
:104140005BD013ABE35A38B20792CDF814C0089392
:104150000FF0DAFA9E4B53F834100FF029FB0FF0F2
:10416000EDFC0FFA89F39842079ADDF814C004DBDE
:104170000FFA8AF39842B8BF0346DDF820E095496C
:1041800073440D989BB263521BB210B1B8F804008F
:1041900016E0BCF1000F11D0B2F810E0BBF8060039
:1041A000C0EB0E00DDF824E0864504DCB8F8000022
:1041B000BBF800E006E0BBF8020001E0B8F8000040
:1041C000B8F802E0834203DB7345B4BF184670467B
:1041D0000E9B08537BB10A9B6BB1BCF1000F0AD157
:1041E0000B9B43B9538ADDF830E09E4503DAB8F8FB
:1041F0000410784BE1520234A0E7734B1A7802F0B6
:10420000040202F0FF033AB1734B1B78013BDBB2AF
:10421000182B00F24E810AE0AB42F5D26D4A02F152
:10422000180131F8131022F813100133F4E70122BA
:104230009A406A4B1340002B00F03B81684B1A8A6E
:1042400012F4807F614A07D0198BADF86410598B46
:10425000ADF86610998B17E0B3F894116148ADF88A
:104260006410B3F896110068ADF86610B3F89811B1
:10427000C004ADF8681009D5D3F8A001B2F9064022
:10428000008A844202DA4942ADF86810B6F9344037
:104290004FF47A7004F5E16444434FF4616194FB98
:1042A000F1F4A4F5FA74ADF87C40B6F9324004F5A7
:1042B000E164604390FBF1F1A1F5FA71ADF87E1075
:1042C000B6F8B4111088A1F2DC51ADF86A10D6F836
:1042D000A011098A401AADF86C005088401AADF858
:1042E0006E009088401AADF87000D088401AADF882
:1042F00072001089401AADF874005089401AADF868
:1043000076009089D289401A511AADF87800ADF83C
:104310007A1000223448002111520232102AF9D1B9
:10432000D3F89C40D3F8E43108940A932F4B1B78C0
:104330005B0009930B46099DAB4200F09F802C481F
:104340000A1894793CB10125153405FA04F4089D46
:104350002C4000F08E80455C0A980E2707FB05076D
:10436000B7F90000B7F9026092F904B0361AB6B294
:1043700006FB0BFB64209BFBF0FB92F801904FEADD
:10438000560892F803C0C8EB0B0B1FFA8BFB92F890
:1043900005A018484FEA490E20ACBCF1000F03D12C
:1043A000744434F81C4C0CE0A6443EF91CECC45E8A
:1043B000744521DAA444A44503DBE645B4BF744642
:1043C0006446C45223E000BFDA3200202E0F0020E2
:1043D000880C0020B8190020840A00209920980138
:1043E0000418002070090020940A0020480D0020C5
:1043F000490D0020EC19002009DDCCEB040CF4453C
:1044000003DBA445B4BFE646A64620F803E04FF020
:10441000010E0EFA09F9D7F80A7092F9022019EA8A
:10442000070F0CBF77464FF0FF37DFF874E15B48AA
:1044300033F90EE00FFA8BFB02FB0EF24FF0640E25
:1044400092FBFEF25A4530F81540BFB20CDB4FFA32
:104450008AFB06FB0BFB9BFBFEFBC8EB0B0B0FFA6F
:104460008BFB9345A8BF93460BFB074B20F815B079
:1044700001E04B4A9C52023307315CE7494B002470
:10448000D3F8E48125460E2303FB0583434E93F9BD
:104490000630A75FE8B25F43642397FBF3F7A753A7
:1044A00006F086FA01353844082DA05304F10204C1
:1044B000E9D13D4B3B4C1B68384D13F0200F2ED0FB
:1044C000002006F075FA28800646012006F070FAF2
:1044D000D4F89C3068801B0621D5D4F80832B4F992
:1044E00032201B78B4F93470012B1CD1D4F8E4319C
:1044F00093F9141093F906304A435B425F4332212B
:1045000092FBF1F26FF0310392B297FBF3F3134495
:1045100097FBF1F71E443A442E8010446880D4F88B
:10452000E461002314E0D4F8E41191F9063091F924
:1045300014105F434A43322397FBF3F73E4492FB48
:10454000F3F32E801844E9E7EA520233102B0ED021
:10455000C3EBC3003044B0F90020E95EB0F90200BB
:104560009142F1DB02B29142B8BF0A46ECE708F093
:10457000E9FD08B108F0C4FC0123A3730BE00BF0C4
:104580006BFC00283FF40CAB084B4FF480521A80B0
:104590000A23FFF704BB21B0BDE8F08F940A002086
:1045A000EC1900200418002070090020C814002015
:1045B0002DE9F04F87B008F0CBFF914B1D78002D0F
:1045C00040F0D5858F4F3B68580540F1D0858E4B24
:1045D0008E4CB3F8DE9023788D4E002B00F0908146
:1045E000336862689A1A7C2A40F28A816360237A6F
:1045F0000133237205F12400C0B206F07BF9854B2C
:1046000053F825000FF080F8834B804618880FF090
:104610007BF8014640460FF07FF980490FF0C8F85B
:104620000FF08CFA013500B206F090F9032DE1D1BC
:10463000302006F05FF97A4BDFF8D081B3F9000043
:1046400006F084F906F064F9237A990733D1D8F893
:10465000043041F2883293421AD9102006F04AF908
:10466000D8F80C00642590FBF5F000B206F06EF966
:10467000212006F03FF9D8F80C3093FBF5F005FB4C
:10468000103585EAE570A0EBE57000B206F05EF942
:10469000142006F02FF9634BB3F904000A2390FBB2
:1046A000F3F006F053F91C2006F024F9002006F080
:1046B0004DF906F02DF9237A5A0740F0FE800220CA
:1046C00006F018F9514B4FF0050818696423323091
:1046D00090FBF3F000B206F039F9534B0320B3F925
:1046E000065006F007F9514B95FBF8F51B78ADB273
:1046F0005B070BD54E48494608F0C2FB20B93B6822
:1047000013F0100F18BF002528B205E0494B1B68B5
:10471000DB89B3FBF8F000B206F018F93B689807A4
:1047200040F19980DFF81C81434D98F800202B88D8
:10473000642101FB0323B4F8149052004FEA0919D5
:10474000B3FBF2F31FFA89F949EA03291FFA89F941
:10475000C3F3032349EA0309062006F0CBF80FFA56
:1047600089F006F0F3F8A28A98F80030013292B28C
:1047700092FBF3F103FB1122A282304A1268917B73
:10478000012905D1392006F0B5F8B5F9000020E07F
:1047900029886E254D43D27B152195FBF1F5ADB2ED
:1047A0000AB195FBF3F53A204FF0640906F0A2F840
:1047B000B5FBF9F80FFA88F006F0C8F83B2006F0D0
:1047C00099F809FB185080B205300A2390FBF3F0EA
:1047D00000B206F0BBF8282006F08CF8184B1868D9
:1047E0000A2390FBF3F000B206F0B0F8042006F0C4
:1047F00081F8104B1B68DB8933B30AF06DFB27E0AF
:10480000DC3200207009002050040020101A002023
:10481000943200204C1500200600002000007A444D
:1048200064150020361800201C180020DA32002001
:1048300084060020641400209E190020D01300205C
:1048400070150020C0000020A84B186880F31000ED
:1048500000B206F07BF805A9A54806F0D5FC1320A8
:1048600006F048F8BDF9140006F070F81B2006F0B9
:1048700041F8BDF9160006F069F8232006F03AF871
:104880004E2006F063F805A9994806F0BDFC1220F9
:1048900006F030F8BDF9140006F058F81A2006F0BA
:1048A00029F8BDF9160006F051F8222006F022F88A
:1048B000452006F04BF806F02BF8237A282B1FD161
:1048C0008C4B002235681A724FF47A73B5FBF3F9FA
:1048D00017203C2506F00EF8B9FBF5F8B8FBF5F00B
:1048E00005FB1080000200B206F030F8182006F038
:1048F00001F805FB189000B206F028F806F008F859
:10490000A37D7C4D002B00F0B18005F0B3FEAB69B8
:10491000794AC31A9342804635D9784B00229A705F
:104920001A71774A4FF47A701288D1B2120A9977C5
:10493000DA7719755A753168EA698A1A714909680E
:10494000097C41438A420BD36F4A1268EA616F4A7D
:104950001278013A012A03D810229A7002221A71A1
:104960006B4AC4F8188011680A2291FBF2F119779A
:10497000091259775D49096891FBF2F283F820200A
:10498000121283F8212094F820A05A4DBAF1000F9A
:104990000ED1A86A05F0F6FE012809D90228DFF831
:1049A000789100F0968305F001FF012389F800302B
:1049B000E06A504B002859D093F820203AB15A6B46
:1049C00040F6B731C2EB08028A4215D84EE0012208
:1049D00083F820204F4A986A12681278022A04D875
:1049E0000430022108F090FE02E0022105F0B0FE42
:1049F000002384F8383037E093F830209AB9DA622F
:104A000083F82020434A986A12681278022A04D850
:104A10000430012108F078FE02E0012105F098FE43
:104A200005F0C4FE20E0013AD2B283F8302093F8BA
:104A3000381093F839E042B94A1C0EF1010E83F8A0
:104A4000382083F839E0986A0CE0024612F8015BDE
:104A50000EF1010E2944986A83F83810DA6283F85F
:104A600039E0294605F0B0FEC4F8348094F83A30B5
:104A7000D6F800801F4A002B00F04981D36B33B178
:104A800092F84030013B012B8CBF00230123D90752
:104A900040F13D81E06B174D05F074FED0B1E86B3D
:104AA00005F06BFE95F8413081467E2BD6F800A0CC
:104AB0000DD102231B2885F8403008D1E86B05F0A2
:104AC00061FE20B90123C5F844A085F8483084F878
:104AD0004190DFE732686B6CD31A41F6583293424B
:104AE0003FD9032385F8403011E100BF681500204D
:104AF00080969800101A00203F0D0300E513002057
:104B00009E190020DC13002094320020681400203D
:104B100070150020E01300202C00002093F84910AD
:104B2000A24A32F8110018B983F849004FF4036023
:104B300094F84930B0F5826F03F101039C4D84F87D
:104B4000493000F0C28067D8B0F5007F00F0968051
:104B500016D8B0F5807F00F09980B0F5887F00F01E
:104B6000A28094F84820924B002A00F0D08032684E
:104B7000C8EB0202012AD1D9002283F84820C6E0FE
:104B8000B0F5047F61D0B0F5806FEAD195F84A3076
:104B900042F210710133DBB2032B88BF012385F889
:104BA0004A3094F84A305943824B1B78D80748BFA3
:104BB00001319A0748BF02315D077F4B48BF04317E
:104BC0001B88D80748BF0A319A0748BF14311D0611
:104BD00048BF2831D80548BF28315A0748BF64313B
:104BE0001D0748BFC831980548BF01F5C8719A062E
:104BF00048BF01F57A71DD0648BF01F5FA61580634
:104C000048BF01F57A614FF4806005F03FFE684BC4
:104C1000002283F84820A4E7B0F5E26F51D008D80D
:104C2000B0F5C06F39D0B0F5E06F9AD1634B196819
:104C300049E0B0F5046F3ED0B0F5116F55D0B0F536
:104C4000E46F8ED15D4B99683DE03B689A0788D54B
:104C50005B4B1B68DA7B5B4B2AB11A885A4B1B787B
:104C600092FBF3F300E01B880A2159434FF40470D0
:104C700005F00CFE002384F8483072E73B681B0502
:104C80007FF56FAF514B19680A2338E0504B1B6812
:104C900059077FF566AFE96833E03B681A057FF591
:104CA00060AF4C4B05E04A4B1B685B077FF559AF83
:104CB000494B196825E0494B0A21B3F9043059439F
:104CC0001FE03E4B59682C2319E0414B1B6813F041
:104CD00020097FF446AF3B681A067FF542AF49468C
:104CE00005F0D4FD85F848903BE73B689B077FF5CE
:104CF00038AF344B0A211B885943334B1B7891FB47
:104D0000F3F105F0C3FD002385F8483029E794F856
:104D10004B30274F002B00F0B680FB6C002B00F0CF
:104D2000B280D6F800803B6DC3EB0803632B40F2E2
:104D3000AA802A4D412005F051FDB5F902000A264E
:104D400090FBF6F080B205F071FDB5F9000090FB24
:104D5000F6F080B205F06AFDB5F9043093FBF6F089
:104D600080B205F063FD05F06AFD97F8545015F028
:104D7000010564D1104B1B88DF0532D4DE060DD44B
:104D80009D060DD458060DD419070DD4DA0727D483
:104D900013F0020F0CBF0125032522E00D2520E0B2
:104DA00009251EE004251CE008251AE0DCC50108E1
:104DB000101A0020DA320020141800204C150020B0
:104DC000141400209E190020C0000020701500203F
:104DD000100E0020681500206415002036180020F1
:104DE0000225C04B1E78C04BC6F38006DB7813B19A
:104DF00046F00206F6B2532005F0F0FCBB4B1888D3
:104E000000EB800000EB8000800080B205F00EFD1A
:104E1000002005F00BFDB64BFE201B88584340F2E6
:104E2000FF3390FBF3F0C0B205F0F0FC002005F07A
:104E3000EDFC46EA850005F0E9FC05F000FD94F87C
:104E400054309BB94F2005F0C9FC07F047F907F033
:104E500045F907F043F9012005F0D8FCA54B187877
:104E600000F0010005F0D2FC05F0E9FC94F85420B4
:104E70000A230132D2B2B2FBF3F103FB1123C4F8CF
:104E8000508084F8543094F855609B4D022E40F0C9
:104E90000A8105F0EFFBAB6DC3EB000840F6B833B9
:104EA000984508D9002385F85530B5F85C300133B2
:104EB000A5F85C305BE195F862303A2B40F0058153
:104EC00005F15E0095F8601001F09AFB002840F0B3
:104ED000FC80864B894F1B88C7F86C80FB61884B30
:104EE000DFF838821B68D8F80000FB62EB68FB63D0
:104EF000844B1B68FB64B5F85C30FB650CF0BCF8B8
:104F00008246002840F0CF803146D8F8000005F0F6
:104F10001FFC042387F8743095F8673095F861908A
:104F2000642B794E4AD195F86830784A072B08BF30
:104F300085F868A094F868502B01D15802EB030B58
:104F40000846029111F0A2FEDBF804305FFA80FA05
:104F50001846019311F09AFE5FFA80FB0AEB0B02F0
:104F60000832F27125F00F02B27205F00F0272736F
:104F70000BEBCA02B27302995246654811F021FE4A
:104F8000019B0AF10900DFF898A119465A465044DE
:104F900011F017FE96F807B00AF1010A584607F01B
:104FA0007FF80AF80B00484607F062F80135002345
:104FB00084F8673084F8685000235DE097F87550F6
:104FC0002B0708BF01354FF0000308BFEDB2B372E5
:104FD000504B072D28BF01259C462801391891F810
:104FE00010E001F10C0240EA0E0E83F800E0DFF859
:104FF00034A11279C9681AF8022003921A46DDF822
:105000000CB002F1010E9B44C2EB0B0B0BF0FF0B3B
:10501000BBF1010F03D95170090A7246EFE738441A
:10502000427C013521F06001EDB21143082D0EF1F3
:1050300001038EF800100AD03049CCEB030201EBDB
:105040000511097C1AF801100A44132AC5DDCCEBBE
:10505000030A0AF1060A5FFA8AFA4AF04003F3717A
:10506000504607F01DF82C4B87F8755003F80A00DE
:10507000484606F0FDFF9FE7B2785D1CDBB29A421E
:1050800007D9214AD8F80000D15C05F09DFB2B46DA
:10509000F2E794F867200323013287F8743084F82C
:1050A000672084F85530154D95F87430032B5ED188
:1050B0001A4E306805F051FB002858D030680121A5
:1050C00005F046FB022385F87430002384F8553040
:1050D0004DE099F800303BB3C5F8248089F800A072
:1050E00066E400BFDA320020040F00209E19002081
:1050F0006C150020B90D0020101A00202C00002093
:1051000070150020681500202914002030000020B0
:10511000381400203614002030140020F80F00202E
:105120002F1400204DC601086B6AC3EB0803B3F5CA
:105130007A6FFFF43DAC0123A86A89F8003005F0CE
:105140001CFB8146A86A05F018FB19F07F0F7FF45D
:105150002FAC8E287FF42CAC95F82030002B7FF4F8
:1051600027AC044BEB622D2385F8303020E407B0E8
:10517000BDE8F08FE5130020436A8269D154436A89
:1051800002690133934228BF00234362436B23B17A
:105190001B68DB0706D406F055B9036DDA6842F0E8
:1051A0008002DA607047F8B505F064FA064600F14F
:1051B000FA07224D224C2B781B01E118E3589A681C
:1051C000CB881A4209D005F055FAB842F1D9FF2030
:1051D00032E005F04FFAB842F9D82B781B01E118FC
:1051E000E3589A68CB881A42F3D005F043FA154B7E
:1051F000801B18605B6898421BD806F5FA762B78FE
:105200001B01E118E3589A68CB881A4208D005F0D0
:1052100031FAB042F3D9DAE705F02CFAB042D6D829
:105220002B781B01E118E3589A68CB881A42F3D017
:1052300001E0012000E0002040B2F8BD731600201C
:10524000A81500207C1A002038B5002504460570FA
:10525000FFF7A9FF431C0FD0012803D1A8402378F2
:10526000184320700135082DF2D1044B21781A7AA9
:1052700001204A401A7238BD002038BD7C1A002037
:105280002DE9F047224A80461078224B224900013E
:105290000D681E181C58F088023591461F46A368F9
:1052A000184203D00B68AB42F9D32EE005F0E2F9C7
:1052B000054600F11B0405F0DDF9A042FBD30026F2
:1052C00005F2232A354699F800301B01F918FB58DE
:1052D0009A68CB881A4203D00123B3401D43ADB274
:1052E0003434544505D005F0C5F9A042FBD301364E
:1052F000E9E740F201232B40B3F5007F05D16D08AB
:1053000088F800500120BDE8F0870020BDE8F08754
:1053100073160020A81500209432002038B58000B4
:1053200040F4806405F0A6F944F0010405460C4AF7
:105330000C4B127814F0010F4FEA021203EB02013A
:105340009B58CA8805F1340514BF1A615A61640874
:1053500004D005F08FF9A842FBD3E8E738BD00BFC1
:1053600073160020A815002008B50DF09BFB024B1A
:105370004FF400621A8008BD0600002037B50546CC
:105380000DF090FB2C4B1A682C4B9A420ED14FF427
:105390000053ADF8043002238DF807300423284869
:1053A0000DEB03018DF806300CF09FFB254C0DF042
:1053B00079FBA36880216B209847642005F081F970
:1053C000A368072168209847642005F07AF9A3684C
:1053D00000216B209847642005F073F9A368012130
:1053E0006B2098470F2005F06CF9A36818211B204B
:1053F00098470F2005F065F9A36818211C209847ED
:105400000F2005F05EF9A36829461A2098470F205F
:1054100005F057F90C4AA3681178192098476420C1
:1054200005F04FF9A368102137209847A3680121A0
:105430003820984703B030BD00000020001BB700A3
:10544000001001401C1E0020A01E00201FB50123DB
:10545000ADF80830ADF80410002301A9ADF80A300A
:10546000ADF80C30ADF8062000F004FE05B05DF894
:1054700004FB10B5A0F5127494F83C22C2B9A36ADB
:10548000616A994229D0591CA069A162C05C236954
:10549000C0B299424FEA400343F40073A4F83E328D
:1054A0004FF00A0384F83D3228BFA262012312E0C4
:1054B00094F93D327BB1B4F83E1220464B08A4F873
:1054C0003E3201F001010CF0E0FA94F83D32013B6C
:1054D00084F83D3201E084F83C3294F83832002BF5
:1054E0004FD194F839320133DBB2092B84F83932C9
:1054F00004D12046BDE810400CF0B2BA0A2B40D1CE
:1055000094F83B322BB9B4F8403243F00103A4F8CD
:1055100040326379D9071CD5B4F84002820501D422
:10552000C30705D4B4F844320133A4F8443210E080
:10553000E36AC0F347000BB198470AE0E369626988
:10554000D054E269E3680132B2FBF3F103FB1123AB
:10555000E361012284F8382294F83B220023012AD7
:1055600084F839320DD1A27984F83B32236B12F0E2
:10557000010F1868997A0CBF02220022BDE8104082
:1055800064E710BD38B5A0F513746379A579DB071E
:1055900045D594F8383205F00105F3B1236B18684E
:1055A000828DC2F34E02828494F83C2222B1B4F878
:1055B00042220132A4F84222997A6A00FFF746FF9C
:1055C000012384F83B32002384F8393284F83A32DC
:1055D00084F83832A4F8403238BD94F83B32204683
:1055E000012B04BF94F8393284F83A320CF038FABF
:1055F00094F83B22236B3AB9012284F83B221868C5
:10560000997A05FA02F207E0002284F83B229542DB
:105610001868997A08BF0222BDE8384016E738BDFD
:10562000F7B50023454D464E8DF8033060236B607F
:1056300033780746152B06D0122B04D0012B14BF4C
:105640008C24022401E044F62064FFF7ACFD00281E
:1056500002DA013CF9D114E00A24FFF7A4FD01307D
:105660000FD0013C14F0FF04F7D12B685A0802EB6D
:1056700093036B60FFF797FD431C02D00028F9DC11
:1056800001E0002457E000230DF103002B72FFF727
:10569000DBFD00284FD09DF803301B2B4BD10DF1C3
:1056A0000300FFF7D1FD002845D0244B9DF80320CF
:1056B0005B7A9A423FD10DF10500FFF7C5FD9DF8D9
:1056C0000530012B37D801A8FFF7BEFD9DF8043047
:1056D0008BB30DF10300FFF7B7FD60B39DF8033006
:1056E0000E2B28D10DF10300FFF7AEFD18B39DF886
:1056F000032033789A421ED10DF10300FFF7A4FD79
:10570000C8B19DF80330B3B93E46BDF80430F21B72
:1057100092B2023B9A4205DA3046FFF795FD50B14E
:105720000136F2E70DF10300FFF78EFD2C7AD4F17C
:10573000010438BF0024204603B0F0BD7C1A0020CD
:10574000741600200F4B1A78832A17D1598840F21B
:105750001452914212D11A79BE2A0FD193F8102512
:105760000020EF2A0CD113F8012B5040064A934237
:10577000F9D1D0F1010038BF0020704700207047F8
:10578000704700BF00F8010814FD01082DE9F3413E
:1057900006F0C2FD4A4B83221A7040F214525A801E
:1057A000BE221A71EF2283F81025002283F81125FA
:1057B00011461E46B35C0132594040F214539A42DE
:1057C000F8D13F4B3F4A83F811153F4B04275A60ED
:1057D00002F188325A600020013F17F0FF075DD0C8
:1057E000394B3422394CDA60C4F309037BB13319E5
:1057F00003F17843A3F5FC33D3F800804FF4005055
:105800000023019306F02AFF0428E5D11BE04FF4A2
:10581000302006F023FF0428DED12B4D4FF430203A
:105820002B6943F002032B616C612B6943F0400349
:105830002B6106F013FF2A6941F6FD73134004281B
:105840002B61D4D0C8E7204D4FF400502B6943F0B2
:1058500001032B611FFA88F3238006F0FFFE042862
:1058600012D1A31C0193019B4FEA1848A3F80080B2
:105870004FF4005006F0F2FE2B6941F6FE721A401A
:1058800004282A6106D0A7E72B6941F6FE721A4068
:105890002A61A1E70E4B04349C42A5D10A4B04288F
:1058A0001A6942F080021A6102D1FFF74BFF10B96A
:1058B000052009F081FE06F019F802B0BDE8F0817C
:1058C00050040020230167450020024000F8010831
:1058D00014FD010808B5044804F0ADFEFFF756FFBB
:1058E000BDE8084009F04ABE57C6010813B5FF23BA
:1058F00004468DF807300DF10700FFF7C1FC10B921
:105900000CB1013CF7E79DF8070002B010BD37B5B8
:105910001F4B01390022CDB29A72DA721A735A7390
:105920000135FF2304468DF8073005442046FFF774
:10593000A7FC20B314F8010B04F0BEFDAC42F5D176
:10594000144B1B78BBB1124C04F10C00FFF798FC10
:10595000A8B104F10D00FFF793FC80B10DF1070031
:10596000FFF78EFC58B16289A3899A4207D0C223FF
:105970008DF8073003E00DF10700FFF781FC9DF87B
:105980000700B0F130035842584103B030BD00BFAA
:105990007C1A0020DC1400202DE9F041194E1A4D2C
:1059A00033780F461B01E918044607F1FF38E85821
:1059B0000C310CF09AF85FFA88F8144B0022A044DE
:1059C00037469A72DA7208F101081E462078FFF70E
:1059D000A5FC14F8010B04F06FFD4445F6D10C4B07
:1059E0001B782BB1B07AFFF799FCF07AFFF796FCA1
:1059F0003B781B0103F10801E8582944BDE8F04158
:105A00000CF073B873160020A81500207C1A002033
:105A1000DC14002073B5FE238DF8043000238DF8CC
:105A200005308DF806300B7806460C4615468DF885
:105A3000073013B901238DF8063001A80421FFF7C0
:105A4000ABFF0220FFF752FFFF281CD160682178CE
:105A5000FFF7A2FF2820FFF749FFB0F130025042C4
:105A6000504188B1012301A802218DF805308DF83D
:105A70000460FFF791FF2846FFF738FFB0F13003CD
:105A80005842584100E0002002B070BD07B50368DD
:105A9000114A23F07F4323F0FF03934217D0FF23E3
:105AA0008DF8043000238DF80530437804218DF8FB
:105AB0000630837801A88DF80730FFF76DFF0220CC
:105AC000FFF714FFB0F130035842584100E00120C5
:105AD00003B05DF804FB00BF00FFFF0037B50546CB
:105AE00008460C46FFF7D2FF60B1237801A80221D7
:105AF0008DF804508DF80530FFF74EFF606821786F
:105B0000FFF705FF03B030BD074B1A781044C0B251
:105B1000020648BF803818701A78044B1B789A42E6
:105B200001D10BF033BF704779280020F8270020FF
:105B3000F8B5214B06461A78082742401A701F4DC7
:105B40001F4C2B7816F0010F4FEA031304EB0302EE
:105B5000D288E3581A610AD0402004F0A7FD2B78C0
:105B600040201B01E218D288E3585A611BE0202034
:105B700004F09CFD2B7820201B01E218D288E3580A
:105B80005A6104F093FD2B7820201B01E218D28883
:105B9000E3581A6104F08AFD2B7820201B01E218DB
:105BA000D288E3585A61013F04F080FD17F0FF07E7
:105BB0004FEA5606C3D1F8BDC21C00207316002060
:105BC000A815002008B5104B104A1B781B01D118EE
:105BD000D0580C310BF089FFFF20FFF7A9FFFF2001
:105BE000FFF7A6FF7F20FFF7A3FF094B00221B2032
:105BF0001A70FFF79DFF074B587A0130C0B25872F8
:105C0000BDE8084094E700BF73160020A8150020E7
:105C1000C21C00207C1A002003788B4286BF024BF6
:105C200033F8110000207047881C0020014B33F826
:105C300021007047601C002030B500221346214926
:105C400014180C5D83EA0423082413F4004F4FEA70
:105C5000430318BF83F4815304F1FF3418BF83F06A
:105C6000010314F0FF049BB2EFD10132192AE6D1EF
:105C700000F119028D5C00F11A028A5C02EB052228
:105C800092B29A421DD1104B1D782346DAB2AA4235
:105C900014D2441C04EB4202D2B28C5C01328A5C06
:105CA00002EB0424A4B24FF4AF625443074A241316
:105CB00004F5487422F813400133E7E7044B01224E
:105CC0001A7030BD8C1A0020F40F0020AE1A00208C
:105CD000F00F002003788B4283BF034B03EB41019D
:105CE000488C0020704700BF8C1A002003788B423C
:105CF0000AD9064B1A78064B53F8210002B1400826
:105D000000F5777080B2704700207047CE2F0020DA
:105D1000701B002007299ABF024B33F82100002096
:105D2000704700BF1C1C0020024B33F81100C00854
:105D3000704700BFE41B002008B5074B53F8210053
:105D40000DF0DEFC05490DF033FD05490DF028FC92
:105D50000DF01AFF80B208BDA00F00200000203F08
:105D600000005C44014B33F81100704774150020AB
:105D7000014B33F811007047AA1C0020014B33F887
:105D800011007047AA1C00200020704710B504467F
:105D900004F070FC0D4B40F6B831DA6BD863821A10
:105DA0008A4284BF002283F8402093F840200AB939
:105DB000202C0AD106491F2A8C5403D1054B0122FD
:105DC0001A7010BD013283F8402010BD8C1A0020DB
:105DD0003D1C00203C1C0020F8B5074604F04AFC9E
:105DE0002B4E2C4C736C2C4DC31AB3F5FA5FB36475
:105DF000706402D9002323702B7023781BB9A12F64
:105E000004BF01222A702A781AB1FFB2F754013375
:105E10002370224B21781A781F46914236D1204BAD
:105E20001B78052B02D0062B03D02CE00020FFF7B7
:105E300003FF73781E2B26D13878002201381346D1
:105E4000D1B2814219DA775C19463B46082781EACC
:105E5000030C1CF0010F1CBF83F01803C3F34603AF
:105E600007F1FF370CBF5B0843F0800317F0FF0713
:105E7000C1F34701EBD10132E2E7325C934202D138
:105E80000320FFF7D9FE00232B702370F8BD00BF5D
:105E90008C1A0020F20F0020F10F0020F30F0020D9
:105EA000F50F002010B5044604F0E4FB0F4B41F25F
:105EB0008831DA6CD864821A8A421A6584BF00225B
:105EC00083F8542093F854300F2B0DD85A1C0749EF
:105ED000D2B281F854200649E4B2102ACC54054BC2
:105EE00014BF002201221A7010BD00BF8C1A0020BE
:105EF0005E1B00205D1B002010B5044604F0BAFBB9
:105F00000D4B41F288319A6D9865821A8A42DA65A2
:105F100084BF002283F8602093F86030074A142B76
:105F2000D45403D1064B01221A7010BD024A01332A
:105F300082F8603010BD00BF8C1A0020051C0020C4
:105F4000041C002010B5044604F094FB244A536E50
:105F50005066C31AB3F57A6F84BF002382F86830A5
:105F600092F8683033B9A82C39D11E490B701E49FC
:105F70000B8006E0022B02D11C490C7001E0242B9F
:105F800001D81B49CC540133DBB282F86830174A80
:105F9000127802325200934217DA134AE0B21388A1
:105FA00083EA0020082310F4004F4FEA400018BF96
:105FB00080F4815003F1FF3318BF80F0010013F02B
:105FC000FF0380B2EFD1108010BD0132934206D1A1
:105FD000034B002283F86820024B01221A7010BD87
:105FE0008C1A0020BA1B0020BC1B0020BB1B002009
:105FF000BE1B002010B5044604F03CFB104A40F6DE
:10600000AC51D36EC31A8B42C4BF002382F87030E8
:1060100092F8703023B90F2C10D10949C86601E0FD
:10602000182B0BD8591CC9B282F87010054A1929CF
:10603000D454054B14BF002201221A7010BD00BFBA
:106040008C1A0020A11B0020A01B0020084BDA683E
:10605000D10709D4DA68520708D4DB6813F0100FAF
:106060000CBF0420032070470120704702207047B6
:10607000002002400A88F0B54B888F880E89CD88B1
:10608000002A3AD1048C834A24F001042404240C0D
:106090000484018B048C89B221F0F30141EA0616D5
:1060A000B6B29042A4B246EA070743F0010315D006
:1060B00002F50062904211D0B0F1804F0ED0A2F5EF
:1060C000983290420AD002F58062904206D002F5E2
:1060D0008062904218BF24F00A0401D124F0020427
:1060E000234307830384038B23F00C031B041B0C43
:1060F0000383038B9BB21D4344E0042A44D1048CE8
:10610000644A24F010042404240C0484018B048CBD
:1061100021F440710905090D41EA063189B241EACD
:1061200007279042A4B2BFB212D002F5006290429B
:106130000ED0B0F1804F0BD0A2F59832904207D02C
:1061400002F58062904203D002F58062904207D14E
:1061500024F0200444EA03139BB243F0100304E04C
:1061600024F0A00443F01003234307830384038B2C
:1061700023F440631B041B0C0383038B9BB243EA91
:106180000525ADB20583F0BD082A018C3ED121F46E
:1061900080710904090C0184818B3E4A89B221F087
:1061A000F301048C41EA0616B6B29042A4B246EA64
:1061B000070712D002F5006290420ED0B0F1804F76
:1061C0000BD0A2F59832904207D002F5806290423F
:1061D00003D002F58062904207D124F4007444EAAF
:1061E00003239BB243F4807304E024F4206443F45B
:1061F0008073234387830384838B23F00C031B0466
:106200001B0C8383838B9BB21D4341E021F480519F
:106210000904090C0184828B048C22F4407212055B
:10622000120D42EA072242EA06361A4AA4B2904206
:10623000B6B212D002F5006290420ED0B0F1804F9B
:106240000BD0A2F59832904207D002F580629042BE
:1062500003D002F58062904207D124F4005242EA52
:10626000033292B242F4805205E047F6FF522240D8
:1062700043F480531A4386830284838B23F4406360
:106280001B041B0C8383838B9BB243EA0525ADB2B1
:106290008583F0BD002C01401FB50123ADF8083007
:1062A0000023ADF80C30ADF80A30094BADF80410FE
:1062B0001B7801A9012B08BF0323ADF8062008BFF6
:1062C000ADF80C30FFF7D6FE05B05DF804FB00BF5B
:1062D000A40A002038B510F80E2C044650F8043CEF
:1062E00052B9012200F80E2C20F80C1C997A18687B
:1062F0000222BDE83840CFE730F80C2C20F80A1C09
:10630000891A89B220F8081C074A10F80F0C0025DA
:1063100022F8101004F80E5C1868997A2A46FFF7E4
:10632000BBFF04F8065C38BDAA1C002038B50D4B35
:106330000D4C1A681D46D16812898968114203D034
:1063400004F098F9606707E004F094F9636F9842ED
:1063500002D9064AC31A13602B681A69044B5A61A2
:1063600038BD00BFFC0F00208C1A0020AC000020BC
:1063700000040140054B1A685B69034004D01042D9
:106380000CBF0020012070471846704700040140F0
:10639000154B016810B51C68CA4314401C605C684A
:1063A00022405A60027902F1804202F5823214687A
:1063B0002143116002689C68D1430C409C60DC68FA
:1063C0002140D9604179102906D19968114399601B
:1063D000D9680A43DA6010BD01F1804303F58233C6
:1063E00019680A431A6010BD00040140CB78F0B56B
:1063F000DA0648BF8A78098803F00F0548BF1543BD
:1064000011F0FF0F1DD0046800220127974007EA12
:106410000106BE4211D197004FF00F0C0CFA07FC99
:1064200005FA07F724EA0C04282B44EA070401D1F3
:10643000466102E0482B08BF06610132082AE4D118
:106440000460FF291FD94468002202F108060127D1
:10645000B74007EA0106BE4211D197004FF00F0C7A
:106460000CFA07FC05FA07F724EA0C04282B44EA87
:10647000070401D1466102E0482B08BF06610132E2
:10648000082AE2D14460F0BD2DE9F84305460C46E8
:10649000006869684C4B023A03C3A86843F8800956
:1064A000062A05D8DFE802F0080C121A1F2327007D
:1064B0009A6F2260DA6F0DE0DA6F22609A6F03E064
:1064C0009A6F52422260DA6F524203E0DA6F524210
:1064D00022609A6F6260D3F8803015E09A6F524262
:1064E0002260DA6F0CE0DA6F22609A6F08E09A6F30
:1064F0002260DA6F03E0DA6F524222609A6F5242F2
:106500006260D3F880305B42A360304B1B78002B75
:1065100057D120680DF0F8F8804660680DF0F4F867
:106520000746A0680DF0F0F8294D06462968404658
:106530000DF03EF9E968814638460DF039F901461B
:1065400048460DF02DF8A969814630460DF030F926
:10655000014648460DF024F810F09EFD6968206061
:1065600040460DF025F92969814638460DF020F99D
:10657000014648460DF014F8E969814630460DF0B1
:1065800017F9014648460DF00BF810F085FDA96893
:10659000606040460DF00CF96969804638460DF0A0
:1065A00007F9014640460CF0FBFF296A07463046D2
:1065B0000DF0FEF8014638460CF0F2FF10F06CFDCD
:1065C000A060BDE8F88300BF041B00200400002089
:1065D000D80D0020094B44F6FB711B681A7802EBBA
:1065E000421200FB021059789B78C1EB0131B0FBDD
:1065F000F1F0B0FBF3F080B2704700BF64140020EC
:10660000002330B504461846DAB28A420DD2E25C65
:106610000133424082EA0212D2B21509000A85EA29
:10662000C20540EA02206840EEE730BD114B00F1A0
:106630000C021B6803EB4202911D927912B1022AEF
:1066400010D00BE0022805D9032807D10A4A1268A6
:10665000D20401D5188A7047588B7047074B33F81E
:1066600010007047487800EB800000EB800000F2DB
:10667000EE207047280F0020700900202E0F002008
:10668000094B93F884205AB9084A094912680978D5
:10669000127E0432D2B28A4228BF0A4683F884208E
:1066A00093F88400704700BF8C1A0020280F002048
:1066B000E80F002008B5104B1B78012B0ED008D333
:1066C000022B0FD10D4A13689288D9684A40DA60CC
:1066D00008E00A4B1A689B88136103E0074B1A68AD
:1066E0009B88536103F0C6FF054B00F5F42000F5CD
:1066F0009070186008BD00BFF917002074090020D1
:10670000FC17002038B50D4D04462B68834206D196
:1067100003F004FF284600214C2210F076FAEB6CBF
:10672000A34209D1204603F0F9FEBDE838400448F1
:1067300000214C2210F069BA38BD00BF640E002061
:10674000B00E0020064B10B504462146186803F031
:106750005DFF044B1B689A7954409C7110BD00BFCB
:10676000241500201C15002008B5054B1B689879DE
:10677000FFF7E8FF034B1868BDE8084003F0DCBFF3
:106780001C1500202015002038B50F4B0446186852
:106790000D4603F0D7FF2420FFF7D4FF4D20FFF76D
:1067A000D1FF002C094C0CBF3E202120FFF7CAFF6F
:1067B0002368002228469A71FFF7C4FF236893F8E4
:1067C0004900BDE83840BDE7201500201C15002019
:1067D00001460020D8E710B50446C0B2FFF7B2FF6B
:1067E000200ABDE81040ADE710B5044680B2FFF7BF
:1067F000F2FF200CBDE81040EDE7564B2DE9F04FBD
:106800001A888DB012F0010F0CBF0020022012F088
:10681000020F0CBF0021042112F0040F0CBF002353
:10682000102303934C4B02F0080A1B6812F0400F30
:1068300003F0C00B03F480794BEA0A0A0CBF002571
:10684000202503F4805812F0100F4AEA090A01903B
:1068500003F4005C0CBF00204FF400704AEA080A01
:1068600012F0200F029103F480470CBF00214FF477
:1068700080614AEA0C0A12F4807F049505900CBFEF
:1068800000254FF4006503F4003003F400464AEAA3
:10689000070A0795089003F480354AEA060A06912C
:1068A0004AEA050A03F48021089D099103F40020B7
:1068B0004AEA050A099D0A9003F480114AEA050A8A
:1068C0000A9D0B914AEA050A0B9D244803F00074C7
:1068D0004AEA050A007803F000654AEA04042C43FA
:1068E00003F08053C0F38000234303430198029DCB
:1068F000034303982B43049D034305982B43069DB4
:106900000343079812F4007F43EA050343EA0003B8
:106910000CBF00214FF40011194312F4806F104B8B
:106920000CBF00224FF0806200201D780A4303460E
:10693000AB420CD20B490124595C04FA01F111421B
:1069400018BF9C4003F1010318BF2043F0E70DB0CE
:10695000BDE8F08F14180020A0180020DA320020C3
:10696000620E0020440E002010B503F09AFD04468C
:1069700003F097FD04EB002080B210BD10B5FFF7C7
:10698000F3FF0446FFF7F0FF04EB004010BD00BF2B
:1069900038B50378F3B9204B1B680133132B1C4621
:1069A00005D81E4A0C2101FB032295681DBB01344A
:1069B000132C01DD002400E005D8184A0C2101FB4E
:1069C00004229568BDB99C42F1D11548BDE8384014
:1069D00005F03EB910F0AFF91328044605D80F4B67
:1069E0000C2202FB00339D682DB921460D48BDE8FD
:1069F000384005F02DB9084B1C6008F063FE0A48CA
:106A000021462A4605F024F90C235C43034B185D0C
:106A1000BDE8384008F06ABEA4000020E0CA0108C2
:106A20005EC6010874C601088CC6010838B50A4D57
:106A30000A4803F000FE286803F0DCFD084B002440
:106A40001C70084B1C60084B1C7006F03DFA08F0E7
:106A500095FD2C6038BD00BFE0140020A3C60108DE
:106A6000EC140020E8140020DC3200202DE9F04F67
:106A7000012828BF012089B00190019A142000FB51
:106A800002F3DFF8C4B16A4A0BEB03015BF8037051
:106A9000684E019BF469176013710A690D892243DE
:106AA000F261BA88B1F80A9022F440724C6812047C
:106AB000120C49EA0508BA8003A9C4F81080022222
:106AC0008DF80E002046ADF80C808DF80F200BF0ED
:106AD0000CF84FF0080AA268154203D10A2003F00F
:106AE000E5FDF8E70A20656103F0E0FD25610A2075
:106AF00003F0DCFDBAF1010AEDD10A20C4F81490CC
:106B000003F0D4FD0A20656103F0D0FD0A20256161
:106B100003F0CCFD0222C4F8109020468DF80F201F
:106B200003A91C228DF80E20ADF80C800AF0DDFFC1
:106B3000414A9742326905D142F4001232614FF462
:106B4000001004E042F4800232614FF4800005F04E
:106B50007DFDBA8803A822F440721204120CBA8098
:106B60003A88012592B242F001023A80BC8805F0D1
:106B700023FD24F03F04059830492404B0FBF1F1D3
:106B8000240C0C43A4B2BC803A88142322F00102E6
:106B90001204120C3A802A4A0024B0FBF2F24FF49D
:106BA0009670414392B24FF47A70002A91FBF0F153
:106BB00008BF0122013142F4004289B23984BA830C
:106BC0003A8803A892B242F001023A803A8822F44D
:106BD000816222F002021204120C3A804FF48042C9
:106BE0003A81019A8DF80D4003FB02B77B7B8DF84B
:106BF0000E408DF80C308DF80F5007F065FB3B7B95
:106C00009DF80F208DF80C308DF80D408DF80E405A
:106C10001AB103A807F058FB07E0590903F01F0356
:106C20009D40084A203142F8215009B0BDE8F08F5C
:106C3000141B0020001002400054004040420F008E
:106C4000009F240000E100E0E8AB010808B5054B17
:106C50001A88013292B21A80034B1879FFF706FFA7
:106C6000002008BD48150020141B002013B51E4B42
:106C70004000C0B2587102AC1868997104F8012D37
:106C800000210122DA71DC6019721C611A755A75D3
:106C9000997538B38288920515D40288D4050DD42D
:106CA0004FF480520188890502D5013AFAD112E0E9
:106CB0008AB1028892B242F480720280828892B2D3
:106CC00042F4407282804FF48052597D11B1013AF2
:106CD000FBD100E012B9FFF7B9FF03E0024B987D4A
:106CE00080F0010002B010BD141B002010B5400060
:106CF0001C4CC0B26071A17101200021E1712072B1
:106D00002275607520682361E360A17540B38388B4
:106D10009B0515D40388D9050DD44FF48053028800
:106D2000920502D5013BFAD112E08BB103889BB2E8
:106D300043F48073038083889BB243F44073838061
:106D40004FF48053627D12B1013BFBD100E01BB9CF
:106D5000BDE81040FFF77ABF024B987D80F001003C
:106D600010BD00BF141B002037B5044603211E20B0
:106D700006226B46FFF7BAFF70B39DF801309DF80D
:106D80000000164D43EA002000B20CF0BDFC29685B
:106D90000CF00EFD0CF0D2FE9DF8033020809DF823
:106DA000020043EA002000B20CF0AEFCA9680CF02F
:106DB000FFFC0CF0C3FE9DF80530A0809DF8040098
:106DC00043EA002000B20CF09FFC69680CF0F0FC74
:106DD0000CF0B4FE6080012003B030BDB400002090
:106DE00007B5002101AB03227720FFF77FFF9DF855
:106DF00005009DF80430000240EA03409DF806308B
:106E0000184303B05DF804FB08B5FFF7E9FF014B39
:106E1000986108BD141B002008B5FFF7E1FF014B86
:106E2000D86108BD141B002007B5F7216B46062268
:106E30007620FFF75BFF9DF800209DF801301203DC
:106E400042EA03129DF8023042EA1312084B1A601C
:106E50009DF803209DF80430120342EA03129DF8C6
:106E6000053042EA1312034B1A6203B05DF804FBCB
:106E7000C0320020141B0020104B07B51B7813B143
:106E80000F4B1B78BBB1032201AB7720F621FFF734
:106E90002DFF9DF805209DF80430120242EA0342BE
:106EA0009DF806301A43074BB3F92030C3F10803AD
:106EB000DA40054B5A6203B05DF804FBAB000020DA
:106EC000C42F0020441E0020141B00200B4B07B5CC
:106ED0001B7813B10A4B1B786BB1022201AB7720F0
:106EE000F621FFF703FF9DF805309DF8042043EAE3
:106EF0000222044B1A8503B05DF804FBAB000020AE
:106F0000C42F0020141B002030B505460C46134644
:106F1000294622466820BDE83040E7E613B5062240
:106F2000044601211C206B46FFF7E0FE08B39DF8E4
:106F300001309DF800209DF8021043EA022242F33E
:106F40008D02042392FBF3F222809DF8032042EA93
:106F5000012242F38D0292FBF3F262809DF804104D
:106F60009DF8052042EA012242F38D0292FBF3F3E1
:106F7000A38002B010BD13B50622044602211820DA
:106F80006B46FFF7B3FEB8B19DF800309DF80120C5
:106F90009B0803EB022323809DF802309DF8032019
:106FA0009B0803EB022363809DF804309DF80520C5
:106FB0009B0803EB0223A38002B010BD314B2DE9E7
:106FC000F3411B780546002B3CD00024264627467B
:106FD000A04601345320322108226B46E4B2FFF769
:106FE00085FE08B900204AE09DF801209DF8003098
:106FF000202C03EB02231BB29DF8032098449DF83C
:10700000023003EB02231BB21F449DF805209DF8BC
:10701000043003EB02231BB21E449DF8073003F03B
:107020007F0301D0002BD4D1174B98FBF4F897FBCA
:10703000F4F796FBF4F6A5F800806F80AE8083F835
:107040002A401CE05320322106226B46FFF74EFEF9
:107050000028C7D09DF801209DF8003003EB0223E3
:107060002B809DF803209DF8023003EB02236B80F8
:107070009DF805209DF8043003EB0223AB8002B09D
:10708000BDE8F0812D1E0020141B002010B5204CFF
:107090002368998A89B211F4706F1CBF0122A2750E
:1070A00011F4E06F2AD01A8B9A88890522F4806245
:1070B0004FEA02424FEA12429A801FD41A88920580
:1070C0001CD41A88D0050ED51A88D105FCD41A888C
:1070D00092B242F400721A801A889205FCD4207988
:1070E000FFF7C4FC0AE01A8892B242F400721A80D8
:1070F0009A8822F440721204120C9A802268938AB1
:1071000023F470631B041B0C93820023637510BD72
:10711000141B00200B4B07B59A690B4842F0100274
:107120009A614FF40053ADF8043002238DF8073014
:1071300001A910238DF806300AF0D7FC03B05DF8E2
:1071400004FB00BF001002400010014040F2E93390
:107150000B4A1189890709D5908140F2E933084A21
:107160001189C90707D59089C0B27047013B9BB20E
:10717000002BEDD1F0E7013B9BB2002BEFD1F2E702
:107180000038004070B5064C4FF480550E466561DE
:10719000FFF7DCFF3046FFF7D9FF2561012070BD06
:1071A000000C014070B5164B9B894FF47A7312F1B5
:1071B000FF3216D311B10C78013100E0FF24104DDD
:1071C0002E89B6070ED5AC814FF47A730C4C258905
:1071D000ED070DD5A489E4B20028E8D00470013091
:1071E000E5E770BD5E1EB6B2002BECD03346E6E795
:1071F000013B9BB24FF6FF75AB42E7D1EAE700BF18
:1072000000380040F8B5094C4FF480550E4617463B
:10721000656140F08000FFF799FF38460021324653
:10722000FFF7C0FF25610120F8BD00BF000C014041
:107230000F4B73B518781E4698B105230D4C8DF889
:1072400000304FF4805500238DF8013001A86561AE
:1072500069460222FFF7A6FF25619DF8050000F0B0
:10726000010000F00100307080F0010002B070BD3C
:1072700051140020000C0140064B70B51C680646F6
:107280001D46FFF7D5FF18B92B681B1BB342F8D971
:1072900070BD00BF94320020F7B5144603228DF86C
:1072A0000420020C8DF805208DF80700020A062044
:1072B0000F468DF80620FFF7DFFF78B1084D4FF439
:1072C0008056002001A904226E61FFF76BFF38464B
:1072D00000212246FFF766FF2E61204603B0F0BD75
:1072E000000C01402DE9F04F9F4B85B01A68D10387
:1072F00040F1C5829D4B1B78002B00F0C0829C4B57
:107300001A7802F0FF03002A40F0B982994A9A4F96
:10731000126812F4804F0CD03A7862B1974A116823
:10732000974A99500433802BF8D104F0F7FA0023E0
:1073300000E001233B703B78002B00F0A08203F0BB
:1073400099F9904D04462B686E68C31ADB43DB0F36
:107350000193AB68861BC31A6FEA0308019BF643CF
:10736000F60F4FEAD8782BB9B8F1000F02D1002EF2
:1073700000F085824FF0000A95F80C905FFA8AFBC6
:10738000CB45DFF844C251D2DCF8003003EB8B0967
:10739000B9F802301A050ED413F4805F784B06D08A
:1073A000794A99F80110126852F8212001E0734AD5
:1073B000126843F82B20B9F80230D8050DD499058E
:1073C00031D5724B1B7813F0040F0CBF704A714A11
:1073D0006B4B126843F82B2025E06F4A584649460C
:1073E00006F0C8FE6D4B1B885A0603D55846494621
:1073F0006B4A16E0580703D558464946694A10E0DB
:10740000190703D558464946674A0AE09A0703D543
:1074100058464946654A04E0DB0704D5644A5846A5
:10742000494606F0A7FE0AF1010AA5E7614B78225A
:10743000B3F90630DCF80010A3F57A7353434FF428
:107440007A7293FBF2F303F22B13039302914FEA48
:10745000890A0023534511D0029A1A4452885005D4
:107460000AD5474A0399985A084440F2671190FB9D
:10747000F1FB01FB1B0199520433EBE716B304F552
:10748000C333A0336B606B7B3E4ADBB936499373E1
:107490000B68990704D54849097809B1012191730E
:1074A000D80506D5454BDB781BB1AB7B43F0020317
:1074B000AB73364B1B7813F0050F03D1AB7B43F056
:1074C0000403AB73AA7B1AB92E4B5B7B002B7DD0D8
:1074D000697B11F0010FA1F10C001BD1032907D822
:1074E000264BDFF8ACB012F0040F18BF5B4600E08B
:1074F000224B0439072904D8314912F0010F18BF73
:107500000B46C0B2032810D82E4912F0020F18BF44
:107510000B460AE0C0B2032806D8184B1D4912F0EA
:10752000020F18BF0B4600E0144B0020C1B24945C2
:107530000DD2DCF8001001EB80014988090604D562
:10754000D3F800B00E4941F820B00130EEE7002E2C
:1075500042D0002A3BD06A7B0A4B0132D2B2142AB5
:1075600039D1002237E000BF700900202010002030
:10757000DD320020A0180020A800002038B4010847
:107580004C130020401B00201C100020DA32002089
:10759000909301088093010810AC01081418002092
:1075A00016AC01081CAC010822AC010828AC01088B
:1075B0002EAC01082E0F002068140020040F0020BC
:1075C000A0930108989301081810002026B16B7B46
:1075D000002BC0D100E05A73019B0BB3A9483221A4
:1075E000B0F90230B0F90020002BB8BF5B42002A8E
:1075F000B8BF524293FBF1F392FBF1F1DBB2C9B297
:107600008B4238BF0B46A04A0BB192FBF3F22244E7
:107610002A60EA7B9D4B0AB9012200E00022DA735E
:107620009B499A4B0978EA7BC9B9B8F1000F00F081
:107630002181DCF80060974B01961E78964B06F08E
:1076400004060022F6B295F80CA097F801B0D3F822
:1076500000C00296BF78914913461546AAE01AB9B0
:107660008F4A1A61002308E08E4AFAE7DCF800200E
:107670001A445188480603D404335345F6D1D4E75D
:107680008049B1F90000192822DD167895F8149088
:1076900006F00F0BCB4528690BDCDFF8F09199F869
:1076A0001590B9EB161F04DCD0F800907E4E43F81D
:1076B0000690167895F8169006F00F0BCB452EDB4A
:1076C000DFF8C89199F81590B9EB161F27DC23E075
:1076D000193024DA167895F8149006F00F0BCB4584
:1076E00028690BDCDFF8A49199F81790B9EB161F05
:1076F00004DBD0F800906C4E43F80690167895F8AD
:10770000169006F00F0BCB4509DBDFF8809199F856
:107710001790B9EB161F02DB066863481E50B1F9DB
:107720000210192918DD1678287D06F00F09814509
:1077300029690BDCDFF8549199F81590B9EB161F05
:1077400004DCD1F80090584E43F80690127802F00D
:107750000F0686421BDD8FE719318DDA1678A87D7A
:1077600006F00F09814529690BDBDFF8209199F8B4
:107770001590B9EB161F04DCD1F800904A4E43F87F
:107780000690127802F00F068642FFF675AFE87D8C
:10779000B0EB121FFFF670AF0968434A99506BE7D0
:1077A000019E06EB8200B0F8028018F4006F05D14C
:1077B00001320431D0B25045F2D323E0029E4EB1E3
:1077C00003EB0B0898FBF7F907FB1988B8F1010FD9
:1077D0000DDC01E055B9012590F801800CEB880023
:1077E0003CF8289090F80280C07803E0029D0020C9
:1077F00080468146013321F8029C81F80080487060
:10780000DBB2D5E7294A9178FF2912D10621B3FBD3
:10781000F1F001FB103010F0FF0F05D1917006E080
:10782000D90703D4C3F34703062BF9D89370012378
:10783000537051781D4B0139C9B2517009B99A780A
:107840005A70144B1B785B070DD5194B4FF47A72A5
:10785000B3F90630A3F57A7303EBC30393FBF2F39A
:107860000133DBB200E00123074A92FBF3F3074A3E
:107870001C44946005B0BDE8F04F04F04FB805B06B
:10788000BDE8F08F1C180020400D0300401B0020B5
:10789000B8160020DA3200201C1000204E13002001
:1078A0009C93010838B401084C130020A800002064
:1078B0002E0F00202DE9F84FBA4BBB4F1C683B78C8
:1078C00043B1BA4B1B68E31A002B03DBB84A002311
:1078D0003B701370B74B1D6842F201032B400BB98C
:1078E000B24A1371280740F1E681B34B1B681B7A3B
:1078F000082B00F2CF81DFE813F0090009003800FF
:10790000E60020014D014D0173019E01A7494B790D
:10791000002B00F0C08100234B71A84B93F800C0EE
:10792000A74B1B6893F80080A64B93F800900223A6
:10793000CE18B27903F1010B42FA0CF202F00F02F9
:1079400042459A480DD20B2A0BD896F806A000EBB8
:107950000B06B67900EB82020AEA090006EB00206A
:1079600090610233102BE3D18FE1904B93F84820C4
:10797000002A00F0A68093F84B0093F84A100022EA
:1079800083F8482000F007068F4A41EA062111607B
:1079900093F84C1001F03F06760146EAD0005060A3
:1079A00093F84D00800040EA911093F84E1001F0DA
:1079B000010640EA8620906093F84F0000F00F0621
:1079C000F60146EA5101D16093F8501001F07F06AC
:1079D000360146EA1010106193F85100400040EA69
:1079E000D11193F8520000F0030641EA462151619B
:1079F00093F8531001F01F06B60146EA900090611B
:107A000093F85400C00040EA511193F85600D16138
:107A100093F8551000F0070641EA0621116293F829
:107A2000571001F03F06760146EAD000506293F805
:107A30005800800040EA911093F8591001F00106B7
:107A400040EA8620906293F85A0000F00F06F60193
:107A500046EA5101D16293F85B1001F07F063601CE
:107A600046EA1010106393F85C00400040EAD11120
:107A700093F85D0000F0030641EA4621516393F854
:107A80005E1001F01F06B60146EA9000906393F87D
:107A90005F0093F86030C00040EA5111D163D9070C
:107AA0004CBF40F21471AD219E0711644CBF40F2EF
:107AB0001471AD2113F0080F51640CBF012303238F
:107AC000E9E01346E7E0394A002392F862101046D5
:107AD00089B392F86310B2F864C002EB410696F8DD
:107AE000698096F86A6082F8623046EA0826B445F2
:107AF00040F0D18092F86720012A04D0812A40F01A
:107B0000CA80032300E01346102984BF102280F8A6
:107B1000632090F8636000227600B24200F0BB80E0
:107B20002A48811891F803C00979263041EA0C21CE
:107B300011520232F1E70B46ADE01C4B93F8AC203A
:107B40009846002A00F0A680002388F8AC3098F808
:107B5000AD30A82B40F09E8098F8C060002E40F019
:107B6000998008EB460393F8B00093F8B13003EB2B
:107B700000200BF0C5FD16490BF0CEFE15490BF0A9
:107B80000DFD0CF001F8144B43F826000136082EC9
:107B9000E7D17AE0114A1378002B7CD000231370D0
:107BA00073E000BFB8320020B8160020581B002038
:107BB000B916002070090020280F0020CC2F0020CB
:107BC000C82F0020CD2F0020A00F0020BE1B0020BA
:107BD000CDCCCC400080BB431C1C0020F00F00200B
:107BE0005C49002291F8E430002B54D081F8E42065
:107BF00013464FF6FF72574901F1E5001E5C013351
:107C0000921B1E2B92B2F6D191F8046191F80331C8
:107C100003EB06239BB29A424FF000033BD1C218FC
:107C20009178D27801EB02214B4A42F813100233CB
:107C3000142BF4D129E0494E3378B146022B29D1D7
:107C4000DFF83481404698F80210FEF7D9FC42462E
:107C5000E8B91178537843EA012343F601618B4276
:107C600003D043F603618B420CD10023D118C879AD
:107C7000897901EB00203A49C0F3CC005852023315
:107C8000202BF3D1002389F80030012303E00023E7
:107C9000337000E00023D8070DD52E4A0121117161
:107CA0003049C3F340030B7083F001033B7004F5CC
:107CB000C333A033136015F4804F264B12D02A49EA
:107CC0000A7812B100220A7001221A7152B10122FF
:107CD0003A70244A0021117004F543321D4902F51F
:107CE000A0720A60E90712D593F8500193F8512168
:107CF000184982420BD01D4A012616701C4A0026E4
:107D0000167004F5C332A0320A6081F85101AA044A
:107D100008D500220F4901F5A970105A70B9023236
:107D2000182AF7D11B7933B9124B1868241AE0438B
:107D3000C00FBDE8F88F0120BDE8F88F0B4A012085
:107D400010700B4A0020107004F5C332A0320A6094
:107D5000E8E700BF581B0020601C0020E81D002041
:107D6000881C00202000002098150020B916002053
:107D70002100002088160020F01D0020F8B50368BF
:107D80000446DB690E4617468BB90D46F3195B1B9B
:107D9000002B0BDD236820469B6898470028F9D00C
:107DA000204615F8011B02F00FFDEFE7F8BD9847DC
:107DB000F8BD08B5054802F03EFC06F04FFEFDF7A1
:107DC000E5FCBDE8084007F0D9BB00BFCFC60108FD
:107DD00038B50D4B0D4D93F86A01FDF7A9FE2B78D0
:107DE0000B4C1B01E218D288E35820201A6102F0E4
:107DF0005DFC2B781B0103F10801E0582144BDE82C
:107E0000384009F072BE00BF581B002073160020D6
:107E1000A81500201E4B70B51D240E461C7005468B
:107E2000FDF7D0FE0020FDF783FE0820FDF780FE61
:107E30000E20FDF77DFE2046FDF77AFE0420FDF7BB
:107E400077FE0420FDF774FE0020FDF771FE302060
:107E5000FDF76EFE0020FDF76BFE0E4C3046FDF781
:107E600067FE0020FDF764FEFFF7B2FF2046FDF736
:107E7000D7FB224658B1237843B96378302B00D022
:107E800023B9937813B9034BDB782B70012070BDB5
:107E900074160020751600200C4B10B501241C70C0
:107EA000FDF790FE0020FDF743FE2046FDF740FE63
:107EB0000E20FDF73DFE2046FDF73AFEFFF788FF56
:107EC000BDE810400248FDF7ABBB00BF74160020B0
:107ED0007516002038B50368164A23F07F4323F057
:107EE000FF039342044623D0134B06251D70FDF774
:107EF00069FE0020FDF71CFE0520FDF719FE0E208F
:107F0000FDF716FE2846FDF713FE0020FDF710FED4
:107F10000020FDF70DFE6078FDF70AFEA078FDF762
:107F200007FEFFF755FFBDE838400448FDF778BB72
:107F3000012038BD00FFFF007416002075160020D8
:107F400073B5047805462CB104F10A03ADF804308A
:107F5000002604E04FF48573ADF804300126FDF7E8
:107F600031FE9DF80500FDF7E3FD9DF80400FDF7E7
:107F7000DFFD0E20FDF7DCFD194B1878FDF7D8FD6D
:107F80003046FDF7D5FD2046FDF7D2FD0020FDF778
:107F9000CFFD0020FDF7CCFD0020FDF7C9FD00203E
:107FA000FDF7C6FD0020FDF7C3FD0020FDF7C0FD75
:107FB0000020FDF7BDFD6B68013C1878FDF7B8FDAA
:107FC0006B6814F0FF0403F101036B60F3D1FFF75A
:107FD000FFFE044802B0BDE87040FDF721BB00BFC2
:107FE000741600207516002038B505780446D5F1C2
:107FF000010538BF0025FDF7E5FD0020FDF798FDE0
:108000000420FDF795FD0E20FDF792FD094B187831
:10801000FDF78EFD2846FDF78BFD2078FDF788FDE6
:10802000A020FDF785FDFFF7D3FE6068BDE838406E
:10803000FDF7F6BA74160020254B10B55343254AB8
:10804000254C12680139B2FBF3F20388013AA042D1
:1080500089B292B29BB212D004F50064A0420ED055
:10806000B0F1804F0BD0A4F59834A04207D004F5AE
:108070008064A04203D004F58064A04202D123F0C2
:1080800070039BB2154CA04206D004F58064A04258
:108090001CBF23F440739BB203800F4B8185984231
:1080A00002850FD003F5006398420BD003F54063BF
:1080B000984207D003F58063984203D003F58063AC
:1080C000984201D1002303860123838210BD00BFA3
:1080D00040420F00C4000020002C0140001000406E
:1080E0002DE9F74FA34F0C4697F86B6105461146F3
:1080F000006891469B462246731C87F86B31FFF758
:108100009BFF2B896868ADF8043018238DF8063082
:1081100001A902238DF8073009F0E7FCAB7A07F5D7
:10812000B677360107EB060A2C680C2B00F2F280BA
:10813000DFE813F00D00F000F000F0004D00F0005B
:10814000F000F0008200F000F000F000B600238C98
:10815000894823F001031B041B0C2384218CA28873
:10816000238B844223F073034FEA03434FEA134304
:1081700089B292B243F0700314D000F500608442DB
:1081800010D000F5406084420CD000F5806084423D
:1081900008D000F58060844204D021F0020141F053
:1081A000030107E021F00E0122F4407241F00301C7
:1081B00042F48072A2802383A4F834B02184238BFC
:1081C00023F008031B041B0C43F0080332E0238C4C
:1081D000694823F010031B041B0C2384218CA28804
:1081E000238B844223F4E6434FEA03434FEA1343CD
:1081F00089B292B243F4E04308D000F500608442B3
:1082000004D021F0200141F0300107E021F0E0012D
:1082100022F4406241F0300142F48062A280238364
:10822000A4F838B02184238B23F400631B041B0CB7
:1082300043F4006323836DE0238C4F4823F4807361
:108240001B041B0C2384218CA288A38B844223F063
:1082500073034FEA03434FEA134389B292B243F0E8
:10826000700308D000F50060844204D021F400714E
:1082700041F4407107E021F4606122F4405241F47E
:10828000407142F48052A280A383A4F83CB02184C0
:10829000A38B23F008031B041B0C43F0080338E0F6
:1082A000B4F820C0344A2CF4805C4FEA0C4C4FEAFE
:1082B0001C4CA4F820C0B4F820C0A388B4F81C80DB
:1082C0002CF4005C28F4E6484FEA08484FEA0C4CCE
:1082D0004FEA18484FEA1C4C94429BB248F4E048DD
:1082E0004CF4405C03D002F50062944203D123F4C5
:1082F000804343F48043A380A4F81C80A4F840B0DA
:10830000A4F820C0A38B23F400631B041B0C43F4CC
:108310000063A3832B7B43B1B4F844306FEA43433B
:108320006FEA53439BB2A4F8443023889BB243F0D6
:1083300001032380AB7A0C2B14D8DFE803F007137A
:1083400013130A1313130D131313100004F1340342
:1083500007E004F1380304E004F13C0301E004F118
:108360004003BB515046AAF80890CAF8044003B035
:10837000BDE8F08F581B0020002C01400C4B10B5BD
:1083800004462146186802F041F90A4A0823108879
:1083900080EA042010F4004F4FEA40001CBF80F434
:1083A000815080F00100013B80B2F3D1108010BDFC
:1083B0006C160020851600200FB407B504AB53F8E7
:1083C000042B05490020019303F07EFB03B05DF808
:1083D00004EB04B0704700BF09030108074B93F892
:1083E0000535012B08D1064B1868064BDB6898420F
:1083F00034BF002001207047002070475004002047
:10840000541400200C00002030B585B030B1264B4C
:108410001888B0F5805F34BF00200120234D10F094
:10842000010F234C23482449244A254B2D880AD088
:10843000007891F8201012781B782580A070E170E8
:108440002271637119E0007891F8201012781B787E
:108450008DF806008DF807108DF8082001A8214638
:108460000622ADF804508DF809300EF09BFBC8B120
:108470000198BDF808302060A380532007F0FEFC6F
:10848000208807F085FEA07807F082FEE37801A837
:108490000193237902936379039307F0DEFD024B86
:1084A00000221A8005B030BDC81400201418002026
:1084B000841D0020B90D0020040F0020B8160020F4
:1084C0001E170020F8B50478054674B9314D2146D1
:1084D000B5F87622B5F878322F48013403F0B8FBAE
:1084E000042C05F10405F2D1F8BD2C490EF096FBE1
:1084F000A8B9284B4FF47A714FF4FA62A3F87612B8
:10850000A3F87822A3F87A12A3F87C22A3F87E12AB
:10851000A3F88022A3F88212A3F88422F8BD28468B
:108520000EF009FC032807462CD8284620210EF01F
:10853000A0FB044630B1441C20460EF0FCFB012594
:10854000064600E00546204620210EF092FB18B9B1
:10855000BDE8F84002F08AB801300EF0ECFB012DC6
:10856000F6D1A6F2EE2240F2DC539A42F0D8A0F205
:10857000EE229A42ECD8074B9C3703EB8707FE802C
:108580003881F8BD064800210322BDE8F84003F019
:1085900013BD00BF50040020E5C6010801B8010862
:1085A0001CB601082DE9F04FB5498BB004460EF01A
:1085B00035FBB449002820460CBF022501250EF0EA
:1085C0002DFBB1490028204608BF04250EF026FBEC
:1085D000002808BF082515F0090F00F0A881AB4856
:1085E00002F029F8002003F0F3FCA94CA94802F09E
:1085F00022F8A94802F01FF86279A84B013AA8486E
:1086000053F8221003F024FBA64803F021FB0027B7
:108610002646D4F81080002140460BF05DFA28B1C0
:10862000A14803F015FB9A4C002769E09F483946A2
:10863000D4F814B0D4F818A0D4F81C9003F008FBB8
:10864000404600210BF052FA10B1202001F0ECFF5F
:1086500006A9404603F0A3FE0146954803F0F8FA48
:10866000584600210BF042FA10B1202001F0DCFF47
:1086700006A9584603F093FE01468D4803F0E8FA38
:10868000504600210BF032FA10B1202001F0CCFF4F
:1086900006A9504603F083FE0146854803F0D8FA48
:1086A000484600210BF022FA10B1202001F0BCFF57
:1086B00006A9484603F073FE013701467D4803F0E2
:1086C000C7FA0C2F04F11004A3D1A9E749B294F81A
:1086D000E62094F8E730009194F8E910764801918B
:1086E00094F9EA100734029194F9E410039194F894
:1086F000E51004913946013703F0AAFA102F03D090
:1087000094F8E8100029E1D16C4801F094FF6C4C1A
:10871000D6F8088054F8041F19B16A4803F098FA93
:10872000F8E70F46684B53F8274054B10123BB408C
:1087300013EA080F03D06548214603F089FA013790
:10874000F0E7634801F077FF624FD6F80885012310
:10875000A34013EA080F14BF5F486048B9680134AA
:1087600003F076FA122C07F10C07F0D15C4801F007
:1087700062FF00239A1992F834220AA90A4459493F
:10878000595C0133082B02F8101CF3D106A9564896
:1087900000278DF8207003F05BFA544801F04BFF7E
:1087A000534800F073FB534801F045FF504805F073
:1087B00065F9514801F03FFF4D4805F0EDF84F488D
:1087C00001F039FF4A4805F01BFF4D4801F033FF27
:1087D000474805F07CFE4B4803F03AFA4448FFF75F
:1087E00071FE494801F027FF414805F035F84FF088
:1087F0000E0808FB07F800240122A240434B1B6827
:108800004344D3F80A301A4240F0A18001340E2CC0
:10881000F2D10137082FEAD13D4803F019FA0020C0
:1088200006F0FAFB3B4801F006FF314805F058FF1F
:1088300015F0080F384C71D02368002093F83440AD
:1088400096F8586408F0D2F9002007F059F9012091
:1088500007F056F9022007F053F9012008F0C6F995
:10886000002007F04DF9012007F04AF9022007F037
:1088700047F9304608F0A8F9204604F0E5FA56E03A
:1088800031C10108F8C60108FEC6010802C7010887
:108890005004002010C7010822C7010834AC0108A9
:1088A0002EC7010839C7010846C7010853C7010888
:1088B00046CE01089EC601086BC701085BC70108C8
:1088C0009CAC01088AC70108A0AC010898C7010840
:1088D000A5C70108E0CA0108B4C70108C1C701085B
:1088E000CDC70108D0CB0108D9C70108E2C70108EC
:1088F0000FBF0108F1C70108FDC701080BC8010837
:1089000015C8010824C8010832C80108E819002068
:10891000EAD001083EC801084018002096F8580423
:1089200008F064F9236893F8340007F0E9F8AA071F
:1089300004D50B4B93F8580408F058F96B070CD585
:10894000084B1B6893F8340007F0DAF805E0064896
:108950003946224603F07CF958E70BB0BDE8F08FAA
:1089600050040020401800204BC8010808B50848F2
:1089700003F06EF907F07AF9FEF75AFC18B9642093
:1089800001F09FFEF8E70348BDE8084003F060B936
:1089900062C801086FC801082DE9F04FBC4B89B0CF
:1089A00018881D46DFF81483002840F0B28098F83C
:1089B0000335012B05D198F80405B0F1200460427D
:1089C000604100F00100B34FFFF71EFD03F0D6FB3E
:1089D00049203C6807F052FAAF4B2546186807F06B
:1089E000D7FB55F8040B07F0D3FB284607F02AFC09
:1089F00004F1100007F026FC10260122B240A74D1A
:108A00002B681A4205D004EB860353F8240C07F0B8
:108A1000CEFB0136132EF0D104F12800032107F01C
:108A20003DFCB8F8D030B4F92E00C01A07F0B0FB06
:108A30002B68D80408D59A4B1888B4F86C30C01A43
:108A4000C0F30D0007F0A4FB2B68990403D5B4F81C
:108A50006E0007F09DFB2B685A0504D504F17400E5
:108A6000032107F01BFC2B681B0502D5206F07F0C4
:108A70009EFB2B685E0402D5E06F07F098FB2B6825
:108A8000180403D5B4F8800007F082FB04F130002D
:108A9000032107F003FC04F13600032107F0FEFB7D
:108AA00004F13C00042107F0F9FBB4F94400B8F8E4
:108AB000D0300126C01A07F06BFB7A4B1B789E4220
:108AC0000ADA04EB4603B3F94400B4F94430013642
:108AD000C01A07F06CFBF0E72B68990505D5B4F9CF
:108AE0006600A0F2DC5007F062FB3B686E4A6F49FB
:108AF0007B60BB609B1A9B104B430321013393FBAC
:108B0000F1F101EB41015B1A842101FB03223A6080
:108B1000A5E1674B1C68674B1A6894420ED01C6035
:108B2000654B1B78093B012B08D8452007F0A6F9B7
:108B3000002007F0A3F9204607F02AFB98F8033538
:108B4000298898F8042519440139B1FBF2F002FB99
:108B500010129A4280F086814E4C0120FFF754FC9F
:108B600003F00CFB50202668656807F087F9A268BF
:108B7000236810681B68102718446368A1461B68A7
:108B8000A0EB430007F013FB72686B686846D31ACA
:108B90000093B268AB68D31A0193F268EB68D31AFA
:108BA000029307F04FFB32692B696846D31A009392
:108BB00072696B69D31A0193B269AB69D31A0293D4
:108BC00007F04BFA0121B940344B1A68114209D021
:108BD000BB00F2182B4452F8240C53F8243CC01A62
:108BE00007F0E5FA0137132FECD10023F218B2F9A0
:108BF0002810EA18B2F928208A1A4DF813200233F7
:108C0000082BF3D103ABADF10401002753F804297D
:108C1000BF00FFB26AB102F108000F2802D847F086
:108C2000010706E08032FF2A94BF47F0020747F0B1
:108C300003078B42EAD1384607F020F90024A24608
:108C4000A34607F00302022A18D0032A38D0012ACB
:108C500055D1BBF1000F06D15DF8043093461B01DE
:108C60005FFA83FA4BE05DF804004FF0000B00F070
:108C70000F0040EA0A0007F001F940E0BBF1000FE5
:108C800027D05DF80400C0F3031040EA0A002FE08B
:108C9000A4180020E42F0020A81800209818002015
:108CA0009C180020840C0020F02F0020E1830F3E50
:108CB0008431002080310020601400205004002006
:108CC0005DF80400BBF1000F08D1C0F3072007F0E6
:108CD000D5F81DF8040007F0D1F810E0C0F3033018
:108CE00040EA0A0007F0CAF85DF80400C0F3071074
:108CF00007F0C4F85DF804301B015FFA83FA04340E
:108D0000102C4FEA97079CD1BBF1010F02D15046BE
:108D100007F0B4F858490B6813F4805406D0B6F83D
:108D20006C10B5F86C2001248A1A00929A040AD5B6
:108D300008A901EB8402B6F86E00B5F86E10013494
:108D4000411A42F8201C5F0510D500AA02EB8401ED
:108D50000022B018B0F97470A818B0F97400381A6D
:108D600041F812000232062AF3D10334180508D55F
:108D700008A901EB84002A6F316F01348A1A40F888
:108D8000202C590408D508AA02EB8400F16FEA6F81
:108D900001348A1A40F8202C1A040BD508A901EBDB
:108DA0008403B5F88020B6F8801001348A1A43F89D
:108DB000202C00E0F4B1012C03D1009807F0F7F962
:108DC00018E000A9631E01EB8402002052F8041D84
:108DD0004000C0B209B140F00100013BF6D507F0F8
:108DE0004DF800275DF8270008B107F0E0F90137DA
:108DF000A742F7DB3020032107F030FA36200321A9
:108E000007F02CFA3C20042107F028FA1B4B4420E1
:108E1000197807F023FA184A13689B0506D5B6F9A6
:108E20006600B5F96630C01A07F0C1F9D9F8043008
:108E3000D9F80020C9F80830114B1249C9F80420AC
:108E4000D21A92104A430321013292FBF1F101EB55
:108E50004101521A842101FB0233C9F800300A4B48
:108E600001221A7098F80535012B01D106F0A4FFF4
:108E700009B0BDE8F08F00BF98180020840C0020D6
:108E8000F02F0020E1830F3ED8140020F0B50278C7
:108E900087B08AB94A4C04F1280594F8A42200232B
:108EA000484950B2595681426ED00C333C2BF7D111
:108EB0000834AC42F1D181E0002204920592461CB4
:108EC0000DF039FFC4B260B201F03AFB074618B1A9
:108ED0008DF81040012500E00546304620210DF0B8
:108EE000C8FE044638B1441C20460DF024FF01356D
:108EF000ADF81200EDB20026204620210DF0B9FE9B
:108F0000B0B3441C20460DF016FF00222E495FFA34
:108F100082FC51F82230834204D00132082AF5D174
:108F2000002300E0634651F82320824220D1022E24
:108F30000FD0032E12D05A1E012ED2B204D0042A12
:108F400013D88DF814300EE0042A0ED88DF81530A1
:108F500009E0052B09D88DF8173004E09A1E052A80
:108F600003D88DF816300135EDB20136042EC3D189
:108F7000052D04D807B0BDE8F04001F077BB04AB85
:108F800003CB3860796019E094F8A9020E4B94F88D
:108F9000A86253F82000B4F8A622009094F8AB021F
:108FA00053F82000019094F8AA0253F8200053F8D7
:108FB00026300290054802F04BFE79E707B0F0BD7D
:108FC00050040020480A002018B40108E9CB010829
:108FD0002DE9F74F434802F03BFE434C0025434B3D
:108FE000D4F800B0D4F804801A680023934206DA5B
:108FF0003F4951F82310A14203D00133F6E7002383
:1090000000E00123E16A226B0091616AA06A01918C
:10901000002B5ED05FFA85F94FF47A76B9F1010F33
:10902000B2FBF6F61ED1334B18880AF069FB3249C1
:109030000AF0BEFB01464FF07E500AF06DFC0AF0CC
:10904000A3FD2E4B87B293F8E831012B02D997FB91
:10905000F3FA15E02A48294642465B4602F0F8FD3D
:10906000BA4612E00AF04CFB23490AF0A1FB014684
:109070004FF07E500AF050FC0AF086FD1FFA80FA8D
:10908000204829465A4602F0E3FD9DE806001E48A6
:10909000534602F0DDFDB6F57A7F05D34FF47A71C1
:1090A0001A48B6FBF1F101E01948314602F0D0FD53
:1090B000B9F1010F09D1114B93F8E831012B04D913
:1090C000144841463A4602F0C3FD1348314602F0C7
:1090D000BFFD01350F2D04F1340480D103B0BDE88C
:1090E000F08F00BF08CC0108C8000020B414002095
:1090F00070140020D8320020BD378635500400207F
:1091000020CC010815CC01082ECC010858CC010850
:109110005ECC010863CC0108EAD001082DE9F041DA
:10912000FCF710FB10B9042006F046FAA74C03F038
:10913000F3F8A74940F2145220460DF042FD94F88E
:1091400058345C22012B84BF002384F8583494F8EF
:109150005834A04902FB034303F5687393F83420A5
:109160009D4F0A700C213B6001FB02339B49363353
:10917000A2680B6042F2010313403BB944F20803BA
:1091800013401BB94FF4005002F018F8A368DB0736
:1091900003D54FF4005002F009F8A3685E0409D526
:1091A000082002F003F84FF4005001F0FFFF012007
:1091B00001F0FCFFA3681D0706D54FF4005001F035
:1091C000F5FF012001F0F2FFA368980413D54FF4D6
:1091D000004001F0EBFF7D4B93F81E32012B03D1D1
:1091E0004FF4006001F0E2FF4FF4803001F0DEFF49
:1091F000402001F0DBFFA368590603D54FF480300F
:1092000001F0D4FFA3689A040DD503F42063B3F5ED
:10921000206F08D16D4B93F81E32012B03D14FF410
:10922000006001F0C3FF6E4B6E4A98461360002247
:109230001146A318B3F8A6325D0805F077359808F3
:1092400000F033305D1B2D1AD80800F011302D1AB4
:1092500005EB251505F00F35FF2095FBF0F013F019
:109260000106284418BF013100F0FF0018BFC9B241
:10927000012809D9022840F0A680002E00F0A38022
:1092800013F0BC0F00F09F800832282AD1D1013999
:10929000012900F2988003F0B5FD002130225248E8
:1092A000524D0DF0B2FC524B3E681D60514B0020F8
:1092B0001E6002F0F1FF504B80F0010018704F4B20
:1092C00005F58D711960D4F8E0214D4B1A604D4BB6
:1092D00005F5FE721A60307801F01AFC4A4B05F56C
:1092E000E4721A6094F8982264214A43474BC832CA
:1092F0005A6000229A60DA601A615A619A61DA61F2
:1093000083F8202083F82120414B05F5AC721A60C8
:10931000D4F8F4213F4B404E1A60404B05F18602D1
:109320001A603F4B05F1F6021A603E4B05F1080248
:109330001A603D4B05F5DE721D603C4BB4F8E4014C
:109340001A6005F5E3733360394BC3F800800AF007
:10935000DBF938490AF0E0FAF060B4F8E6010AF007
:10936000D3F934490AF0D8FA94F80C32321D7371EB
:1093700094F88A323F6833742F4BB0601A602F4BD9
:1093800005F594721A602E4A2E4BB4F80E021A603C
:1093900077610AF0B9F901462B480AF0BDFA2B496A
:1093A0000AF006FA2A4A2B4B05F5A97111602A4AE0
:1093B000186005F59673B761F36115603362BDE817
:1093C000F04102F093BA02F07DFF64E75004002000
:1093D00000F80108AD170020401800209019002067
:1093E00084060020280F00207C1700202005002084
:1093F0009C150020A0150020280000203419002012
:10940000C0180020CC13002038170020040F0020C3
:1094100040290020CC280020A01D0020E8190020B1
:109420000C1A0020A8190020AC1900209419002063
:10943000A419002000401C46200E0020B82800205F
:109440003661023DA8280020000061444C3D0F44D5
:10945000481800208C18002060180020026D70B59C
:1094600015880446ADB2A90613D5036B8BB9C36A40
:109470001BB1908880B298470BE0E16992884069FF
:109480004E1CD2B2E6614254E169E268914228BFC3
:10949000E3612B0614D5636AA26A9A42236D0BD04E
:1094A000511CA069A162825CD2B29A802369994260
:1094B00006D30023A36270BDDA6822F08002DA606E
:1094C00070BD08B501F063F9094908220B8883EAE9
:1094D00000239BB213F4004F4FEA43031CBF83F4F5
:1094E000815383F00103013A9BB2F3D10B8008BD95
:1094F000701600202DE9F34101F0BCF88D4D6B6A28
:10950000C31A002BC0F2308200F5433303F5A07379
:109510006B62894B95F828201E78C6F38006B21A34
:1095200018BF012285F828604EB1002A00F01C8285
:10953000824B5A789A7001225A701A7025E07F4B3C
:109540002AB1DA7842F00202DA709A785A70D97841
:1095500001F0020404F0FF023CB9784CA468041B3B
:10956000002C03DB01F0010200E0012202F0010403
:109570001C70724A4CB1CC0707D51379704901337E
:1095800003F003031371CB5C53706C4CDFF804825F
:1095900023787BB3E37823F00203E370694B034441
:1095A000AE20A36009F093FB08B109F095FB88F8A1
:1095B0000000002800F0D881B02009F088FB40208E
:1095C00009F085FB002009F082FB102009F07FFBE9
:1095D0004FF48067013F0020BFB209F005FB002F68
:1095E000F8D1384609F0E7FB6278574B53F8220070
:1095F00009F064FB98F80030002B00F0B581637827
:10960000052B00F27081DFE813F008006E011900ED
:10961000750006002B0100241DE14C494C4A4D4BBE
:109620004D4802F0EFFC012009F0C5FB4A4809F063
:1096300045FB022009F0BFFB484852E1484B1A683D
:10964000984612F0020F2ED0464C0A232188464F2E
:10965000B1FBF3F203FB121339789BB200913E4841
:10966000424902F0CFFC01F013FE012009F0A3FBF8
:10967000394809F023FB3E4B3A781868248803796F
:10968000642102FB13444C43C1780220CB1A5A4395
:10969000B4FBF2F4E4B209F08EFB2146152009F088
:1096A000C1FA032400E00124D8F80030180540F185
:1096B0001A81304B30491F680968642397FBF3F225
:1096C00003FB1273009124482C4902F09BFC01F02B
:1096D000DFFD204609F06FFB1F4809F0EFFA05F0A7
:1096E000FBFB0746601C09F066FB1520394609F0B4
:1096F00099FAF8E00120224F09F05DFB214809F0BA
:10970000DDFA3B68990747D51F4B20495A68124834
:1097100000929A68032401921B681D4A02F072FCB1
:1097200001F0B6FD022009F046FB0B4809F0C6FA2D
:1097300033E000BFA01D0020DA320020040E00201C
:10974000E5CB0108404B4C0058AD01087ACC01082C
:1097500083CC01085DBF0108C91D002089CC010828
:10976000700900209E190020C00000208ECC010846
:10977000641400207015002068150020A6CC010894
:10978000100E0020BBCC01084C150020D1CC0108E4
:10979000E0CC0108FC0D002002243B68DA0717D555
:1097A000734B74495A68744800929A6804F101082E
:1097B00001921B68714A02F025FC01F069FD204608
:1097C00009F0F9FA6C4809F079FA5FFA88F844462A
:1097D0003B681B0715D56A4B66495A686648009274
:1097E0009A68671C01921B68664A02F00BFC01F044
:1097F0004FFD204609F0DFFA5F4809F05FFAFFB23B
:109800003C46614A5C48B2F90210B2F9003000915E
:10981000B2F904100A2291FBF2F2019255495B4A17
:1098200002F0F0FB01F034FD204657E00E2C5AD038
:109830006008013009F0BFFA204609F01CFA3B78B5
:10984000A34206D9202009F0D4F9601CC0B209F067
:1098500012FA0234E4B24E4F3B78A342E6D842E01B
:109860004C4C4D4994F85824434802F0CBFB01205E
:1098700009F0A1FA404809F021FA484B48491F78FD
:109880003D483A4602F0BEFB022009F094FA3A48FD
:1098900009F014FA5C235F43E31993F8D4330C22E4
:1098A00002FB037707F5747727443E49FA79BB79C1
:1098B000314802F0A7FB01F0EBFC032009F07BFA32
:1098C0002D4809F0FBF9397BBA7AFB7A2A480091D6
:1098D000354902F097FB01F0DBFC042009F06BFA3C
:1098E000254809F0EBF9002E3ED1304BB02093F81B
:1098F0002030052B97BF2E4A3F249B181C7E09F071
:10990000E6F90C2009F0E3F9162009F0E0F9204609
:1099100009F06FF9B02009F0DAF9022009F0D7F95F
:10992000172009F0D4F9234B1B78002B224B14BFCE
:10993000722021201B78002B18BF522009F059F902
:10994000B02009F0C4F9082009F0C1F9172009F086
:10995000BEF995F83F40194B185D013404F003043B
:1099600009F047F985F83F4002B0BDE8F08100BF3B
:10997000B0180020D1CC0108C91D0020E4CC01089A
:10998000581500200AD3010836180020E8CC010839
:10999000E80F002050040020ECCC0108AD17002097
:1099A000F8CC010809CD01081ACD0108040F0020E8
:1099B00058AD0108B81600201E1700202CCD010854
:1099C000024B1B689B0300D594E57047700900208B
:1099D00038B5044600F04EFE2B4B2C4D1A68821A07
:1099E000B2F57A7F83E8050007DD29492820087051
:1099F000284900222A701A720A70297861B93D2C10
:109A000005D03E2C3ED101221A72234A03E0214A9E
:109A100001201070214ADA60D8681B4A4454013191
:109A2000C9B2062929701A4C16D1127A012A02D11C
:109A30008278282A07D9174A11780129114604D1BA
:109A40008278092A01D8227038BD002228202A7085
:109A500020701A720A7038BD23788B4212D1137AA3
:109A6000012B04BF022313720A4B1A78012A05D175
:109A700002221A7000F0FEFD094B186000232B70C3
:109A80002823237038BD00BFE01D0020F60F002002
:109A9000F70F0020651A0020F01D00206E1A00202C
:109AA000681A00202DE9F04F8FB00391074600217E
:109AB0001646AF480C2202939DF860809DF8649092
:109AC000AC4D0DF0A2F800211422AB480DF09DF82A
:109AD000AA4BDFF8F4B22C78A3F118024FF0000A79
:109AE000012C8CBF1C46144651460C228BF838A022
:109AF0008BF839A00BF13C000DF087F82320CBF850
:109B0000484000F0DEFD752001210DF11702FDF740
:109B1000FBF95C46A0B19A4B50462364994B012156
:109B2000636406AA432384F83C30FDF7EDF99DF801
:109B3000183003F07E038DF8183000284CD154E023
:109B400094F84C3083BB03F1804303F504339A69E6
:109B5000DFF878A242F008029A6110238DF82230D3
:109B60004FF4805B0323504608A98DF82330ADF8ED
:109B700020B007F0BAFF844BCAF810B01A8822F060
:109B800040021204120C1A801A8822F038021204C1
:109B9000120C42F008021A801A8892B242F0400277
:109BA0001A80012384F84C3008AA75200121FDF7A2
:109BB00029FB9DF82030A3F17002012A01D9AF2BB7
:109BC00065D1052384F83830432384F83C306F4B4B
:109BD00023646F4B63645AE0682B06D1012384F839
:109BE00038301D2384F83C3051E09DF8173003F0E5
:109BF0007E03682B8DF8173044D10223062084F8A9
:109C0000383008AA236C014698479DF823309DF808
:109C1000252003F0010302F001025B0043EA820306
:109C20009DF82120DFF8A0A102F00102134303F008
:109C3000FF0B9BB1BBF1010F01D100231FE0BBF172
:109C4000020F03D1012384F8393020E003F003032D
:109C5000032BF7D0032005F0AFFC18E0DAF8403012
:109C60000C20012107AA98479DF81C3013F00F0320
:109C7000F0D0042B02D18AF839B008E001238AF829
:109C8000393004E0702B04BF042384F8383094F892
:109C9000383040490020022B08700BD1364A3E482C
:109CA00010603E4850603E48D0603E48106101223E
:109CB0000A701FE0012B0DD12F4A3B480B7010603A
:109CC000364804235060394890603548D0603548A4
:109CD00010610FE0043B012B00F28383264B344AD2
:109CE0001A602E4A5A602E4ADA602E4A1A610123FF
:109CF0000B7007232F4A13702F4B19689B4641F0B6
:109D0000010119602D4B00221A709C46082F00F2A9
:109D10004683DFE817F00900440309005D00730083
:109D200092005D00A900A9002B78012B50D84FF0BC
:109D3000000A0EAB03F818AD532051460122CDF8AE
:109D400004C0FCF7D3FFDDF804C0002840D09DF824
:109D50002030E52B3CD1064B194A84F84DA01A60FF
:109D6000184A5A6004238CF8003002238BE000BFAD
:109D7000C0280020DB3200202C0E002090AD01080E
:109D8000096F0008712701080038004005720008BB
:109D900085710008BC180020852B0108D117010827
:109DA000B517010890C1793D5DF600087D170108DF
:109DB0007D530008D8030020100E0020DE32002062
:109DC00031280108BD6F0008E01D0020000C014093
:109DD00094F83830022B11D16C4B6D4A1A606D4AE1
:109DE0005A606D4A92F83920002A14BF6E226F2201
:109DF0001A7201238CF80030032344E02B78012BE6
:109E00001BD800220EAB03F8182D1C200D210122B7
:109E1000FCF76CFF88B19DF820302A2B01D01A2B5B
:109E20000BD15A4A5D4984F84E3011605C495D4B54
:109E3000516002221A70042325E000210EAB03F8C2
:109E4000181D18200122FCF751FF68B19DF8203041
:109E5000FB2B09D14D4B544A1A60544A5A60514B5E
:109E600001221A7005230EE094F83830043B012BD0
:109E700000F29582454B4E4A1A60464A5A60494B59
:109E800001221A7008234B4A5370DBF8003043F06C
:109E90000203CBF800302B78012B05D1FDF73AF9FE
:109EA000454B4FF400525A61042E00F2BB81DFE8AB
:109EB00016F00500C2016600050080010A2000F0CE
:109EC00000FC7720A021012207ABFCF70FFF002840
:109ED00055D01E2101227720FCF7C8FE4FF42F60D9
:109EE00000F0E4FB0026A6F160010027C9B20222BF
:109EF00008AB77208DF820708DF82170FCF7F6FE06
:109F00009DF821309DF8201043EA0121224B03F1F6
:109F10005002B1520236102EE5D1B3F85EE00121B5
:109F20000EF00F060EF47F4EA3F85EE03A463B4675
:109F300022F001002044B0F85000002818BF002192
:109F4000D70703D5C0B24340082002E083EA1023BC
:109F5000FAE71F0448BF83F4C05301384FEA4303B4
:109F6000F7D10132102AE3D146EA0E0E0A4AA4F8CC
:109F70005EE021B9C3F303339E4200F0158294F8EA
:109F80006040054ED4B102264EE100BFC02800203B
:109F9000592B010819180108E01D00207D27010830
:109FA0001D6F0008DE3200200D280108776F0008C1
:109FB00069530008D803002000100140A84FFDF7A6
:109FC000A9F84FF0280B4FF4804A384607A9ADF89E
:109FD0001CA08DF81EB007F088FD4FF400533B61C4
:109FE0005846A04905F05CFB0E21022007F068FDF1
:109FF0000823CDF820A008A84FF0010A8DF82530DD
:10A000008DF824408DF826A0FCF7C2F98DF818B021
:10A0100006A84FF0030B8DF819B08DF81A408DF893
:10A020001BA004F051F9142000F04BFBD021772045
:10A03000524607ABFCF75AFE3946002800F0A080D4
:10A040009DF81C30A6F884B0552B86F87B3040F084
:10A050009780D121524607AB7720FCF747FE9DF849
:10A060001C30772003F00F021B0986F87C2086F84D
:10A070007D30162208ABAA21FCF738FE9DF820207F
:10A080009DF8213043EA0223A6F864309DF822208F
:10A090009DF8233043EA0223A6F866309DF8242079
:10A0A0009DF8253043EA0223A6F868309DF8262063
:10A0B0009DF8273043EA0223A6F86A309DF828204D
:10A0C0009DF8293043EA0223A6F86C309DF82A2037
:10A0D0009DF82B3043EA0223A6F86E309DF82C2021
:10A0E0009DF82D3043EA0223A6F870309DF82E200B
:10A0F0009DF82F3043EA0223A6F872309DF83020F5
:10A100009DF8313043EA0223A6F874309DF83220DE
:10A110009DF8333043EA0223A6F876309DF83420C8
:10A120009DF8353043EA0223A6F8783041F2707387
:10A13000A6F8883046F67813A6F88A304A4BC6F857
:10A140008C304A4BC6F89030494BC6F89430494B96
:10A15000C6F89830484BC6F89C3096F8603043B942
:10A1600008F0FCFA42F6E06000F0A0FABC68C4F324
:10A170008034424B01221C70414B83F8602002E77F
:10A18000404B1A6822F480421A6000233E4C354E40
:10A190001A195068B04206D11857282803D1002355
:10A1A0005360137002E00833182BEFD14FF40053C3
:10A1B0004B61334C94F8A060002E40F00C811420C9
:10A1C00000F07FFA04F1A1037620D0210122FCF7F0
:10A1D0008DFD94F8A130582B2DD104F1A4038821D2
:10A1E00018227620FCF782FD7620F4213122FCF73C
:10A1F0003DFD012384F8A030244BA4F88860C4F806
:10A200009030234BC4F88C3045F6D813A4F88A302C
:10A21000204BC4F89430204BC4F898301F4BC4F83E
:10A220009C30D8E0012E06D01D4B9E701D4B1A6845
:10A2300042F004021A601B4E33689B0702D51A4B8A
:10A240001B689847B8F1000F30D0B8F1070F14BF62
:10A250004FF47A737D2318BF4FF0010927E000BF48
:10A2600000100140F5B300085D270108CD6E00081D
:10A2700037270108796E0008A1160108AB000020FD
:10A28000E01D002000040140983200209D160108C6
:10A290009F1601082D270108296E0008C114010826
:10A2A000D8030020100E0020C02800207D2309F1D3
:10A2B000FF395FFA89F909FB03334B4A4B4F1360AF
:10A2C0004B4B87F8C0901B6840469847494B2D7808
:10A2D000A3F11802039C012D8CBF1D461546464B69
:10A2E0000022042C1A70984679D8012202FA04F34D
:10A2F00013F01A0171D113F0050F6ED00EAB03F8F5
:10A30000181D1E200A21C7F8C450FCF7EFFC0028D6
:10A3100063D09DF82030482B5FD1384B384A1A6003
:10A32000384A5A60032388F80030374B0222DA702B
:10A33000336843F008033360344B93F8C7210AB104
:10A3400033490A7093F8C8210AB132490A7093F868
:10A35000C9310BB188F8003033682F4C13F0080F67
:10A3600019D0029A642692FBF6F5284609F0CCF93A
:10A37000029B074606FB153000B209F0C5F92749D4
:10A3800009F016FA0146384609F00AF9244909F09D
:10A390000FFA206001E000232360012021E0012F5B
:10A3A0007FF679AD0027ADE442F21073A2F8883051
:10A3B000A2F88A301B4B0326C2F88C301A4BC2F825
:10A3C00090301A4BC2F89430194BC2F89830194BA0
:10A3D000C2F89C3028E7042626E7012CACD90024DB
:10A3E0007DE70FB0BDE8F08F58140020E01D00207D
:10A3F0002C0E0020C0AD0108DF320020140E00201A
:10A4000089280108696D0008D80300205004002045
:10A41000BC180020DE3200209C2800208988883C5F
:10A420000000204123270108096E000819270108B0
:10A43000196E00081913010870477047034A044B4E
:10A44000128808B11A6170475A617047BC0D00202C
:10A4500000080140034A044B128808B15A61704752
:10A460001A617047BC0D002000080140074910B573
:10A470000A6852B1064B642418686043054CB0FB6F
:10A48000F2F2228000220A601A6010BDBC14002083
:10A49000C01400201018002003685A1C02601970B4
:10A4A0007047044B1B68DA79511CD9711344187A30
:10A4B000704700BF1C15002010B50C4908220B88FE
:10A4C00083EA000414F0010F4FEA530318BF83F42A
:10A4D000204302F1FF3214BF83F001039BB212F05C
:10A4E000FF024FEA5000EBD10B8010BD861A00200E
:10A4F00030B5084900230A780C4607495D56854265
:10A5000003D1FF25013A5D54D2B20C333C2BF4D178
:10A51000227030BD440A0020480A00200023074A68
:10A520001A445168814203D00C333C2BF7D1704759
:10A530000023C36213815360704700BF480A0020A4
:10A5400010B5084B01461A680023D41894F902404C
:10A55000901C8C42184403D00833282BF5D10020DE
:10A5600010BD00BF400A002038B1438811EA030043
:10A5700003D08B4214BF02200120704730B50B4B33
:10A580000B4A1C681378042B0DD8591C04EBC30329
:10A590009D88C9B2284203F1020302D01170184607
:10A5A00030BD0B46EFE71370002030BD400A00209D
:10A5B000A81E0020014B00221A70DFE7A81E002011
:10A5C00010B544780078002303FB03F11939614387
:10A5D00001F6C4115943414340F6C41291FBF2F114
:10A5E000034A22F813100133072BEDD110BD00BF31
:10A5F000B217002010B5427A044632B1036804F164
:10A600000A01406898470023637210BD10B5447A70
:10A61000037A621CD2B2044493424272A17202D8FD
:10A62000BDE81040E6E710BD014B01461868EDE7B4
:10A63000E0140020EAE710B5441E14F8011F21B110
:10A64000024B1868FFF7E2FFF7E710BDE0140020A7
:10A6500008B50448FFF7EFFF034B1868BDE8084052
:10A66000C8E700BF4DCD0108E01400200048E2E734
:10A6700052CD010810B50A4A0A491368886800BF1C
:10A6800012689342F7D1084A11684FF47A7202FBBC
:10A6900001F4201AB0FBF1F002FB030010BD00BF73
:10A6A0009432002010E000E06809002038B504462C
:10A6B000FFF7E0FF0546FFF7DDFF401BA042FAD39E
:10A6C00038BD10B504462CB14FF47A70FFF7EEFF99
:10A6D000013CF8E710BD08B50F4B1A780023D9B23A
:10A6E000914207D20D49002051F823100133096827
:10A6F0000880F4E73220FFF7E4FF094B1B685A0398
:10A7000008D5084B9B685B0304D4BDE8084040F2C1
:10A71000DC50D6E708BD00BF840C0020340C0020BC
:10A72000700900205004002008B5024B1B689847B0
:10A7300008BD00BFB432002008B503685B6A03B1EE
:10A74000984708BD08B503681B6A03B1984708BD60
:10A7500008B503689B69984708BD08B503685B693D
:10A76000984708BD10B504462046FFF7F6FF18B914
:10A770000A20FFF7A6FFF7E710BD08B50368DB68FE
:10A78000984708BD08B503685B68984708BD10B5D1
:10A79000054C23681868FFF7F5FF0028F8D02368F8
:10A7A000BDE810401868E8E76816002010B5054CB1
:10A7B0002068FFF7E7FF18B12068FFF7DEFFF6E734
:10A7C00010BD00BF381A002008B503681B68984701
:10A7D00008BD014B1868F7E72815002038B5094C6B
:10A7E000094B05460022206824215A70FFF7ECFF30
:10A7F00020685421FFF7E8FF20682946BDE838406B
:10A80000E2E700BF5C1A0020A81E0020054B10B52F
:10A81000044621461868FFF7D7FF034B5A78544087
:10A820005C7010BD5C1A0020A81E002010B5044604
:10A83000C0B2FFF7EBFF200ABDE81040E6E7024B8D
:10A840001868024B5978BFE75C1A0020A81E002048
:10A85000A0F17D03012B70B504460D460A4E05D8C4
:10A8600030687D21FFF7B0FF84F020043068214676
:10A87000FFF7AAFF35B12B881C4404EB142404F025
:10A88000FF042C8070BD00BF4C1A002030B585B08D
:10A8900004AC002524F8025D0091ADF806002146C5
:10A8A0001020FFF7D5FF9DF806002146FFF7D0FFE7
:10A8B0009DF807002146FFF7CBFF9DF800002146D9
:10A8C000FFF7C6FF9DF801002146FFF7C1FF9DF885
:10A8D00002002146FFF7BCFF9DF803002146FFF769
:10A8E000B7FF9DF80E002946C043C0B2FFF7B0FF86
:10A8F00005B030BD38B5054C05465E212068FFF730
:10A9000063FF20682946BDE838405DE77C270020CA
:10A91000014B5E21186857E77C27002010B50A4CD0
:10A920005E280146206805D15D21FFF74DFF2068B4
:10A930003E2105E05D2903D1FFF746FF20683D2158
:10A94000BDE8104040E700BF7C27002010B504465A
:10A95000C0B2FFF7E3FFC4F30720BDE81040FFF7E4
:10A96000DDBF38B500240F4D21460F4870222C70F2
:10A970000CF04BF921460D4B1B680B4493F9022058
:10A9800072B11C6808480C500A18988807319080EA
:10A990009B79702993712B7803F101032B70EAD115
:10A9A00038BD00BF480D0020490D00208C0A002052
:10A9B000094B0E221B6802FB0030437AFF2B07D0A5
:10A9C000064A12789A4203D9054A32F8130000E089
:10A9D000808800B2704700BFE8190020E80F00200F
:10A9E0002E0F0020454B2DE9F74F1D68444B29469B
:10A9F000D3F800B0434B1C68434B1E68304608F048
:10AA0000D7FE59460090304608F0D2FE2146074650
:10AA1000304608F0CDFE59468146284608F0C8FE6B
:10AA200021468246284608F0C3FE21468046584605
:10AA300008F0BEFE59460646584608F0B9FE0146E3
:10AA400008F0AEFD21460190204608F0B1FE014617
:10AA500008F0A6FD019983464FF07E5008F09EFD58
:10AA6000594608F09BFD294C49462060504608F0A5
:10AA700095FD014608F094FD39466060404608F0B7
:10AA80008FFD014608F08CFD4946A060504608F055
:10AA900087FD014608F084FD2946E060284608F05D
:10AAA00087FE014608F07CFD01464FF07E5008F01D
:10AAB00075FD5946054608F071FD00992061304644
:10AAC00008F06CFD014608F06BFD394660614046B8
:10AAD00008F064FD014608F063FD0099A06130466E
:10AAE00008F05EFD014608F05BFDE0612846019933
:10AAF00008F054FD206203B0BDE8F08F90280020DC
:10AB00009428002098280020B00000206818002019
:10AB1000044B20B1022814BF034A044A00E0044A4F
:10AB20001A607047D403002081210108591C0108D4
:10AB300099C9000810B5084C0021606808F0CCFFE6
:10AB400038B1064B186808F0DBFD054908F030FE07
:10AB50006060606810BD00BFA81E00205C1400206B
:10AB6000BD37863538B50546487E08F0CDFD0C4921
:10AB700008F0D2FE0B4B044633F915000028D8BF6D
:10AB8000404208F0C1FD084908F0C6FE01462046D3
:10AB900008F00EFE01464FF07E5008F0FFFC38BD75
:10ABA0000000C8421C1800200000FA43194B2DE990
:10ABB000F0411D6806460E2D984627DC0023AB4267
:10ABC00006DA154A52F82320B2421FD00133F6E7C5
:10ABD0000024AC421ADC104FA10057F82430601C4E
:10ABE00073B92A1B07EB80003944920001350BF042
:10ABF000F1FF47F82460C8F800500120BDE8F0815B
:10AC00001A7D337D9A42ECD30446E2E70020BDE88A
:10AC1000F08100BFB414002070140020102870B51B
:10AC200002D00E2803D970BD144B186803E0144BF2
:10AC3000342202FB003021B9124B00221C681D4651
:10AC400006E0C368002BF7D0BDE87040AEE70A46C7
:10AC5000A24212DA0C4B53F8221003EB8206814217
:10AC600002F10101F3D1A21A304603EB81019200F7
:10AC7000013C0BF0AFFF2C6070BD70BDC414002010
:10AC8000C8000020B4140020701400202DE9F843FF
:10AC90000C463049164608F08BFD0546304608F054
:10ACA0002FFD2D4908F084FD01464FF07E5008F03D
:10ACB00033FE0146284608F02FFE06460CF02AFA1D
:10ACC000054630460CF0B2F924490746304608F0F4
:10ACD0006FFD294608F020FE0CF01CFA01462846BC
:10ACE00008F066FD394606464FF07E5008F056FCE7
:10ACF0004FF07E518046304608F052FC4FF07C51B8
:10AD00000546404608F054FD294608F005FE294650
:10AD100081462060404608F0FFFD4FF040416060F2
:10AD2000C4F80890384608F043FD294608F0F4FDC1
:10AD30003146E0604FF07E5008F030FC294608F0C4
:10AD4000EBFD00232061A36163612362E361BDE841
:10AD5000F88300BFDB0FC940BD378635CA92283F54
:10AD6000F0B56FF003074F438D004C1E5319002CB4
:10AD700009DD03EB070C53F8086CAC444CF8046C89
:10AD8000013C043BF3E71060002003468B4204DAE9
:10AD900052F8234001332044F8E790FBF1F0F0BD76
:10ADA0002DE9F0410C464E69CD690968074608F067
:10ADB000FFFC61688046304608F0FAFC01464046D8
:10ADC00008F0EEFBA1698046A06808F0F1FC01469E
:10ADD000404608F0E5FBE1688046284608F0E8FCBC
:10ADE0000146404608F0DAFB216A8046206908F0F7
:10ADF000DFFC0146404608F0D1FBA6616761256291
:10AE0000E061BDE8F081F8B507460C4648680021CE
:10AE100015461E4608F060FE48B11149284608F064
:10AE2000C7FC01464FF07E5008F076FD6060616817
:10AE3000304608F0B5FB0146304608F06DFD256848
:10AE400006462946384608F0A9FB0146304608F078
:10AE5000AFFC0146284608F0A3FB2060F8BD00BF08
:10AE6000DB0FC9402DE9F04102780346202A00F1AA
:10AE70000100F9D0092AF7D02D2A02D10346414D0D
:10AE800004E02B2A08BF03464FF07E551E460024DF
:10AE9000334616F8012BA2F13007F9B209290DD873
:10AEA0003949204608F084FC0446384608F02CFC5A
:10AEB0000146204608F074FB0446E9E72E2A17D124
:10AEC000314F334616F8010B3038C2B2092A0FD879
:10AED00008F01AFC394608F01FFD0146204608F02C
:10AEE0005FFB29490446384608F062FC0746E8E75C
:10AEF0001A7802F0DF02452A38D15A782D2A02D179
:10AF00000233012604E02B2A14BF0133023300264A
:10AF1000013B002713F8012F303AD1B2092903D899
:10AF20000A2101FB0727F5E7B7F59A7F28BF4FF401
:10AF30009A77B8464FF07E51B8F1070F07D9084607
:10AF4000124908F035FCA8F108080146F4E707F0BB
:10AF5000070737B108460C4908F02AFC013F0146B3
:10AF6000F7E72EB1204608F0D7FC04E04FF07E5101
:10AF7000204608F01DFC0146284608F019FCBDE8F3
:10AF8000F08100BF000080BF0000204120BCBE4C0B
:10AF9000F0B50124B0FBF4F58D4201D34C43F9E741
:10AFA0000026DCB1B0FBF4F504FB1500B4FBF1F4B2
:10AFB0001EB9002D01DC002CF3D1092D03F101078E
:10AFC0005FFA85FC04DD002A0CBF5725372500E019
:10AFD000302565441D7001363B46E2E71C70F0BD2C
:10AFE000F0B50124B0FBF4F58D4201D34C43F9E7F1
:10AFF0000026DCB1B0FBF4F504FB1500B4FBF1F462
:10B000001EB9002D01DC002CF3D1092D03F101073D
:10B010005FFA85FC04DD002A0CBF5725372500E0C8
:10B02000302565441D7001363B46E2E71C70F0BDDB
:10B0300070B50646B6FBF2F40846154614B1204634
:10B04000FFF7F6FF05FB1464024B1B5D00F8013BA4
:10B0500070BD00BF60CD01082DE9F843089E002BAC
:10B060000746884614460CBF4FF020094FF03009C0
:10B07000334613F8012B0AB9254603E0002CFBDD0B
:10B08000013CF6E7002D04DD38464946C047013D46
:10B09000F8E724EAE4742546331B595D19B13846B4
:10B0A000C0470135F8E72846BDE8F88380EAE07339
:10B0B000A3EBE0738B4206DB002801DD401A7047EA
:10B0C00002D0084470470020704770B5044608F06D
:10B0D00035FD2030402857D820462C4908F024FD63
:10B0E00028B120462A4908F059FA0446F4E72046D8
:10B0F000284908F0FBFC28B12046254908F050FA01
:10B100000446F4E72046244908F00EFD30B12249F8
:10B11000204608F043FA01461F480AE020461F492E
:10B1200008F0E4FC40B11C49204608F039FA014619
:10B130001A4808F033FA04462146204608F038FB46
:10B1400005462946204608F033FB002106462846DE
:10B1500008F02EFB124908F021FA0146284608F0B3
:10B1600027FB104908F01CFA0146284608F020FB8E
:10B170000D4908F013FA0146304608F019FB014664
:10B18000204608F00DFA70BD002070BDDB0F49406D
:10B19000DB0FC940DB0F49C0DB0FC93FDB0FC9BF65
:10B1A00092E741399730083C15A82A3E024B9A682D
:10B1B00022EA00009860704750040020024B9A6811
:10B1C00010439860704700BF500400200A4B1A8853
:10B1D00001321A80094B1A6801321A60084B1A882A
:10B1E000013292B2202A04D100221A80054B1A881B
:10B1F00001321A80704700BFC8140020A818002030
:10B20000A41800207E310020114A30B50028B8BFB4
:10B210004042104C90FBF2F304FB03003C256843D2
:10B220000D4D90FBF2F22D682D7B25B903EB8303C6
:10B2300003EB830301E0C3EB031302EB830304FB83
:10B2400002020B804FF47A7392FBF3F24A8030BD16
:10B2500080969800806967FFD0130020022803D0F1
:10B26000431E584258417047064B1B681B7823B158
:10B27000054B1868C0F3C0407047044B1878C0F302
:10B2800080007047CC130020A0180020DA32002084
:10B2900008B507480BF0FAFCC0B21428044B04D8D8
:10B2A000421C20211954D0B2F7E700221A5408BDDD
:10B2B000C91D0020074A13689B020AD5064B0021CE
:10B2C000197001684FF6FE730B4003604FF40013D2
:10B2D0005360704700000240DD3200202DE9F0414C
:10B2E00005460BF0D3FC2E4B04469E6888B92D48CA
:10B2F000FFF7A1F92C4B53F8241041B10123A340CF
:10B30000334202D0294800F0A3FC0134F2E7284878
:10B3100021E02846274922460BF0C0FC58B92648B0
:10B32000FFF789F9254C54F8041F0029EFD01F4876
:10B3300000F08EFCF7E72B7800262D2B03BF01359C
:10B3400004F1FF344FF001084FF00008164B53F89A
:10B35000267027B91A48BDE8F041FFF76CB92846B6
:10B36000394622460BF09AFCB8B90120B0400306DA
:10B3700001D51448EFE7B8F1000F03D0FFF716FF2F
:10B38000114802E0FFF71AFF1048FFF754F9394659
:10B390000F48BDE8F04100F05BBC0136D6E700BFC6
:10B3A0005004002085CD0108A0AC01088FCD010814
:10B3B000EAD0010893CD010898CD01089CAC0108A2
:10B3C000A4CD0108B3CD0108C1CD0108CACD010843
:10B3D0009DC6010810B5054C23681869FAF7CAFF25
:10B3E00018B123681A69024B5A6110BDA41E0020CF
:10B3F0000004014008B54FF48040FAF7BBFF012874
:10B4000005D1034B4FF480425A61024B187008BDBE
:10B4100000040140C42F002010B5074C23681869B0
:10B42000FAF7A8FF30B123681A69044B5A61044B3C
:10B4300001221A7010BD00BF281E00200004014028
:10B44000B01E0020826A8169436B1144D960416A51
:10B45000914203D98A1A5A60816204E001698A1A0A
:10B460005A6000228262002280F844201A6842F06A
:10B4700001021A607047F0B5884C894A23689D8A9A
:10B48000ADB2E9B211F0010F32D0198821F4006198
:10B490000904090C1980198889B241F48061198066
:10B4A000002151707F4908787F49A8B1907818B978
:10B4B0007E480078FF280FD1012090707C480078EA
:10B4C000022804D1188880B240F4006018800978FE
:10B4D00041F00101198203E1097801F0FE011982AE
:10B4E000724B1B78FF2B00F0FB80FF235370F7E0BB
:10B4F0008F073CD5BFF35F8F6D490878C0B2012834
:10B5000014D1684D2D788DB195787DB1198821F4CD
:10B5100080610904090C1980BFF35F8F198B1988AA
:10B52000D07089B241F4007119801BE0188BBFF311
:10B530005F8F087802280BD15A48007840B1907884
:10B5400030B1198821F480610904090C1980C1E027
:10B550000978032906D15349097819B1917800294E
:10B5600040F0B880998889B241F48061B7E04E0715
:10B570005BD50121D1704B49097800293AD09178E7
:10B58000002937D04A49507809784A4D022919884C
:10B590001ED921F480610904090C19801F8A2E68C4
:10B5A000C1B2FFB240B23754188880B240F4007084
:10B5B00018808B1C5370236828681D8A013149B29A
:10B5C000EDB24554998889B241F48061998027E0B1
:10B5D00089B241F4007119801E8A2D68C1B2F6B299
:10B5E00040B22E541B8A481C40B2DBB203312B54AC
:10B5F000517015E0917811B92F49097841B1198836
:10B6000089B241F40071198053780133537007E017
:10B61000198889B241F480711980214B01219970F8
:10B6200021680B88D805FCD45AE001F0400101F0F4
:10B63000FF061F48F1B11F49B3F810C00F685178D9
:10B640005FFA8CFCCDB26E1C49B2F6B207F801C0AD
:10B650005670077876B2F11C8F4205D1998821F493
:10B6600080610904090C99800378B34238D102350E
:10B67000557035E0290633D551784DB26F1C1FD077
:10B680000E4E01313668C9B2755D5170EDB21D8242
:10B69000007849B2884223D11CE000BF141B00206F
:10B6A000B01E00201C1B0020191B00201A1B0020AC
:10B6B000281B0020241B00201B1B0020201B002017
:10B6C000134956700978C9B219821249097809B923
:10B6D000017829B9998821F480610904090C9980BD
:10B6E0000D4B92F9011018780C4B421C91420DD170
:10B6F00000229A70DB7833B12268938823F4407378
:10B700001B041B0C9380064B00221A70F0BD00BF77
:10B710001A1B00201C1B0020281B0020B01E00202C
:10B72000291B0020F8B50468054620460E4617463A
:10B7300006F079F9032845D8AB7A9B089AB246B946
:10B740004FF0020C0CFA03F3A18989B221EA03033A
:10B75000A3810A2101FB00211B4B43F82160043126
:10B7600043F8217046B1AA7A0225920805FA02F23E
:10B77000A1890A4392B2A281282202FB003000F183
:10B780002002EFF31286502383F312880023C1189E
:10B790000D6915B115600A6904320433102BF6D116
:10B7A00000231360F3B283F31188036A23B1A389E2
:10B7B0009BB243F0010304E0A38923F001031B04BF
:10B7C0001B0CA381F8BD00BF8C09002070B5046D6F
:10B7D0000546A389866823F400531B041B0CA38130
:10B7E000837986B013F0020F0CBF00204FF4005095
:10B7F00013F0040F6B790CBF00214FF4806113F03C
:10B80000010F14BF042200229B07238A48BF42F085
:10B8100008029BB223F4405340EA03032382A38926
:10B8200048BF92B29BB223F4B05323F00C030B43F6
:10B830001A43A281A38A01A823F440731B041B0CA2
:10B84000A38200F0B9FE2549049A039B8C4208BFED
:10B850001346A2891921594312B2002AB4BF7600B7
:10B86000B600B1FBF6F16423B1FBF3F2120110094B
:10B8700003FB1011A08900B2002806DAC90032319A
:10B88000B1FBF3F303F0070305E009013231B1FB2B
:10B89000F3F303F00F031A4392B22281AA792B6DBE
:10B8A00012F0010F06D00E498B4203D1042001F59E
:10B8B0004841086112F0080F9A8A03D092B242F010
:10B8C000080203E022F008021204120C9A829A89FC
:10B8D00092B242F400529A8106B070BD0038014025
:10B8E00000440040417171E781606FE708B5FEF7E1
:10B8F000C1FE064B02221860054B1A70054B1A68F0
:10B90000054B9A60012283F8212008BD9016002083
:10B910008C16002094320020040F00202DE9F04FF7
:10B92000624C63686249581C0A78894602F0FF0C31
:10B930000AB10346F6E7277B667BA57B2169636036
:10B94000E0461FFA88F213B21F2B00F39380594987
:10B9500001EB8300C278807831F82310C0F1FF003A
:10B9600080B2002861D0C0F1FF0050433C23B1FBFE
:10B97000F3FA0012BAF1050F5AD8DFE80AF0030B08
:10B980001A283846161A4E43C5B2B6FBF3F62E44B3
:10B99000F6B248E0B1FBF3F703FB1717BFB2C5B22D
:10B9A000C7F13C07101A4743B7FBF3F72F4416467D
:10B9B00029E0B1FBF3F503FB1515C7B2ADB2101AC0
:10B9C0004543B5FBF3F53D44EDB2164630E0B1FB1F
:10B9D000F3F603FB1616B6B2C7B2C6F13C06101A50
:10B9E0004643B6FBF3F63E441546F6B220E0B1FB03
:10B9F000F3F703FB1717C6B2BFB2101A4743B7FBE2
:10BA0000F3F737441546FFB212E0B1FBF3F503FB41
:10BA10001515ADB2C6B2C5F13C05101A4543B5FBCC
:10BA2000F3F53544EDB2174602E0154616461746C3
:10BA30004FEA072A4AEA064A4AEA050A1723012179
:10BA400099400CF1170211EA0A0FC3EB02021A49DE
:10BA50000CBF0920112092B213F1FF338854EED2AB
:10BA60000CF1180C08F101081FFA8CFC1FFA88F879
:10BA7000124966E7012389F80030114B628140F2D8
:10BA80002A3227736673A5732161A4F808C05A602F
:10BA90000C4A00219184118889B241F00101118082
:10BAA0001A6842F001021A60BDE8F08FB01E002053
:10BAB000DD3200204C13002021100020BC1E00208D
:10BAC0006C000240000400402DE9F04F814689B02F
:10BAD0000F4615461E4600242978002900F0B48040
:10BAE000252902D001354846ABE06B78302B02D0D7
:10BAF0000235002202E0AB78012203350392A3F164
:10BB00003002092A4FF000081AD8A3F13002D1B24E
:10BB1000092907D80A2A13DC0A2303FB082815F889
:10BB2000013BF2E7A3F16102052A02D8A3F1570213
:10BB3000F0E7A3F14102052A02D8A3F13702E9E7B1
:10BB40006C2B03BF2B78012201350022642B29D0F6
:10BB500011D8252B73D002D8002B75D0BCE7582BF9
:10BB600040D0632BB8D1317806F104084846B84775
:10BB700001344646B0E7732B54D005D86E2BABD1B9
:10BB8000336804361C60A7E7752B02D0782B29D0C8
:10BB9000A2E706F1040B0DF1140A30680A219AB3EA
:10BBA00000222AE006F1040B0DF1140A306862B19C
:10BBB000002806DA2D238DF8143040420DF11503CC
:10BBC00000E053460A21002218E0002806DA2D235F
:10BBD0008DF8143040420DF1150300E053460A2160
:10BBE000002212E006F1040B0DF1140A3068102156
:10BBF0003AB1B3F15806724272415346FFF7F0F979
:10BC000005E0583B5A425A415346FFF7C1F9CDF877
:10BC100000A0484639464246039BFFF71DFA5E46A0
:10BC2000044459E7336848460093394642460023A6
:10BC3000FFF712FA06F1040A044456464CE7484658
:10BC40001946B847013447E7204609B0BDE8F08FF0
:10BC50000FB407B5064904AB53F8042B086805492F
:10BC60000193FFF731FF03B05DF804EB04B07047B8
:10BC7000E014002035A60008F0B504468FB0204639
:10BC80000BF004F8C5B21DBBA548FEF7D4FCA54CCB
:10BC900094F8E81009B9A4484EE049B294F8E620B7
:10BCA00094F8E730009194F8E910A048019194F9D4
:10BCB000EA100734029194F9E410039194F8E51026
:10BCC000049129460135FFF7C3FF102DE0D1E2E7CB
:10BCD0002046974905220AF0E1FF054690B99548AC
:10BCE000294670220AF091FF28468E4B0E2202FB55
:10BCF0000033013000220828A3F86021A3F8622154
:10BD0000F3D10AE120468C4904220AF0C7FF054618
:10BD10002046002D47D120210AF0ABFF002800F07B
:10BD2000FC80461C30460AF0B1FF2C460746834B88
:10BD300053F8245025B982480FB0BDE8F04087E79A
:10BD400030462946FAB20AF0A9FF01340028EED1A4
:10BD50007449002342180730702882F8EC3082F8CA
:10BD6000E83082F8E73082F8E6300E46F0D17549C7
:10BD700011F83420934211DA01EBC4014F68C3EB90
:10BD8000C302B0183A44176800F1E601C0F8E67043
:10BD900090880133888092798A71E8E76A48294659
:10BDA000FFF756FF8AE0694907220AF077FF054648
:10BDB0002046002D47D120210AF05BFF06460AF0FD
:10BDC00065FFC4B264BB6248FFF742FF2146614889
:10BDD0000134FFF73DFF0E2CF8D15348FFF738FF31
:10BDE00000245D482146FFF733FF00250122AA40C9
:10BDF0004C4B0E2101FB0433D3F8603157491A42F2
:10BE0000574B584818BF19460135FFF721FF0E2D33
:10BE1000ECD145480134FFF71BFF082CE1D17CE051
:10BE2000304651490AF08CFF2C46002848D0082C97
:10BE30004BD00AF080FF06AB18514B4900200AF0A6
:10BE40007FFF0434F1E748490AF07AFF002460B12B
:10BE5000082C35D00AF06FFF06AB43F824004249A6
:10BE600000200AF06DFF0134F1E7082C28D1069B71
:10BE70000F2B25D8079F072F22D8089E0D2E1FD8DD
:10BE8000099D05F16402C82A1AD80A9CFF2C17D80C
:10BE90000B99642914D80C9A642A11D891420FDAAC
:10BEA0000D9803280CD8C3EBC30E304B73449F711D
:10BEB000DE711D725C729972DA7218732C4CDEE6B8
:10BEC0000FB0BDE8F040FEF7D1BB069B072B20D892
:10BED000079A0D2A1DD8017872290DD06E2918D124
:10BEE00010490E2000FB0313012101FA02F2D3F8DE
:10BEF000601121EA020209E00A490E2000FB031347
:10BF0000012101FA02F2D3F860110A43C3F860215B
:10BF100001E0FEF7ABFB0D4CB1E60FB0F0BD00BF8A
:10BF2000DACD010850040020EAD0010805CE01084E
:10BF300001B801083605002021CE010834AC010803
:10BF4000A4CD01089092010826CE0108D2CD0108A7
:10BF500047CE010832CE010817CD010893B8010879
:10BF6000C8B7010837CE01083BCE010830050020D4
:10BF70000FBF010838B500240B4BE518E058FEF759
:10BF80005AFB696811B10948FFF762FEA96811B14F
:10BF90000748FFF75DFE07481034FEF74CFBB4F589
:10BFA000F87FE9D138BD00BF70A501083DCE01087A
:10BFB00043CE0108EAD0010830B505460C461346C9
:10BFC000294622460148BDE8304041E649CE0108F5
:10BFD00007B5064B06480093064B07490193074AED
:10BFE000074BFFF735FE03B05DF804FB54BF0108B3
:10BFF00068CE01085DBF010889CC010883CC010827
:10C0000048BF01080EB40FB505AB53F8042B0190DF
:10C01000064901A80393FFF757FD019B00221A7000
:10C0200004B05DF804EB03B0704700BF99A40008AA
:10C030000FB413B50B4904AB08680B4953F8042B34
:10C0400009680193FFF740FD0446084B1868FEF7A6
:10C0500084FB0028F9D0204602B0BDE8104004B0AF
:10C06000704700BF4C040020480400202815002021
:10C0700038B50A4CE179E07001F03F018B1C01F109
:10C080000A056371A57020460831FAF7B9FAA31EB4
:10C09000E854A378000A013C185538BD2914002043
:10C0A00010B500231A46D9B2814211D209490A4C6F
:10C0B0001944C97901334A40910081EA4201514053
:10C0C000D20802F0180244FA02F24A40D2B2EAE779
:10C0D000104610BD291400200007090E08B50020E5
:10C0E000FEF794FB0020FEF791FB0020FEF78EFB8D
:10C0F000BDE808400020FEF789BB1E4B30B518682C
:10C100003B2390FBF3F0B0F5C87F1B4A0DDC002801
:10C110000DDB11684B1C052B02D101231371002389
:10C1200002EB81018860136001E04FF0FF3012796B
:10C13000114BF2B103F1080017C888429B6902DD78
:10C140000546084629469C4202DD25461C462B46EC
:10C150008B42A8BF0B468442A8BF2046934202DD13
:10C16000194613460A468242B8BF10469842B8BFE5
:10C17000184630BDAC000020C41E0020354B10B561
:10C180001C68354B1B682360344B1A6862605A6820
:10C190009B68A260E360324B1A6822615A689B6810
:10C1A0006261A3612F4B1A68E2615A689B68226240
:10C1B00063622D4B1A8822855A8862859A88DB88AB
:10C1C000A285E385294B1A6822865A6862869B6895
:10C1D000A386274B1A68E2865A689B682287638782
:10C1E000244B1A88A2875A88E2879A88DB88A4F8A9
:10C1F0004020A4F84230204B1A780023934208DAFA
:10C200001E4804EB430130F813000133A1F8440049
:10C21000F4E71B4B1B88A4F86C301A4B1B88A4F85E
:10C220006E30194B1A68A4F874205A689B68A4F8F9
:10C230007620A4F87830154B1B682367FFF75DFF65
:10C24000134BE0671B88A4F88030124B5B89A4F87D
:10C25000663010BDE42F0020B8320020582A00209C
:10C26000642A0020702A00201C180020B01800202A
:10C270004C15002008180020840C0020B81900205C
:10C280007C310020EC270020581500201C1A0020CB
:10C290006C150020940A00200023094A1A4492F8E1
:10C2A0005914814205D192F85B1492F85C249142B2
:10C2B00004D30433502BF0D1002070470120704785
:10C2C0005004002038B52A2210480021104C0AF0F2
:10C2D0009CFC00220F4914F8010F53180425083262
:10C2E00083F8A40283F8A95205200025282A83F8A0
:10C2F000A80283F8AB5283F8AA02EBD10123A1F87C
:10C30000A632522381F8A23238BD00BFF2060020C7
:10C310003BB401085004002008B5FEF7ABF9074B09
:10C3200000F5B71000F558701860054B02221A701E
:10C33000044B9A6802F2DC529A6008BD9016002005
:10C340008C160020040F002070B50646441E14F819
:10C35000011F81B1084D28460AF08BFC0028F6D059
:10C3600005F108039842F2D2451B0448A31B284458
:10C3700080F83432EBE770BDD0CB010850040020C8
:10C38000031E10B50C4603DA2D2201F8012B58428A
:10C390000A22FEF74DFE00230370204610BD30B583
:10C3A00087B005460C4603A800210C220AF02DFC9C
:10C3B0002846002107F0B8FB20B12846284907F09D
:10C3C000EFF803E02846264907F0E8F8254907F08A
:10C3D000EFF907F0B3FB054685EAE570A0EBE570E1
:10C3E0006946FFF7CDFF002DACBF20232D23684603
:10C3F0008DF80C300AF04AFC012807D130238DF863
:10C400000D308DF80E308DF80F300CE0022805D17C
:10C4100030238DF80D308DF80E3004E0032804BF72
:10C4200030238DF80D30694603A80AF015FC03A8E7
:10C430000AF02CFC0338C5B22A4603A920460AF0AC
:10C440004FFC00236355204607490AF005FC03A969
:10C45000204629440AF000FC204607B030BD00BF4A
:10C460006F12033A00007A4488CE010801200021AF
:10C47000FAF78AB90023036043608360C3600361F5
:10C4800043618361C36103624362836270478A6868
:10C4900010B50C6A036814430A6923F4FF4314437C
:10C4A0004A6923F0700314438A691443CA69144328
:10C4B0004A6A14438A6A224313430360CB68436089
:10C4C0000B6883604B68C36010BD02684FF6FE7353
:10C4D000134003600023036043608360C3602A4B02
:10C4E000984222D0294B984229D0294B984230D0EB
:10C4F000284B984237D0284B98423ED0274B984241
:10C5000006D153F8682C42F4700243F8682C704747
:10C51000234B984206D153F87C2C42F0706243F8CA
:10C520007C2C70471F4B984206D153F8042C42F0E4
:10C530000F0243F8042C70471B4B984206D153F866
:10C54000182C42F0F00243F8182C7047174B984211
:10C5500006D153F82C2C42F4706243F82C2C70470F
:10C56000134B984206D153F8402C42F4704243F8E2
:10C57000402C70470F4B984205D153F8542C42F48D
:10C58000702243F8542C7047080002401C000240FF
:10C590003000024044000240580002406C0002405B
:10C5A00080000240080402401C04024030040240A3
:10C5B00044040240580402401F4B10B55A6802F070
:10C5C0000C02042A03D0082A04D01C4A14E01C4A96
:10C5D000126811E05A685968C2F38342C90302F134
:10C5E000020201D4174906E0596811F4003F1449CA
:10C5F000096818BF49084A4302605968124AC1F3E2
:10C600000311545C0168E14041605C68C4F302249A
:10C61000145D21FA04F484605C68C4F3C224145DE0
:10C62000E140C1605B68C3F381331A44137CB1FB02
:10C63000F3F1016110BD00BF0010024000127A004A
:10C640000000002000093D00ECAD0108024B1A6912
:10C6500022EA0000186170470010024010B504463D
:10C66000F9F7F4FC012806D11CB1F9F7EFFC013C05
:10C67000F8E7052010BD002C08BF052010BD00BF45
:10C680002DE9F8432F4B1B685B0758D52E4E2F4DD5
:10C6900037783446012F07D0AB689847EB68984746
:10C6A000012333706B8844E02B6998476B68984787
:10C6B0006B69301D264998472648D6F808C000689F
:10C6C000254900780CF101038342D1F8009072688B
:10C6D000884602D1214B1F700023E1684E1C032EB7
:10C6E00003D1194801260674002604EB81014A6132
:10C6F000217C1548E66069B142698169C0698A4256
:10C7000002DD16460A4631468142A8BF01469142E3
:10C71000A8BF0A4604EB8C010A6204EB8301096A94
:10C72000A360C1EB090900234A4423702B88C8F891
:10C7300000200B4A642B38BF642312681361BDE8E4
:10C74000F88300BF100E0020E01E0020681E0020AD
:10C75000201A0020C01D0020B4270020A827002098
:10C76000C4140020F8B50024224BE0B21F78B84270
:10C770000FD2214B33F81010204B53F8203033B137
:10C780000B2804D81E4A12780AB1DB689847013496
:10C79000EAE71C4B1B685B032AD500251A4E2B4683
:10C7A000EAB2BA4224D2726854689C4218D0204639
:10C7B00005F039F9EFF31283502282F312881349FE
:10C7C0004FF0280CA28C0CFB001092B20132426296
:10C7D000A28ADBB292B242F00102A28283F31188F4
:10C7E00056F8043F00221B6801351A802346D7E71C
:10C7F000F8BD00BF840C0020B8190020340C0020C4
:10C800001C00002070090020300C00208C09002042
:10C810000C4B10B51B68DB0613D50B4B1A680B4B82
:10C8200019683C318A420CD3094C1A6023680B20EA
:10C830005A681B881361FDF739FF23685A681B8803
:10C84000536110BD100E0020943200200010002013
:10C85000FC0F00202DE9F84F80460AF017FA414DF1
:10C860000646D5F80875B0B93F48FFF7F1F901233E
:10C87000B3403B4207D03D4B0C2202FB06333C4801
:10C880009968FFF7E5F90136122EF0D1C7B939489A
:10C89000FDF7D1FE14E04046374932460AF0FEF972
:10C8A000DFF8C8A0044668B93448FDF7C4FE0AEBB7
:10C8B00004032F4899680C34FFF7CAF9F02CF6D11D
:10C8C0002F481BE098F8003000242D2B03BF08F1FF
:10C8D000010806F1FF364FF001094FF000090C2363
:10C8E00003FB04A3D3F808B04046594632460AF089
:10C8F000D5F938B10134142CF1D12248BDE8F84FF4
:10C90000FDF799BEB9F1000F12D0122C01D11E4BC8
:10C9100003E0132C04D1D5F80C35C5F8083505E033
:10C92000012303FA04F42743C5F80875174811E0FA
:10C93000122C02D1C5F808950BE0132C02D1C5F8D2
:10C940000C7506E0012303FA04F427EA0407C5F88E
:10C9500008750F48FDF76FFE59460E48BDE8F84FC1
:10C96000FFF776B9500400208ACE0108E0CA01081A
:10C970009BCE010894CE010893CD0108A0CE0108FA
:10C98000EAD00108A4CD0108FFFF0300C1CD0108D2
:10C99000CACD01089DC601082DE9F04F87B0059367
:10C9A000B34B0546B3F80080049108F002081FFA63
:10C9B00088F30392ABB1AF4BB3F90280B3F9003007
:10C9C000B8F1000FB8BFC8F10008002BB8BF5B4238
:10C9D0009845B8BF9846B8F5007FA8BF4FF40078D7
:10C9E00000E09846002426462746A24B0422F15E2A
:10C9F000A14BDFF8C8A254F803C0A04B9CFBF2F295
:10CA0000BCF1000FB8BFCCF1000C4800BCF5206FA2
:10CA1000C2EB000E54F80390BAF800B011DC0BFB27
:10CA20000EFC09EBEC29DFF898C2B9F57A5FA8BFD4
:10CA30004FF47A59E145ACBF44F8039044F803C081
:10CA400003E04FF0000C44F803C08D4BDFF82CC21C
:10CA500093F800905CF804C08A4BB9F1000F06D13E
:10CA6000DFF8609299F80090B9F1000F0ED053F8FA
:10CA70000490C9F100039C4503DBE145B4BF4B467C
:10CA80006346DFF8F8C144F80C3006E0BCF1000F53
:10CA9000B8BFCCF1000C43F804C0DFF8E0C1EB19DB
:10CAA00054F80C9093F801A093F80BC04FEAE919E1
:10CAB0006F4B0CFB09F90AFB00F01B884FEAA91920
:10CAC0009B074FEAA01043D0DDF80CC04900CCF121
:10CAD0000003994203DB63469942B8BF0B466A499B
:10CAE000DDF814C036F901A03CF90610CAEB030AC0
:10CAF0008A44664942F2107C635853446345A8BF98
:10CB00006346DFF8C4C16345B8BF63466350297A02
:10CB100095F81CC001FB0AFA0CEB8C0C4FEAEA1AE0
:10CB2000CCF100018A4503DBE245B4BF51466146C2
:10CB300095F812C0401A0CFB03F31B13C3EB090951
:10CB400008FB09F908FB00F003EB692901EB602001
:10CB50004F4B95F82C1013F807A04E4B0AFB02FA26
:10CB6000A0EBAA10029029B9995F23F806E0C1EB67
:10CB70000E0102E0995F9A53891AC1EB01414FEA15
:10CB80004B1B91FBFBFAD5F820B00021584606F06C
:10CB9000A3FF88B9FDF7CEFF03465046019306F088
:10CBA000B3FD3D4A0C2101FB0721019B5A46FEF7CC
:10CBB0002AF906F0C3FF824695F8301041B1374B91
:10CBC0003022504602FB0732FEF7CAF84FEA400A0D
:10CBD000334B029913F807B032480BFB0AF2494471
:10CBE0005211314B114490F800E089B2F1521846CD
:10CBF000BEF1000F05D009B24FF0030E91FBFEF11C
:10CC0000F1520299DFF8C4B0284B44F80B100137F9
:10CC10002749022F44F80190E25006F1020604F180
:10CC200004048A4699467FF4E0AE0499114B8A7950
:10CC3000B3F904300F3252005A430F4B52119E6821
:10CC4000042396FBF3F6961B0C4B002AB8BF524206
:10CC5000322A99686C7B3BDC04FB0611154A914231
:10CC6000A8BF1146144A9142ACBF99609A6031E066
:10CC7000141800201C180020B018002040170020B5
:10CC80003C1700207C2A0020361800205C1700206A
:10CC9000CE170020C01F0020A4290020C41F0020A0
:10CCA000D41700205817002098190020702A00205F
:10CCB000642A0020FEFFFF0F020000F05C14002039
:10CCC00080C1FFFFB0190020F0D8FFFF582A0020D4
:10CCD00000229A60EA7856431F4AB6111278032A56
:10CCE0000BD9E98DB1F5C87F07D24A42964203DBE2
:10CCF0008E42B4BF32460A4616469C686FF0FF0368
:10CD000044F34F34B4F5807FA8BF4FF480749C4245
:10CD1000B8BF1C4637196D6ABFB28780002128460C
:10CD200006F0DAFE70B9FDF705FF804638B206F06E
:10CD3000EBFC434609492A46FEF765F806F0FEFE7D
:10CD4000074B98800023CBF80860CAF80840C9F860
:10CD5000083007B0BDE8F08F840C00208C2900203B
:10CD600098190020244B2DE9F04F1A68234BC2F389
:10CD700040721B68C7781A428278214BC2F164095D
:10CD800002EB8208C2F100040CBF0D884FF47A75E3
:10CD90005FFA89F94FEA4808C7F1640AA4B203F1BF
:10CDA000180CA6B230B2002804DC002E14BF1646C0
:10CDB000012600E04E4600FB00FB76430BFB07FB21
:10CDC0009BFBF6F6564470434FF00A0B90FBFBF0CA
:10CDD000404480B258804E8800B2761B70434FF4B6
:10CDE0007A7690FBF6F0284423F8020F5C44634502
:10CDF000A4B2D6D1BDE8F08FA018002070090020A1
:10CE0000D817002010B50D4C2068FDF7D9FB20681D
:10CE10000023047A03FB03F11939614301F6C411BD
:10CE20005943192291FBF2F1054A22F813100133FC
:10CE3000072BEFD1BDE81040024993E7901900207D
:10CE4000C0170020200500200A4B032888BF0220BD
:10CE50001870094B5C2193F858244A43991881F8BB
:10CE6000D4030C2101FB00200449034403F2D63310
:10CE70000B60C7E7AD170020500400209019002078
:10CE80000E4B1B6813F4805F0D4B0CD00D4A1268DB
:10CE9000920008D4008AB3F90630421A93420ADDA0
:10CEA0000844834203E0B3F90620438A9A42B4BFA0
:10CEB0000020012070470120704700BF700900204A
:10CEC0002E0F0020A0180020094B30B51D68094B1B
:10CED00005F480551868084B1C6800230DB1828842
:10CEE00000E0A28805495A520233182BF6D130BD12
:10CEF00070090020A8190020AC190020D0190020CA
:10CF00002DE9F843704B1B78012B0FD1FDF7B2FBD5
:10CF10006E4C6F4AD4F874311268C01A6D4B988009
:10CF2000801AD880FDF7A6FBC4F874016A4B1A6812
:10CF3000994692F90820A2B9684D2B78013B182B2D
:10CF400000F29380DFE803F05191916E9191916628
:10CF500091919191917991919191916E8591917920
:10CF600051005A4F0023A7F87831B7F87861574D30
:10CF700034B2072CE0DC95F87A3105F5BE787BB940
:10CF8000D9F80030B3F9060006F0BEFB504B24215F
:10CF90001A6801FB0481FDF779FE012385F87A31D7
:10CFA0004F4D35F9140006F0AFFB242101FB04813D
:10CFB000FDF7F6FE0AF070F84A4B0E221B6880B2AD
:10CFC00002FB043225F81400B2F9003000B2984296
:10CFD000B2F9022003DB13B29842B8BF0346013610
:10CFE00025F81430A7F87861BFE7D9F800301B792D
:10CFF0001BB13B4B0020598908E03B4B1B7803F0E9
:10D00000040303F0FF00002BF3D1014604F04DFDB3
:10D0100001242BE0324C0020E18804F046FD012081
:10D02000218906E02E4C0020218904F03EFD618913
:10D03000012004F03AFD022418E00024284BE0B25D
:10D0400003EB44039988013404F02FFD062CF5D13D
:10D050000CE00024224BE0B203EB4403D9880134F6
:10D0600004F023FD042CF5D100E000241F4B1A68C6
:10D070001E4612F0200F02D12B78052B0BD1184D34
:10D080002046298804F011FD601CC0B2698804F0B4
:10D090000CFD0234E4B23368DB0206D4144B1B7877
:10D0A00083B1BDE8F843FFF75DBB0025114B601964
:10D0B00003EB4503C0B2198904F0F7FC0D2DEDD048
:10D0C0000135F3E7BDE8F8836C090020E01E00207D
:10D0D0005C1400200818002094190020840A002005
:10D0E000940A0020E8190020DA320020700900209C
:10D0F000BA0D00202E0F002008B50D4B1B68DB0475
:10D100004CBF0C4B0C4B1B689A880C4B19780023B6
:10D11000D8B2884204D20A4820F813200133F7E736
:10D12000FFF720FBBDE808403220FDF7CABA00BF78
:10D1300070090020A8190020AC190020840C0020E0
:10D14000B8190020074B1B68B3F5BC7F08D2064B0B
:10D15000B3F8E40028B1054B1868C0F3804070476D
:10D16000012070475C14002050040020700900204A
:10D170002DE9F0431D469D4B8DB09842894690465F
:10D180009DF8507053D19A4C9A4BA26023609A4BF1
:10D190009A4A636103F58073A3614FF48073E3607F
:10D1A0002361974B62632363A3F54843543BE364D5
:10D1B000A36403F55743FC339A69206542F4804227
:10D1C0009A615A693C0742F001025A614FF002032A
:10D1D0008DF803304FF40073ADF8003001D51C23F7
:10D1E0000FE0A80706D51823864869468DF8023057
:10D1F00004F07BFCE9070AD54FF48063ADF80030FA
:10D200004823804869468DF8023004F06EFC0E23F6
:10D210008DF804300022012301A88DF805308DF827
:10D2200006208DF80730724C01F04EF89DE0764BE9
:10D2300098424AD1754B6F4AC3F808801A604FF480
:10D240008072DA601A61724A18655A6102F580725A
:10D250009A61704A9A64DA646F4BDA6942F4003278
:10D26000DA615A6942F001025A6102238DF80330F3
:10D270003A074FF00403ADF8003001D51C230EE04F
:10D28000AB0706D518235F4869468DF8023004F0D5
:10D290002CFCEE0709D50823ADF800304823594887
:10D2A00069468DF8023004F020FC26238DF8043006
:10D2B0000022012301A88DF805308DF806208DF895
:10D2C0000730524C01F000F84FE0544B984240F0C8
:10D2D000F280534B474AC3F808801A60514A1865D8
:10D2E0005A6102F580729A614FF48072DA601A61B5
:10D2F0004D4A3C079A64DA64474BDA6942F480226B
:10D30000DA619A6942F008029A614FF002038DF8DF
:10D3100003304FF48063ADF8003001D51C230FE0DB
:10D32000A80706D51823414869468DF8023004F055
:10D33000DCFBE9070AD54FF40063ADF80030482361
:10D340003A4869468DF8023004F0CFFB27238DF868
:10D3500004300022012301A88DF805308DF8062045
:10D360008DF8073000F0B0FF2D4C0026012384F823
:10D3700044302662E661A6626662C4F82C9065714C
:10D38000C4F80880A7712046FEF720FAEA0757D5AF
:10D39000236B002B4CD001A8FFF76CF8E36C206BDB
:10D3A00001934FF480530A9380230693E3680B960E
:10D3B00004932023099363690596029307960896C0
:10D3C0000396FFF782F801A9206BFFF760F8236B43
:10D3D0001A6842F001021A60226D918A89B241F006
:10D3E000400191825B689BB2236429E000380140D0
:10D3F0003032002000AE01087C21002044000240B1
:10D40000580002400008014000440040DC31002088
:10D410007C230020044400400010024000480040EB
:10D42000883100207C25002004480040000C014089
:10D43000236D4FF6DF721A80DA6842F02002DA605C
:10D44000AB0730D5636B002B28D001A8FFF712F88B
:10D45000A36C002501934FF480530A938023069315
:10D460002369606B0493102303930B95059507952F
:10D4700008950995FFF729F8606B01A9FFF707F8F0
:10D48000636B1A6842F002021A605D605D60236D92
:10D490009A8A92B242F080029A8204E0236DDA689E
:10D4A00042F08002DA60236D20469A8992B242F4FB
:10D4B00000529A8100E000200DB0BDE8F0832DE914
:10D4C000F34188469DF8206011461A469DF82430A5
:10D4D000054600201A4C07190457AC4203D00C3003
:10D4E0003C28F7D126E0388920BB022D0FD005DC7F
:10D4F00055B1012D1ED1009312480AE01E2D0DD00A
:10D500001F2D17D1012009E000930F4801E00F48BB
:10D5100000933346FFF72CFE044605E005F04CF877
:10D5200031460446FDF714F934B12571A7F8088097
:10D530007C6001E0002000E0204602B0BDE8F08100
:10D54000480A0020004400400038014000480040E4
:10D55000574B73B51878FDF781FE564D04462B786E
:10D56000834223D0D0B1544B1B68FBB193F9000028
:10D5700002230093514B04211B6800225B78003387
:10D5800018BF012301934FF41653FFF798FF4C4B3C
:10D59000C3F8000650B101232B7007E0484ED6F8BF
:10D5A0000006FCF7BBFFC6F800462C70454B464D05
:10D5B0001878FDF753FE2B780446834218D088B1C3
:10D5C000424B1B68A3B10022012493F900000821FB
:10D5D0004FF4964300940192FFF771FF3C4B1860A3
:10D5E00028B905E03A4E3068FCF798FF34602C709B
:10D5F000384B394D1878FDF731FE2B7804468342BD
:10D6000029D000B3354B1B682BB3354A93F9000082
:10D610001268032352782021002A14BF092208220D
:10D62000009301924FF461430022FFF748FF2D4B16
:10D63000186080B12C4A012313702B702B4B1A6891
:10D640002B4B1A6007E0274E3068FCF767FF264B2C
:10D6500034601C702C70274B274D1878FDF7FEFDA9
:10D660002B780446834220D0C8B1244B1A68E2B11B
:10D67000D37992F90000002B4FF00202204C08BF32
:10D6800002230092002254F8233001921021FFF768
:10D6900016FF1C4B186040B101232B7005E0194E9A
:10D6A0003068FCF73BFF34602C7002B070BD00BFE7
:10D6B000D8130020101A0020D4130020D01300200B
:10D6C0007C210020E4130020261A0020E013002013
:10D6D000381A00201C1400204A1A002018140020B8
:10D6E000141400204C1A0020501A002094320020FC
:10D6F000541A0020281400205B1A00202414002053
:10D7000018B401085C1A002073B5094C054620685E
:10D710000E46FCF703FF002295F9000000960192E7
:10D7200008214FF49643FFF7CAFE206002B070BD97
:10D73000381A0020F7B5274C274DE369284643F4F3
:10D740008043E361236901A943F4804323611823E3
:10D750008DF806304FF42043ADF8043003238DF8E4
:10D76000073004F0C2F904234FF480470DEB0301A6
:10D7700028468DF806304FF48056ADF8047004F05A
:10D78000B4F91023284601A98DF80630ADF80460DD
:10D7900004F0ABF9236938463B432361FEF756FF9B
:10D7A0000E4B1A8802F4415242F4457242F00302D1
:10D7B0001A809A8B22F400621204120C9A830722B8
:10D7C0001A821A8892B242F040021A802E6103B087
:10D7D000F0BD00BF00100240000C014000380040C6
:10D7E00038B50D4B04461B680D461B0312D50B4B79
:10D7F0001B78093B012B0DD8452002F03FFB0D2083
:10D8000002F03CFB204602F039FB2846BDE83840D8
:10D8100002F0CDBC38BD00BF7009002060140020AC
:10D820002DE9FF410A48B0F8008085684488878860
:10D83000C66804F08BF800970290019605484146AF
:10D840002A462346FEF704FA04B0BDE8F08100BF83
:10D850000C000020ABCE01082DE9F04105788AB01C
:10D8600004460DB100252FE0484CB4F90410B4F97A
:10D870000020B4F902300091E17945480191217A04
:10D880000E34029114F9081C039114F9051C04913B
:10D8900029460135FEF7DCF9082DE6D172E02D2B83
:10D8A00016D1072D1DDC204609F045FA0AAB6E1C87
:10D8B00003EB450525F8100C631C1C462278013348
:10D8C000303A092AF9D935462378002BE7D104E00C
:10D8D000A3F13002092A09D8E3E7082DBDF818C0E2
:10D8E00009D00AB0BDE8F041FCF7C0BE202BF8D14A
:10D8F00001342E46E7E7BCF1070FF2D8BDF81A1045
:10D9000040F2DC53A1F2EE2292B29A42E9D8BDF87D
:10D910001C20A2F2EE2080B29842E2D8BDF81E7020
:10D920000BB23CB29C42DCDB10B28442D9DC9842A0
:10D93000D7DBBDF8244004F164039BB2C82BD0D8D8
:10D94000BDF8260003B2112BCBDCBDF82060B42E4D
:10D95000C7D8BDF82250B42DC3D80E4B0FFA8CFC9B
:10D960004FF00E0808FB0C3CACF80610ACF8082091
:10D97000ACF80A708CF80D608CF80E508CF80C40E6
:10D980008CF80F000AB0BDE8F08100BFA6050020AA
:10D9900008CF0108A00500202DE9F74305780446CB
:10D9A0008DB9324C94F86313B4F8602394F8623361
:10D9B0002F48009129460135FEF74AF9102D04F150
:10D9C0000404EFD14EE009F0B6F90F28054636DC25
:10D9D0002046202109F04DF9264FEDB2D7F80090EE
:10D9E000441CAD000026204609F0A5F95FFA86F830
:10D9F000B8F1010F83B208D0B8F1020F0BD0B3F524
:10DA0000B47F24D23A6853530AE0FF2B1FD83B68F7
:10DA10002B44987004E0FF2B19D83B682B44D87036
:10DA200020462C2109F025F9044608B1441C02E0E7
:10DA3000B8F1020F0BD10136032ED4D112E00E48FB
:10DA400000210F2203B0BDE8F043FEF7B5BA09EBA1
:10DA500005000021042209F0D8F803B0BDE8F04326
:10DA6000FCF704BE03B0BDE8F08300BF5004002003
:10DA700028CF01081C1000203CCF01082DE9F043FD
:10DA800004788FB00546002C59D17F4B0021142219
:10DA900009A807AED3F8008009F0B7F800210722E3
:10DAA000304609F0B2F8A700002305A9059308EB5A
:10DAB00007058B801A467548B5F802E030F813C0A8
:10DAC0001CEA0E0F0AD00E300DF1380C185C02F172
:10DAD000010E624402F81C0C5FFA8EF20133072B30
:10DAE000E9D100231A466A48B5F802E013F800C0ED
:10DAF0001CEA0E0F0AD006300DF1380C185C02F14A
:10DB0000010E624402F8240C5FFA8EF20133062BF8
:10DB1000E9D118F807308DE842006A785D49029231
:10DB200009A81A0903F00F03FEF76CFA21465A48B8
:10DB300009AA0134FEF78CF8202CA6D1A1E009F047
:10DB4000FAF81F28044600F38F8028462021E4B20B
:10DB500009F08FF81F2C02D9FCF788FD91E04A4BA1
:10DB6000471C1B68002103EB84042046042209F0B3
:10DB70004CF80026494B09AD284600210A2216F828
:10DB800003805FFA86F909F040F80023FA5CF9187F
:10DB900032B10A2B04D0424502D0EA540133F5E7F2
:10DBA000424501F1010765D109F1FF33032B07D885
:10DBB000DFE803F00E040246002239E000221FE0F5
:10DBC000284609F0B8F82378C0B243EA001006E00E
:10DBD000284609F0B0F8237800F00F0018432070B1
:10DBE0003AE00133062B0AD0284800F11B055D5DA1
:10DBF0008D42F6D10344597D63880B436380013223
:10DC0000D3B20DF1380C634413F8141C21B3002374
:10DC1000EAE70133072B0AD01C4800F10E055D5DD1
:10DC20008D42F6D130F8131063880B4363800132C4
:10DC30000EA9D3B20B4413F8141C69B10023EBE70F
:10DC4000284609F078F80F2804DC284609F073F814
:10DC5000607001E0002363700136052E8AD1012433
:10DC600003F0FEFD6CB977E70D4800211F22FEF797
:10DC7000A3F906E020460021042208F0C6FF002494
:10DC8000EEE70FB0BDE8F0831810002028AE0108C1
:10DC90003DAE010842CF010851CF010849AE01084D
:10DCA0003CCF010870B50446204608F0EFFF05465A
:10DCB00050B9194B19485A79194B013A53F82210A7
:10DCC000BDE87040FDF7C4BF204616492A4608F05B
:10DCD000E5FF60B91448FCF7AEFC144C54F8041F7F
:10DCE00019B11348FDF7B4FFF8E7124805E0002624
:10DCF0000B4B53F8261021B90F48BDE87040FCF7D4
:10DD00009ABC20462A4608F0C9FF01360028EFD108
:10DD1000014B0A4C5E71C7E7500400205DCF01083B
:10DD200034AC010893CD010869CF010830AC01087B
:10DD30008FCD0108EAD00108A4CD01080FBF01086A
:10DD40007FB5044608F0A2FF082823D100231E490E
:10DD5000E25C09681144497801F00301022908BF17
:10DD6000203AE2540133082BF1D10025665D1748B3
:10DD7000314608F07EFF28B101356019314608F0C0
:10DD800078FF10B1FCF772FC1CE0082DEED12046A4
:10DD9000FEF7DAFA0E48FCF74EFC00230D4A04A900
:10DDA0001A4492F834220A440849595C0133082B7A
:10DDB00002F80C1CF2D10023074801A98DF80C30A1
:10DDC000FDF746FF04B070BDDC030020D0CB010896
:10DDD0007CCF0108500400209EC601082DE9FF41B8
:10DDE00005780446002D34D16F48FCF724FC6F4CB5
:10DDF0002069002105F070FE002840F0D1802946FE
:10DE00006B48FDF725FF20696946FEF7C8FA014611
:10DE10006848FDF71DFF60696946FEF7C0FA0146D4
:10DE20006448FDF715FFA0696946FEF7B8FA014698
:10DE30006048FDF70DFFE0696946FEF7B0FA01356D
:10DE400001465D48FDF704FF0C2D04F11004CFD10D
:10DE5000A6E05A49052208F021FF38B9534B0022A9
:10DE600003441030C0281A61F8D199E02046544983
:10DE7000042208F013FF06462046002E42D120213E
:10DE800008F0F7FE002800F08B80451C284608F0BB
:10DE9000FDFE344680464B4B53F824601EB94A4879
:10DEA000FCF7C9FB7CE0284631465FFA88F208F0AF
:10DEB000F5FE671C20BB3D4B0021C2181030C02866
:10DEC00011619C46F7D1414B002403EBC702D2F805
:10DED00004E09846BEF1000F04D13D483146FDF7FD
:10DEE000B7FE54E018F837309C42F6DA23010CEB09
:10DEF0000305103573440FCB013485E80F00F1E7BB
:10DF00003C46C8E708F017FF0B28064643DC2046CE
:10DF1000202108F0AEFE054648B1451C2846FCF716
:10DF2000A1FF224B012403EB0613186100E0044615
:10DF30002846202108F09DFE054640B1451C284694
:10DF4000FCF790FF194B013403EB06135861284688
:10DF5000202108F08EFE054640B1451C2846FCF7FE
:10DF600081FF124B013403EB0613986128462021F0
:10DF700008F07FFE10B9FCF779FB11E00130FCF7E7
:10DF800071FF0A4B032C03EB0616F061F3D1114825
:10DF9000FFF724FF04E0104800210B22FEF70CF8E5
:10DFA00004B0BDE8F08100BF82CF0108500400201A
:10DFB0009DCF0108A3CF01089EC6010801B8010842
:10DFC00021CE010834AC0108A4CD010824B5010814
:10DFD00026CE01080FBF01083CCF010873B50378B6
:10DFE00013B9FCF743FB3AE01E4901AA08F005FF0C
:10DFF000002401462646254699B134B1012C08D1AA
:10E00000084608F098FE064603E0084608F093FE2E
:10E0100005461449002001AA08F0EFFE013401462C
:10E02000EAE70B2D02D910480B220BE0022C0FD18E
:10E03000A6F57A73B3F57A7F07D90C484FF47A7155
:10E040004FF4FA62FDF7B8FF09E0094B23F81560B9
:10E05000074B0848294633F91520FDF7F9FD02B0B2
:10E0600070BD00BF3BCE01083CCF01087CC0010859
:10E07000D0190020A7CF010873B502790D4602F030
:10E08000300110290446836806D133495C2091F899
:10E09000581400FB01330CE020290AD12F495C20E1
:10E0A0000E782D4991F8581448430C2101FB0601C4
:10E0B0000B4402F00F01052933D8DFE801F0030516
:10E0C000080A0D0F1B782DE093F900302AE01B8819
:10E0D00028E0B3F9003025E01B6823E069461868A2
:10E0E000FEF75DF901461E48FDF7B2FD002D31D067
:10E0F000237913F0C00F2DD1E06805F005FB6946C8
:10E10000FEF74DF901461748FDF7A2FD206905F01D
:10E11000FBFA6946FEF743F901461248FDF798FD00
:10E1200018E0002312F0C0020AD0402A12D1217B4D
:10E130000D4A52F8312052F82300FDF789FD09E01D
:10E140000A481946FDF784FD25B10948E1682269AE
:10E15000FDF77EFD02B070BD50040020AD17002019
:10E1600046CE01089CCE01083CAF010817CD01083E
:10E17000B6CF01084B8810B5DC0607D52C4B1479B7
:10E180001B6853F824402B4B43F820404B889B06D8
:10E1900007D5274B54791B6853F82440254B43F887
:10E1A00020404B881C070DD5234B0C781B78B3EB14
:10E1B000141F07DB1E4BD4781B6853F824401D4BFB
:10E1C00043F820404B889B070DD51C4B0C781B78DF
:10E1D000B3EB141F07DC164B54781B6853F824402C
:10E1E000144B43F820404B88DC070ED5144B0C78B9
:10E1F0001B7804F00F049C4207DC0D4B14781B685D
:10E2000053F824400B4B43F820404B885B070ED556
:10E210000C4B09781B7801F00F01994207DB044B86
:10E2200092781B6853F82220024B43F8202010BD3F
:10E230001C1000204C130020571B0020551B0020F1
:10E24000541B0020561B002070B5164B164D5A78F3
:10E25000164B33F81240164BA4B21C80154B1A789B
:10E260001E46022A04BF144B1C802B783BB913486E
:10E27000291D4CF25032FCF709FD01232B7020467A
:10E2800005F03EFA0E49FCF78BFD05F07DFC80B2EF
:10E29000F8F7A0F90B4B18803378022B04BF064B1C
:10E2A000588070BDBE0D002080270020CE0D0020BC
:10E2B0007C3100206C09002008180020CDCCCC3E19
:10E2C000842700209E1900200D4B0278D9684378DE
:10E2D000C943C1F30221C1F1040103FA01F1094B61
:10E2E0000901C9B21A4482F80013027801205109C9
:10E2F00002F01F0200FA02F243F82120704700BF2B
:10E3000000ED00E000E100E070B50279034612F094
:10E31000C00202D0402A07D070BD1248D9681A69DD
:10E32000BDE87040FDF794BC067B0F4B0F4803EB34
:10E33000C606FCF780F900243379E5B2AB420BD96D
:10E3400015B10B48FCF777F933680A4853F82510E4
:10E35000FDF77EFC0134EFE70748BDE87040FCF7AD
:10E360006AB900BFBDCF01083CAF0108D5CF010895
:10E37000E5CF01089CCE0108EBD00108F7B52B4B87
:10E380002B491C6809782B4B2B4D1A8855F8210016
:10E390002A4B2B491B78009008884FF47A71642827
:10E3A000A8BF6420B4FBF1F101902648FDF750FCB2
:10E3B000254B26481968264B0024B1FBF3F1FDF7E5
:10E3C00047FC244B2F461E68E3B207EB830211691A
:10E3D000D9B101259D40354215D02A0713D01E4AD8
:10E3E0000B20D25C00FB0323134A1C4802EB83037F
:10E3F0001A6BFDF72DFC022D05D1194B197A11B1BD
:10E400001848FDF725FC0134DEE71748FCF713F93F
:10E41000164B17481A88174B92B2198840F21453BA
:10E4200003B0BDE8F040FDF713BC00BF94320020FC
:10E43000681400209E19002050AE0108C000002082
:10E4400010180020E7CF0108C400002034D00108D4
:10E4500040420F00100E0020D803002044D00108D5
:10E46000C02800204CD00108EAD00108481500203F
:10E4700050D00108D8320020F8B504460E461746A1
:10E4800000252046202108F0F4FB0446D0B1441CAE
:10E49000204608F050FCB0F5617F05DB40F6340300
:10E4A0009842A8BF184601E04FF46170A0F5617072
:10E4B000192390FBF3F00DB9307000E070703B78D9
:10E4C00001333B700135022DDBD12046F8BDF0B59C
:10E4D000057887B0074605BB454C94F8AA04192176
:10E4E000484300F5617094F8AE2494F8A934009084
:10E4F00094F8AB040634414301F56171019194F83D
:10E50000A6143C48029194F8A714039129460135BA
:10E51000FDF79EFB0F2DE0D167E008F00CFC0E2804
:10E520005EDC354B062606FB003620210023781CD6
:10E530008DF8173008F09DFB741C054658B1451C3A
:10E54000284608F0F8FB032805D89DF817306071BD
:10E5500001338DF817302846202108F08AFB054644
:10E5600058B1451C284608F0E6FB0D2805D89DF853
:10E570001730707001338DF817302846611C0DF18B
:10E580001702FFF779FF202108F073FB054658B109
:10E59000451C284608F0CFFB142805D89DF81730F5
:10E5A000E07001338DF817302846202108F061FB18
:10E5B00050B1013008F0BFFB0D2805D89DF8173089
:10E5C000207101338DF817309DF81730062B0CD0D1
:10E5D00000210622204608F018FBFCF747F804E06B
:10E5E000064800210E22FDF7E7FC07B0F0BD00BF92
:10E5F0005004002082D00108F80800203CCF010818
:10E600007FB505780446D5B9324C94F85B041921DE
:10E61000484300F5617094F8592494F85A340090F6
:10E6200094F85C040434414301F5617101912A4876
:10E6300029460135FDF70CFB142DE6D147E008F023
:10E640007AFB13283EDC234B00F58B7603EB860622
:10E65000601C002320218DF80F3008F00AFB751C88
:10E66000044658B1441C204608F065FB1D2805D817
:10E670009DF80F30707001338DF80F302046202147
:10E6800008F0F7FA044658B1441C204608F053FB42
:10E690000D2805D89DF80F30687001338DF80F30C4
:10E6A0002046A91C0DF10F02FFF7E6FE9DF80F3082
:10E6B000042B0CD028460021042204B0BDE8704091
:10E6C00008F0A3BA054800211322FDF775FC04B039
:10E6D00070BD00BF50040020A2D001083CCF01084B
:10E6E0002DE9F347047807464CB9204601A9FDF708
:10E6F00047FE0134FFF7F4FF122CF6D172E008F068
:10E700001AFBC4B2112C68D8384B781C04F59275EA
:10E71000202103EB450508F0ACFA05F10A09AE7AB1
:10E720000346334F18B9B21E5642564140E007F136
:10E73000E00600F1010A5978304608F09AFA60B113
:10E74000861B032C8CBF03200020F6B238443044D3
:10E7500090F8E480B8F1030F02D1FBF787FF41E0A6
:10E76000B8F102035E4250464FF020015E4108F0CE
:10E7700080FAC8B1002EF0D0013008F0DCFA40F287
:10E78000ED2380B2984205DD40F6CA039842A8BF47
:10E79000184601E040F2EE20A0F2EE20192390FB93
:10E7A000F3F089F8010001E0002ED6D185F80A8047
:10E7B000AB7A1F4497F8E02056B199F8013019213F
:10E7C0004B430C48214603F2EE23FDF741FA09E0E2
:10E7D00009482146FDF73CFA04E0084800211122CF
:10E7E000FDF7EAFB02B0BDE8F08700BF500400204F
:10E7F00050AE0108B7D00108C9D001081CB6010805
:10E800002DE9F041002480462546134B4146E75848
:10E81000E618384608F076FA88B110483946FDF710
:10E8200017FA00213046FFF727FC0D48FBF703FFDE
:10E830003046FFF769FD0B48FBF7FDFE0135143448
:10E8400040F668339C42E0D125B90748BDE8F04165
:10E85000FBF7F1BEBDE8F081DC93010815D101089A
:10E86000EBD00108EAD00108A4CD01082DE9F84F4A
:10E87000074608F00BFA054620B101281AD13B786B
:10E880002A2B17D16B48FBF7D6FE00246A4B6B4846
:10E89000E618E158FDF7DCF930462946FFF7ECFBB6
:10E8A0006748FBF7C8FE143440F668339C42EDD14C
:10E8B000BDE8F88F38463D2108F0DBF9002800F06C
:10E8C000B580034613F8012C202A01D1013BF9E75A
:10E8D000DD1B0130804698F800300130202BF9D044
:10E8E0004FF00009142202FB09F2534B52F803A027
:10E8F000D418504608F0CAF98346514638465A465D
:10E9000008F0CCF9002840F08680EBB25B4540F07F
:10E910008280277917F0C0030BD0402B73D194F875
:10E920000C90484B054603EBC90999F804B02F46F3
:10E930002FE0404608F0FFF981464046FCF792FA86
:10E940000646E06804F0E0FE0146304605F0E2F8D5
:10E95000002858D0206904F0D7FE0146304605F063
:10E96000CFF800284FD007F00F07052F16D04E46DE
:10E9700014E088B9D9F80030414653F8250008F072
:10E980004DF9D0F1010038BF002008B12E46012713
:10E990000135EBB25B45ECD3002F34D02179324600
:10E9A00001F030001028A36806D127485C2590F8B4
:10E9B000580405FB00330CE020280AD123485C25CD
:10E9C0000778214890F8580445430C2000FB075075
:10E9D000034401F00F0105290BD8DFE801F0030320
:10E9E000050507091A7004E01A8002E01A6000E0C9
:10E9F0001E6051461648FDF72BF920460021BDE860
:10EA0000F84FFFF739BB1348FBF715FE2046BDE86A
:10EA1000F84FFFF779BC09F10109B9F1920F7FF4C2
:10EA200061AF0D48BDE8F84FFBF705BE3846BDE8BD
:10EA3000F84FE5E6D8D00108DC93010815D10108AC
:10EA4000EAD001083CAF010850040020AD170020B7
:10EA5000EDD00108F8D00108A4CD01082DE9F04F50
:10EA6000E84C85B0002140F214522046E64F08F0F1
:10EA7000CCF804F568733B60E44B00251D70E44B53
:10EA800004F2D6321A6083232370022003236371B9
:10EA9000FCF794FB4FF48070FCF790FB4FF4802060
:10EAA000FCF78CFB4FF42F72A4F82622202284F866
:10EAB000EA216E2240F6C41384F812220A22A4F836
:10EAC000E43184F8132208232B2284F8DC3184F803
:10EAD0001522D04B212284F816222322C4F8E031DB
:10EAE00084F8172201234FF4C87284F8E83184F8BF
:10EAF000D83184F8143284F81832A4F81A2284F831
:10EB00005854A4F8E65184F8DB5184F8E951A4F88C
:10EB10002A52A4F82852A4F82C5284F8C75184F839
:10EB2000C85184F8C951C4F8CC51C4F8D051C4F8C4
:10EB3000D45184F8D95184F8EB5184F8EC5184F81D
:10EB40001952A4F81C52A4F8205284F81E3284F8FA
:10EB50003D3284F83F3240F2DC53A4F844324FF4A3
:10EB60008263A4F8463240F26C73A4F8483240F253
:10EB700075334FF000080522A4F84E3240F64303E7
:10EB8000A4F8503284F8CD5284F8CC52C4F8D08224
:10EB9000C4F8D48284F8D85284F8D95284F8DA526E
:10EBA00084F8DB5284F8DC2284F83C5284F83E522C
:10EBB0002346032DD4BF0022012205F1010583F86D
:10EBC00052220CBF05221E22122D83F8532203F17C
:10EBD0000203EED1062384F84C324FF47A73A4F882
:10EBE0007632A4F87A32A4F87E32A4F88232A4F8FD
:10EBF000D43040F2DC534FF4FA62A4F8D63040F23D
:10EC00007E53A4F87822A4F87C22A4F88022A4F8E9
:10EC1000842240F27E4E0522A4F8D83040F2EA5316
:10EC200000264FF001094FF0320A4FF4C8714FF03F
:10EC30001E0BC82084F88922A4F8D0E0192240F2E3
:10EC40003A7EA4F8DA3040F2B45384F88A22A4F869
:10EC50008E02A4F89212A4F8D2E0A4F8DC3084F872
:10EC6000406284F8426284F84A6284F84B6284F815
:10EC7000866284F8876284F8946284F841B284F8EA
:10EC80004DB284F8889284F88C9284F8909284F83B
:10EC90009692A4F8DEA0A4F8E01084F8E460029054
:10ECA00001910392A4F8E2A0FDF70CFB3B6884F805
:10ECB0000C90DE759E731E76DE735E7622265D7581
:10ECC0009D759E714FF02D0E5A250E2683F801E09A
:10ECD00083F802E0DD701E7428254FF00F0E3526F4
:10ECE0005D7383F8009083F80BB083F80CB083F861
:10ECF00004A083F805E09E76039A5D72DA71212202
:10ED00005A745322DA7637254B229D721D7583F88B
:10ED100008A083F812A01A779A7701990425D9855B
:10ED20003D4983F830500298596219623B49188571
:10ED3000A3F82AA083F82C90DA7783F83120A1F188
:10ED400024033C22142083F8D72383F8DE033222E5
:10ED500000254FF0640940F2DC5083F8D69383F825
:10ED6000D82383F8D95383F8DD53A3F8E00383F85D
:10ED7000DA2383F8DB2383F8DC230C338B42E0D1E6
:10ED8000274B2826C4F8F431152384F8FC31254B91
:10ED90004FF0010AC4F80032234B2448C4F804326F
:10EDA000234BA4F8F051C4F80832A4F8F251A4F8A7
:10EDB000EE5184F8F86184F8F96184F80CA2FDF74B
:10EDC000C3FA4FF44873A4F80E321A4A0A2384F89F
:10EDD000983284F899324FF47A73A4F89A3284F80E
:10EDE000225284F8235284F8246284F825A284F8FD
:10EDF000105284F89C52A4F89E9284F8A052A2F17A
:10EE0000700319E05004002040180020AD170020C6
:10EE1000901900200000A04200008C4274040020E1
:10EE2000000020419A99193FF6287C3F08D101083B
:10EE30003D0A773FC00400204FF47A71A3F85611C1
:10EE40004FF4FA61A3F8581140F2DC51A3F85A11BB
:10EE5000642183F85C115A2183F85D1183F85E11F7
:10EE6000FF2183F85F110E339342E5D1002384F82C
:10EE7000C631E2181033C02BC2F81080F9D1114806
:10EE80000021402207F0C1FE00230F49E218595823
:10EE900004330868382BC2F86003F6D100218022C1
:10EEA0000A4807F0B2FE0A497022084807F089FEB6
:10EEB00002F0D6FC074839685C2205B0BDE8F04F87
:10EEC00007F07FBEB0070020A493010830070020A0
:10EED000ACAF01084C08002038B50F4B1B68DC892B
:10EEE0000E4B186880F31000201A04F00DFC0C493A
:10EEF00004F05EFC0546204604F006FC0146284668
:10EF000004F00AFD04F01AFE6428A8BF642020EA79
:10EF1000E070C0B238BD00BF641400206815002046
:10EF20000000C842274B1B68984201D10BB17047C3
:10EF300000B998B2244B0022B0F57A7F83F8DB2128
:10EF400025D2012283F8E82183F8D92183F8EC2126
:10EF500083F8EB211D4A12681178022908BF83F853
:10EF6000E811F92801D8032206E0B0F5BB7F05D8E7
:10EF70001278022AF7D0022283F8E8217D21B0FB23
:10EF8000F1F0002808BF012083F8DC010DE0082122
:10EF900083F8D92183F8EC2183F8EB21012283F84F
:10EFA000DC1183F8E8214FF47A71B3F8E430064AB3
:10EFB0003BB992F8DC3159437D2904BF032382F821
:10EFC000E8317047581400205004002040180020F9
:10EFD000104B043033F91030B3F5617F05DB40F698
:10EFE00033029342A8BF134601E04FF461730878DF
:10EFF0001922504300F28330984208DA487850438F
:10F0000000F283309842B4BF0020012070470020F6
:10F01000704700BF2E0F002070B5064600240C4B31
:10F02000E5182A7902F03002B2420AD1E1580948C3
:10F03000FCF70EFE28460021FFF71EF80648FBF7F6
:10F04000FAFA143440F668339C42E8D170BD00BF30
:10F05000DC93010811D10108EAD001082DE9F04F35
:10F060007D4B85B01B685A0702D57C4A127812B9CD
:10F07000DB0640F13B827A4B784C1B6862689A1A37
:10F080000292029946F2A712914240F22F82754FE6
:10F0900063603B88744D3BB32B68A2681878E368C3
:10F0A0000138B3FBF0F0082392FBF3F1521A10443D
:10F0B000A06090FBF3F004F027FB6C4904F02CFCFB
:10F0C0006B4908F0B7F801464FF07E5004F066FA3D
:10F0D000684904F06DFB04F031FD3B882061013B81
:10F0E0003B8000236361A3612B681878E3680138D3
:10F0F000B3FBF0F004F004FB5C4904F00DFC5C4948
:10F1000008F098F801464FF07E5004F047FA59494C
:10F1100004F04EFB07F0C0FF2B68574D5E68824637
:10F12000286804F0F1FA314604F042FB8146206978
:10F13000C0EB0A0004F0E8FA314682464FF07E50F8
:10F1400004F02CFA0146504604F032FB01464846D2
:10F1500004F026FA07F0A0FF2860FCF7CEFF474B2B
:10F160008246D3F82090464B4846196804F0C8FC04
:10F17000444E18B14FF0FF33336008E0504604F0BE
:10F18000C3FA494604F014FB04F0D8FC3060D6F80A
:10F190000080B8F1000F0BDD3B4AB2F9002090452A
:10F1A00006DA2A68C5F80080C8EB0202E26138E09E
:10F1B0002E68E269B8F1000FC2EB06062E6030DD62
:10F1C000324AB2F90050A8452BDCC8EB050004F028
:10F1D0009BFA2D4A8146B2F90000281A04F094FAED
:10F1E0000146484604F098FB0546404604F08CFA78
:10F1F000294604F0DDFA8146304604F085FA2946B6
:10F2000006464FF07E5004F0C9F90146304604F03E
:10F21000CFFA0146484604F0C3F904F08FFC164AC1
:10F2200010601B4A106804F06BFA1A49064604F095
:10F23000BFFA194A8346156895B3184A906804F0D6
:10F2400063FA8146284604F05FFA0146484604F016
:10F2500063FB054625E000BF100E0020A827002014
:10F26000B8320020D6320020C01D002080E6C547FD
:10F27000B1DC423ED048874A1C1A002068180020A2
:10F280000C10002014100020061000201010002088
:10F29000C4320020BD378635BC280020AC280020B1
:10F2A0000025944A2846116804F082FA314604F099
:10F2B0007FFA914A4FF07C511268D4F81490D2F83A
:10F2C0000CA003928D4A1668009004F071FA59461A
:10F2D00004F06EFA594602464846019204F068FA74
:10F2E000019A0146104604F05BF9A16904F058F94F
:10F2F000514604F05DFA8346304604F005FA514663
:10F3000002464FF07E50019204F048F9019A0146FE
:10F31000104604F04DFA0146584604F041F9DDF874
:10F3200000C0A06161468246484604F039F974493C
:10F3300000220A604A608A60724981460A60724906
:10F3400060610A603A88002A40F0D080B8F1000F6E
:10F350006E4F06DD6E4AB2F90020904501DA3E603C
:10F3600003E0504604F0EAFB3860206A301A04F0EB
:10F37000CBF9684904F01CFA8246029804F0C0F9FF
:10F380000146504604F0C8FA04F0D8FB624A40F245
:10F39000DC539842A8BF18469042B8BF10460A21D5
:10F3A0002662FBF783FE039B82469E6848463146F1
:10F3B00004F0FEF98046504604F0A6F93146814635
:10F3C0004FF07E5004F0EAF80146484604F0F0F9A8
:10F3D0000146404604F0E4F8606107F05DFE052157
:10F3E0008146FBF763FE4D4A4D4B1188186001F2D0
:10F3F0001F3189B240F23E639942D4F8248008D884
:10F40000508800F21F3080B298428CBF002001204B
:10F4100000E00020002866D0424B434E1B7803BB1F
:10F42000424B43481A683B680A21D21AB2F5FA7F68
:10F43000A8BF4FF4FA728242A8BF1046FBF736FE0F
:10F44000336880221B79584390FBF2F3B3F5967F23
:10F45000A8BF4FF49673A2F5D6729342B8BF134675
:10F4600001E0344B1B683268C9EB0303967A202114
:10F470005E4396FBF1F63049177D0868B6F5967F36
:10F48000A8BF4FF4967603FB07002C4BB0F5C81FBE
:10F49000A8BF4FF4C8109842B8BF18464FF40053A5
:10F4A000086090FBF3F0264B9E42ACBF8619C6184D
:10F4B000907F04F029F941460746284604F070F889
:10F4C0000146384604F074F94FF06C5104F070F9BD
:10F4D00004F034FB6FF095039628A8BF962098425D
:10F4E000B8BF1846301A174B6562186005B0BDE802
:10F4F000F08F00BF400E0020BC1D00201C1A002011
:10F50000AC280020BC280020C43200205C18002059
:10F51000061000200024744924FAFFFF361800204A
:10F520006415002064180020B81D00205818002021
:10F530000CFEFFFFBC320020501800200000E7FF47
:10F54000D4FEFFFF4418002008B5037833B9084BF8
:10F5500008481978BDE80840FCF77ABB07F0EBFBD8
:10F56000022804D8C0B2FDF76FFC0348EDE708BDE0
:10F57000AD1700200ED301080FBF010808B50948D8
:10F58000FBF759F8084B1868FBF734F8074B186875
:10F59000FBF7E8F8FDF7B0FDFBF79DF8044A054BD3
:10F5A000DA6008BD1FD30108E0140020E414002035
:10F5B0000400FA0500ED00E02DE9F84381460B2632
:10F5C000013E36D0224C09F10108A368A2893227F6
:10F5D0005A612368A28805251A61A368A189DA689F
:10F5E00001204A40DA602368A188DA684A40DA607C
:10F5F000FBF79AF83846FBF764F8A368A189DA6844
:10F6000000204A40DA602368A188DA684A40DA605C
:10F61000FBF78AF83846FBF754F83DB1013DDCD1E1
:10F620004FF4FA70FBF74DF8FA2707E008F1FF38BE
:10F6300004E0084A084BDA60BDE8F883B8F1000F2F
:10F6400001D00025C9E74FF47A70FBF73AF8B7E725
:10F65000740900200400FA0500ED00E038B50F4CF5
:10F6600005461920FBF72DF8A368152000219847BF
:10F6700010B90220FFF7A0FFA36845F0180116207B
:10F680009847A368002117209847A36801213D20CF
:10F690009847A36801213E20984738BD1C1E0020D2
:10F6A000074B5A6832B1DA681AB15A69103322B975
:10F6B00000E0083359601870704700207CE700BFF5
:10F6C0009832002010B50020FBF72EF8054B0024DF
:10F6D0001C70F6F7EFFF044B83F82840DC621C86B1
:10F6E0005C6310BDF9170020A827002070B1124BF1
:10F6F000D3F808359A0303D5104B1B689B0701D438
:10F70000002304E00E4B1B78012BF9D8DAE70D49F2
:10F710005A18595C814203D00C33F02BF7D1704753
:10F72000094B596B19B150784978884203D25A6312
:10F7300000221A86DA627047500400207009002007
:10F74000C0000020E0CA0108A82700202D4B70B59A
:10F750001B68DB0402D50A20FFF7C8FF2A4C636B45
:10F76000002B4DD0294EE26A31688A4248D894F87D
:10F770002800228E596808BB8A5C012084F8280082
:10F7800042B31A78224B013A00FA02F2D3F8083554
:10F790001A4201D1FAF7C8FF1E4B01221A70F6F780
:10F7A00089FF238EB3B9184B5B6B1B78053B012B8C
:10F7B00010D8FAF75FFF184B18600BE08B5C002540
:10F7C00084F8285033B12846FAF7AEFF114B1D706C
:10F7D000F6F770FF626B218E52680B4B525CFE2A6B
:10F7E00002D100221A8670BDFF2A02D1BDE8704006
:10F7F00068E730680A2404FB02020131DA621986E4
:10F8000070BD00BFA0180020A8270020943200205F
:10F8100050040020F9170020843100202DE9F04722
:10F820007A4E33689A0774D5794B45F207201A68E7
:10F83000784B996B511A81426BDD774D9A63FEF7D5
:10F8400003FD2B78754C032B238821D10A2B2AD951
:10F85000002328202B70FAF734FFFEF7F5FC704BDD
:10F860001888F6F7B7FE6F4B6F491B68DA7890FB84
:10F87000F2F0421C082A28BF082258791B790A7026
:10F8800092B250435A436949694B08801A800AE092
:10F890000A2B08D80323644A2B7000231370634A91
:10F8A0001380634A13802A785B4B012A0FD002D35E
:10F8B000022A22D02DE05D4B22881988594B1B6803
:10F8C0009B79CB1A9A4224DC01232B7013E0554913
:10F8D00057480968008889792288401A824202DCE8
:10F8E00002221A7012E05148008801448A4202DD67
:10F8F00000221A700DE0082009E04D4B228819887B
:10F90000484B1B689B790B449A42DDDC0720FFF7CC
:10F91000EDFED6F800A01AF4006F74D03C4B3D4CBD
:10F920001B68E26BC2EB030845F2072290456ADDD3
:10F93000E363404B4048B3F906703A4BB0F8DE1031
:10F940001E68A7F57A77337B3C4D012B03D043D358
:10F95000022B20D042E03A4B206C5A7B394B33F8D3
:10F960001210082390FBF3F289B2821A0A4492FB28
:10F97000F3F322649BB240F6E4425343A4F84410EC
:10F9800071894FF47A72C1EB13335343B6F90820EF
:10F9900093FBF2F321E02C4BB6F80A901B78C5F8E4
:10F9A00000905B071AD500F50D70FDF769FA18B9DC
:10F9B0001AF0100F18BF002707FB07F2322392FB43
:10F9C000F3F31F44B6F908305F434FF47A7397FBA3
:10F9D000F3F74F442F6001E000232B602B68D4E93C
:10F9E000120103FB08F84FF47A7398FBF3F810EB5D
:10F9F000080041EBE8710023C4E91201134A04F046
:10FA0000E3F8134B1860BDE8F08700BF70090020D1
:10FA1000B8320020A8270020681400209E1900207A
:10FA20007C31002064140020C00000206A140020F3
:10FA30006C1400201C1800205004002070150020B9
:10FA4000BE0D0020CE0D0020DA320020407E0500E1
:10FA50006815002010B540001428A8BF142000230A
:10FA6000074A022199540B4499181424834201F83F
:10FA7000014CF5DBFF21D1540F20BDE8104035E6E5
:10FA80008A1D0020064B10B51A881C461043904270
:10FA9000188002D00120FFF7DDFF208810BD00BFD5
:10FAA0001418002010B50B4C0123E3704FF4806054
:10FAB000022384F82030FFF7E5FF074B64211A6822
:10FAC000064B1B685B7801FB0323636123880133CA
:10FAD000238010BD040F002094320020381700202E
:10FAE000064B10B51A881C4622EA00009042188086
:10FAF00002D00120FFF7AEFF208810BD14180020AF
:10FB0000022808B50FD8FDF79FF90748FAF793FDCB
:10FB10000648FFF719FD0648FCF79AF8BDE80840CB
:10FB20002020FFF779BA08BD2BD301080FBF0108C9
:10FB3000EAD001082DE9F04F87B001930023064673
:10FB40008B4602921C46029A934204DA5BF8232009
:10FB500001331444F7E7019B0394002B51D1F7F7CD
:10FB600067FB00284DD1019874E002223B4D8DF8CF
:10FB700014201A0C4FF480578DF8152006201A0A0D
:10FB80008DF816208DF81730F7F776FB6F61062099
:10FB9000F7F7DCFA324B01222F6100201A7005A919
:10FBA0006F6104220025F7F7FDFAD8464F462B4631
:10FBB000029A934218DAC44658F8042B002A44D01B
:10FBC000BA424FF00000715932D33A46CDF800C026
:10FBD000F7F7E8FA7359DDF800C03B447351DCF8DD
:10FBE0000030DF1BCCF800701C4B4FF480521A61C0
:10FBF000DAF80030C9EB04044B44CAF80030019B2A
:10FC000033B32CB3DFF860A0DAF800305FFA83F981
:10FC100004EB0902B2F5807F124A88BFC9F58079EA
:10FC2000D26898BFA14693429FD301F0AFFE0FE088
:10FC30000093F7F7B7FA58F8042C7159BF1A0A4421
:10FC40007251009B002248F8042C01330435AFE7C1
:10FC5000039B181B07B0BDE8F08F00BF000C0140EC
:10FC6000511400200C0000205414002038B50D4C15
:10FC70004FF4805545F20820F7F7FEFA656106203B
:10FC8000F7F764FA084B01222561C7201A706561F5
:10FC9000F7F75CFA256101F079FE044B00221A6047
:10FCA00038BD00BF000C0140511400205414002046
:10FCB0002DE9F047314B86B093F805350446012B0A
:10FCC00001D006464CE006F0E1FF03A90546804658
:10FCD000684601F01FFE039B049A029413442B44D0
:10FCE0003F2B05951AD90023684603A90322FFF785
:10FCF00021FF039B3BB9049B2BB901F047FE059BF9
:10FD0000002B37D001E0F5F7FFFE039B049ADDF8E6
:10FD10001480134443447F2B2CD8029CDFF864905A
:10FD200021464F4617F801ABCAF18006B04538BFEF
:10FD3000464607EB0A00B2445FFA8AFA324606F0FA
:10FD400040FFBAF1800F89F800A013D1C6EB080874
:10FD50003846A119424606F034FF89F8008009E0D0
:10FD6000354616F8011B21B1054B1868FAF72CFD32
:10FD7000F6E72D1B284606B0BDE8F08750040020AA
:10FD800090180020F82700201FB50A4B93F8812017
:10FD90001B789A420BD0684602A901F0BBFD02A96C
:10FDA000022201236846FFF7C5FE01F0EFFD05B012
:10FDB0005DF804FBF82700201FB50E4C94F8812055
:10FDC00023789A4212D0684602A901F0A3FD0023CD
:10FDD00002A902226846FFF7ADFEF5F795FE94F8FA
:10FDE00081002378C31A5842584100E0012004B032
:10FDF00010BD00BFF827002038B5144B05461B681E
:10FE000098421ADD124B93F8054514B1012C09D024
:10FE100017E0104B1B68186988B1A842D4BF0220B4
:10FE2000012038BD7F280CDC01F0A0FDC0F17F006F
:10FE3000854208DDFFF7C0FF05E0002038BD012046
:10FE400038BD022038BD204638BD00BFD414002084
:10FE50005004002090180020064B93F8053513B18C
:10FE6000012B04D1A8E7044B1868FAF776BC0020F0
:10FE7000704700BF500400209018002008B5104BB8
:10FE8000014693F80535012B12D10E4B1878421C10
:10FE9000D2B21A70120648BF0022184448BF1A7026
:10FEA000417001F063FD3F2808D9BDE8084083E7B1
:10FEB000054B1868BDE80840FAF786BC08BD00BFCE
:10FEC00050040020F8270020901800202DE9F04F62
:10FED00085B00F9EC2EB030A4F4C109B00290CBF4C
:10FEE0004FF004084FF00608C6EB030B6368814629
:10FEF000013315463AD12368434580F08880474A4C
:10FF0000029152F82300019206F0C0FE0B30FFF779
:10FF100073FF02990746019A08B1012078E0404B2F
:10FF2000D4F800E0186852F82E200390BEF1030FB9
:10FF300098BF49463B480293F8F73EFA039A029B62
:10FF4000101A1860636801336360374B83F882705E
:10FF50000CE08EB103FB0BF2B25C01219140334AFD
:10FF60001268114208D163680133636063680E98B8
:10FF7000294F8342EDDB32E003FB0AF7236805EBF0
:10FF8000070923B9E85906F081FE431D00E0032369
:10FF900018460293FFF730FF029B0028BDD1204A8C
:10FFA0001168CB1A1360204B93F882201AB12C20D1
:10FFB000FFF764FF02E0012283F88220236843B93F
:10FFC000E859FFF775FE99F904104B1CCBD018487F
:10FFD00002E04B4417481979F8F7EEF9C3E710D15E
:10FFE0000120FFF709FF60B90D4B0A201A68013A9A
:10FFF0001A60FFF743FF3B6801333B604FF0FF336C
:020000040801F1
:100000007B60206840452CBF0020012000E00020DC
:1000100005B0BDE8F08F00BFCC14002034B101085A
:10002000D41400203DD30108F827002098180020A0
:100030004CD3010817CD010810B50446C0B2FFF734
:100040001DFFC4F30720FFF719FFC4F30740FFF7B4
:1000500015FF200EBDE8104010E7002270B51346D2
:100060000446A15801F120003F2820D801F10800E2
:100070000F2806D80231032904D9002B08BF012319
:1000800000E0022304320C2AEBD1012B206811D0AE
:10009000022B1DD06368A26803F0030300F0030085
:1000A0009B0043EA001002F0030210431AE0002311
:1000B0001D461AE000F00F0040F04000FFF7DEFEA2
:1000C000A368606803F00F0343EA0010C0B209E0C0
:1000D00000F03F0040F08000FFF7D0FE2079FFF7EE
:1000E000CDFE207ABDE87040C8E6E2189268AD0007
:1000F00002F18001FF2910D902F50041B1F5803FDE
:1001000002D245F0010508E002F50002B2F1807F5D
:1001100034BF45F0020545F00305043B13F10C0F15
:10012000E3D165F03F00C0B2FFF7A8FE002605F05E
:100130000303A059022BC0B209D0032B12D0012B0C
:100140001ED1FFF79BFEA059C0F3072018E0FFF770
:1001500095FEA059C0F30720FFF790FEA059C0F309
:1001600007400DE0FFF78AFEA059C0F30720FFF714
:1001700085FEA059C0F30740FFF780FEA059000E8E
:100180000436FFF77BFE0C2E4FEAA505CFD170BDDC
:1001900010B504467F2C06D964F07F00C0B2FFF78B
:1001A0006DFEE409F6E7E0B2BDE8104066E6430004
:1001B00083EAE070ECE738B51B4B00221A701B4B4A
:1001C0001A7851072ED522F004021A70184B1B68BA
:1001D0001B0322D5174A137815460B2B17D801227B
:1001E0009A4040F603041440BCB912F4C06F0ED01C
:1001F000093B012B0BD84520FFF740FEFF20FFF7FE
:100200003DFE0D48FFF754FD2046FFF737FE0B4B30
:100210001A680B4B5A600B232B700420BDE8384042
:10022000FFF764BA38BD00BFF8170020DA320020AB
:10023000700900206014002051D30108943200207E
:10024000CC14002010B504460068FFF7B0FF6068CA
:10025000FFF7ADFFA068BDE81040A8E70E4B2DE901
:10026000F0411A689F6815185A688846161807449E
:10027000002444450EDA36F9142037F9143035F9E4
:1002800014001344022293FBF2F3C01AFFF78FFF0E
:100290000134EEE7BDE8F081E42F002070B505469B
:1002A0000E460024B44205DA35F91400FFF77FFF4B
:1002B0000134F7E770BD0FB437B506AC54F8045BF2
:1002C0004820FFF7DBFD2020FFF7D8FD2A46234614
:1002D0000B4900200194FBF7F7FB04460A20FFF7C7
:1002E000CDFD084BC4F1FF241A6804F57F04FD34EA
:1002F00022441A6003B0BDE8304004B0704700BF2C
:1003000009030108D41400200846B7E52DE9F04F91
:100310008F4E8BB033688F4C13F0020F00F02084A7
:100320008D4D2B78002B00F01B84FAF7A3F9D4F83D
:100330000480D4F8009008FB08F209FB0922D4F8E5
:1003400008A06B680AFB0A22C31A069364235A4367
:10035000824B36681B8816F0080603FB03F392FBFA
:10036000F3F3A3F15203686008930AD07C4B1E6834
:100370002EB15E681EB19E68003618BF012606F0D9
:100380000106069803F0BCF9764903F011FA764BA2
:10039000764D1C680490286803F0B6F9214603F0F6
:1003A00007FA8346686803F0AFF9214603F000FAC4
:1003B0000390A86803F0A8F9214603F0F9F9684B07
:1003C0000590594658461F685D689C6803F0F0F92F
:1003D000034603980093014603F0EAF9009B0146A7
:1003E000184603F0DDF8034605980093014603F034
:1003F000DFF9009B0146184603F0D2F807F0A2F897
:100400000990002E00F0B880384603F07DF90646CA
:10041000284603F079F90546204603F075F9314680
:100420000446304603F0C4F929460746284603F03F
:10043000BFF90146384603F0B3F821460746204687
:1004400003F0B6F90146384603F0AAF848490746D2
:1004500003F06AFB002800F08F80384607F072F83E
:1004600001464FF07E5003F057FA074639463046B2
:1004700003F09EF939460790284603F099F939466A
:100480000646204603F094F93A4C05462168079841
:1004900003F08EF9616803463046009303F088F953
:1004A000009B0146184603F07BF8A16803462846E6
:1004B000009303F07DF9009B0146184603F070F8A5
:1004C000E16803460798009303F072F92169074633
:1004D000304603F06DF90146384603F061F8616972
:1004E0000646284603F064F90146304603F058F802
:1004F000009B05461946184603F05AF92946064658
:10050000284603F055F90146304603F049F807F054
:1005100019F80146284603F04BF900F1004528463A
:10052000A16903F045F9002103F03AF8E1690746B3
:10053000284603F03DF9002103F032F8216A06460F
:10054000284603F035F9002103F02AF8054616E0A5
:10055000100E00204C1500207C28002006000020F2
:1005600058150020BD378635280E0020B018002011
:100570000AD7233C6818002000252E462F46089BEA
:10058000262B00F28480484603F0BEF881464046A0
:1005900003F0BAF88046504603F0B6F849460446E0
:1005A000484603F005F941468246404603F000F90B
:1005B0000146504602F0F4FF21468246204603F0F1
:1005C000F7F80146504602F0EBFF5949824603F026
:1005D000ABFA00285BD0504606F0B4FF01464FF05E
:1005E0007E5003F099F982465146484603F0E0F800
:1005F00051468146404603F0DBF85146804620468E
:1006000003F0D6F84B4B82461A6A40461146DC6925
:100610000192009303F0CCF8214684465046CDF871
:1006200008C003F0C5F8DDF808C00146604602F0D6
:10063000B5FF0146384602F0B3FF009B07469B69B1
:1006400050461946009303F0B3F8019A82461146CA
:10065000484603F0ADF80146504602F09FFF0146C0
:10066000304602F09DFF21460646484603F0A0F8BA
:10067000009B04461946404603F09AF8014620467E
:1006800002F08CFF0146284602F08AFF05462A4BFD
:100690004FF0000AD3F800905146D9F80480274C57
:1006A000404603F041FA48B30998254903F01EFA81
:1006B00050B33946404603F07BF8049903F078F8CC
:1006C0000146A06802F06CFF3146A060404603F08E
:1006D0006FF8049903F06CF80146E06802F060FFDF
:1006E0002946E060404603F063F8049903F060F89F
:1006F0000146206902F054FF206105E0C4F808A01B
:10070000C4F80CA0C4F810A00E4BD9F808001B7850
:100710005A0708D40C4B1A6844F61F639A428CBFE0
:100720000023012300E0002393B1084912E000BF39
:100730000AD7233C68180020200E00207C280020C7
:10074000C2B8B23EDA3200209432002000002041CC
:100750004FF07E5103F02CF83946804603F028F81C
:10076000A16802F01DFF0146584602F019FF31460C
:100770008146404603F01CF8E16802F011FF014693
:10078000039802F00DFF29468246404603F010F818
:10079000216902F005FF0146059802F001FF4FF0C4
:1007A0007C510746049803F003F80546294648465D
:1007B00002F0FEFF29460646504602F0F9FF2946A0
:1007C0008046384602F0F4FFD4F81490804B8246FD
:1007D000314609F10040D3F800B0E569A7690093FC
:1007E00002F0E6FF414602463846019202F0E0FF81
:1007F000019A0146104602F0D1FE514602462846B3
:10080000019202F0D5FF019A0146104602F0C6FEA1
:100810000146584602F0C4FE314684465846CDF89B
:1008200008C002F0C5FF514602463846019202F068
:10083000BFFF019A0146104602F0B2FE4146024651
:100840002846019202F0B4FF019A0146104602F0D8
:10085000A5FE0146484602F0A3FE41460246584620
:10086000019202F0A5FF51460390484602F0A0FF16
:100870000146039802F092FE31460390284602F0AA
:1008800097FF0146039802F08BFE0146384602F0BE
:1008900087FE51460390584602F08AFF4146824641
:1008A000484602F085FF0146504602F079FE314687
:1008B0008046384602F07CFF0146404602F06EFE5C
:1008C0000146284602F06CFEDDF808C00646614687
:1008D000604602F06DFF019A05461146104602F08F
:1008E00067FF0146284602F05BFE05460398014675
:1008F00002F05EFF0146284602F052FE31460546F0
:10090000304602F055FF0146284602F049FE06F047
:1009100019FE01464FF07E5002F0FEFFDDF808C0E0
:1009200005462946604602F043FF019A009B29468E
:100930001860104602F03CFF29466061039802F0FF
:1009400037FF2946A061304602F032FF214DE061B9
:10095000FAF748F8296AE86906F06AFC1E4902F0CD
:1009600027FF06F099FB1D4E3080A86900F100407A
:1009700006F00EFC01461A4802F010FE164902F07D
:1009800017FF06F089FB29687080E86806F050FCC4
:10099000114900F1004002F00BFF216A02F000FE55
:1009A00006F07AFB83B213F4004F08BFB3802C46E5
:1009B0000C4B2D6A1CBF00F56160B0801968284699
:1009C00003F0B2F8084B1A7880B142F008020FE049
:1009D000B0000020681800204C3D0F44361800205D
:1009E000DB0FC93F240E0020B90D002022F00802C1
:1009F0005F4E1A70306802F087FE8146706802F020
:100A000083FE0746B06802F07FFE2168064648462E
:100A100002F0CEFE61688046384602F0C9FE01460B
:100A2000404602F0BDFDA1688046304602F0C0FE9F
:100A30000146404602F0B4FDA1698046484602F0F6
:100A4000B7FEE1698246384602F0B2FE01465046E2
:100A500002F0A6FD31468246284602F0A9FE014674
:100A6000504602F09DFDE1680546484602F0A0FEB2
:100A700021698146384602F09BFE0146484602F055
:100A80008FFD61690746304602F092FE0146384606
:100A900002F086FD374B00F100461B68364C5B7850
:100AA000012B15D1354B1B785B070CD4636A4020B2
:100AB00093FBF0F0181A02F027FE294602F070FDB1
:100AC00003F03CF86062636A402093FBF0F001E0C1
:100AD0002B4B188802F018FE0146284602F05EFDF6
:100AE000E16A0746049802F05BFD0146049802F0B3
:100AF00013FFA56A81462946384602F04FFD01469C
:100B0000484602F055FE0146284602F049FD0746D8
:100B1000A0624046D4F8309006F0BEFAE56B297822
:100B2000FAF7C4FA484420633046D4F8348006F01B
:100B3000B3FA2978FAF7BAFA404460633846A66BEC
:100B400006F0AAFA6978FAF7B1FA0E4B06991A6814
:100B500030440A441A60236CA0630133236403E029
:100B6000002323606360A3600BB0BDE8F08F00BF7B
:100B70004C150020200E00207C280020DA320020B6
:100B800006000020C432002008B503783BB90B4BA7
:100B90000B4893F85814BDE80840FBF759B806F025
:100BA000CAF8012808D8054B83F85804F4F7EEFD7D
:100BB000F8F7B4FA0348E8E708BD00BF5004002086
:100BC00012D301080FBF010810B5074B044683F884
:100BD0005804F4F7DBFDF8F7A1FA601CC0B2BDE8D9
:100BE0001040FEF737BF00BF50040020012808B5B1
:100BF00018D8FFF7E9FF0C48F9F71DFD0B48FFF780
:100C0000C3FF0B48FBF724F80848FFF7BDFF09486E
:100C1000FBF71EF81020FEF7FFF9BDE80840034877
:100C2000FEF792BC08BD00BF7BD301080FBF0108CF
:100C300089D30108EAD0010808B5F4F7A7FDF8F751
:100C40006DFABDE808400120FEF704BF964B2DE980
:100C5000F7431B689A0740F12381944C6846A36CC4
:100C60009847002800F01A81914B19780023042935
:100C700003D13DF803008F4A98523DF903208E4D71
:100C800045F813200233062BF1D1276D0021384699
:100C900002F022FF70B1894B8748894E1A780146CD
:100CA000F5F7F2FB3388002B6ED0D4F8C410002384
:100CB0008F1E2CE07D4B93F854609EB9814B1A68CF
:100CC00099467AB1DFF8E481384608F15801314499
:100CD000D9F800202436F9F7D9FF6C2EF2D1012380
:100CE00088F8543094F85430002BD4D00026A859FA
:100CF00002F00AFD744906EBC6031944FAF750F8EE
:100D000006F0CAF9A85104360C2EF0D1C3E7328898
:100D1000DFF8D8C1B2F5C87F04BF00224CF8032029
:100D20005CF8032055F803806048904400224CF89A
:100D30000380EA5004330C2B27F8022FE7D13388C5
:100D4000012B1ED1D0F8C83003F1C8074FF4C87387
:100D500097FBF3F70F80D0F8CC70C83797FBF3F709
:100D60004F80D0F8D000C83090FBF3F3574800888C
:100D70001B1A8B80564BA3F8F021A3F8F221FFF742
:100D80005BFF3388013B3380524B1B685B0774D594
:100D9000514F3B88322B14D1D4F8C4301A88A4F8B0
:100DA000D4205A889B88A4F8D620A4F8D830484B81
:100DB000B3F8F021B3F8F231A4F8DA20A4F8DC306B
:100DC00001E0002B38D0D4F8C4300020991E3B88B5
:100DD00055F800C0322B414B04BF00221A501A585C
:100DE000324E944443F800C000232B5004300C28AA
:100DF0001A4621F8023FEAD13B88012B19D1384924
:100E00000A70384A1370FEF771FCD6F8C430B6F891
:100E1000D4201A80B6F8D6205A80B6F8D8209A8006
:100E20002B4BB6F8DA20A3F8F021B6F8DC20A3F8B3
:100E3000F2213B88013B3B802B4A1378EBB1D4F87D
:100E4000E000002332211370D4F8C42090FBF1F0AD
:100E50001080D4F8E40090FBF1F05080D4F8E80062
:100E600090FBF1F119480688891B9180184AA2F875
:100E7000F031A2F8F231FFF7DFFED4F8C4302A686F
:100E8000B3F90010521A2A60B3F902106A68521AB4
:100E90006A60B3F90420AB689B1AAB60012323702E
:100EA00003B0BDE8F08300BF100E00207C280020B6
:100EB0006C090020081800204C150020DE320020AC
:100EC00062140020B8140020D4280020060000205E
:100ED0005004002070090020781700205C290020B1
:100EE0007A1700207417002075170020442900206D
:100EF000484B73B51B681B0740F18A80464B474D32
:100F00001B68D5F8EC209A1A002AC0F2818003F5FC
:100F1000C333A033C5F8EC30414B68465B68984753
:100F2000404CBDF9003021462360BDF90230204617
:100F30006360BDF90430A3603B4B1A78F5F7A4FA5F
:100F40003A4B21461A781E4612F0040F15D0D5F8F8
:100F5000EC000023C5F8F000354800241844A0F840
:100F60002E4231F81300334C185306341853023311
:100F7000062BF1D122F0040232702F4B1B787BB18B
:100F80002B4B0A68B3F92E02121A0A60B3F9300229
:100F90004A68121A4A60B3F932228B689B1A8B6036
:100FA000D5F8F0301D4A002B32D0D2F8EC00234C9B
:100FB000C31AA34202F1FA0002F1F40416D8204A3F
:100FC00013689288DD686A40DA60002351F81320C4
:100FD000E55EAA42BCBF174D5A53C55EAA42C4BFC4
:100FE000184D5A530233062BF0D111E00023C2F8FA
:100FF000F030E55EC15E0E4A294402251A442B44B6
:1010000091FBF5F1062BA2F82E12F2D1FFF714FE98
:1010100002B070BD100E0020B83200207C280020E5
:10102000140E002058150020DF320020B90D0020DA
:1010300050040020702900201C0E00207FC3C9012D
:101040007409002076290020016B0346C26810B5A0
:10105000406941B1196C541A005D013918BF0A4644
:10106000C0B21A6410BD196A405C0131914228BFB8
:101070000021C0B2196210BD036B13B15A68036C32
:1010800001E0C269036A9A4237BFC068C3EB02003D
:101090008018C3EB0000C0B27047436B13B190F8E7
:1010A00044007047826A436AD31A584258417047D5
:1010B000436A816A02698B4238BF9B185B1A416B95
:1010C00021B149680B44511E8B4203D2013AD31A15
:1010D000D8B270470020704743799B070AD5436A0E
:1010E0008269D154426A03690132B2FBF3F103FB16
:1010F000112343627047437903F0020303F0FF02B8
:1011000043B10369416A826A013BDBB2881A23EA70
:101110000000704710467047437913F0010307D071
:10112000C368C169026A013B881A1840C0B270479F
:1011300018467047437910B513F0010304460DD0EB
:10114000FFF7EAFF58B1226A6369985CE3680132ED
:10115000B2FBF3F103FB1123236210BD184610BD4F
:10116000426A806A131A5842584170474171704769
:10117000334A10B5136C90681944081A40F68C2352
:1011800098429160D060516013463CD9127893F92F
:1011900045108A420BD1111F082908D893F8461030
:1011A000182901D8013103E083F8442002E000212E
:1011B00083F8461093F944108A421CD1204991F8D3
:1011C0004710C1B1002191421E4806DA03EB8104A9
:1011D000246920F811400131F5E7511E00EB41016F
:1011E0001630814203D0002421F8024FF9E7164956
:1011F00008780130087083F84520002201211A7018
:1012000083F8471010BD92F84710B9B1A0F2EF244F
:1012100040F2DA518C4208D811780B2905D80B1D01
:101220000131117042F8230010BD002283F84720DD
:10123000991804320020302A0861F9D110BD00BF8E
:101240000C0B0020AA1C0020A81C002010F80A3C4F
:101250000133DBB20A2B00F80A3C07D910F8131C43
:10126000034A002322F8113000F80A3C704700BFFF
:10127000AA1C0020024B1A6C0132114419647047F9
:101280000C0B0020A1F57A714EF66122054B4A4302
:1012900053F8203004481B6892FBF0F23C3292B2C3
:1012A0001A807047340C002090D00300054BC1EB2E
:1012B000C10153F8203006221B6891FBF2F189B27C
:1012C00019807047340C00201522054B514353F808
:1012D000203006201B6891FBF0F292B21A80704712
:1012E000340C0020024B53F820301B6819807047E3
:1012F000340C0020074BA1F57A7153F820304FF4DD
:101300007A701A681B894B4393FBF0F39BB21380EE
:10131000704700BF340C00208C46654B65492DE9B1
:10132000F04F1B684C899846220200234FF00009B9
:10133000B8EB020869EB03098A88002716040A89BA
:1013400089B0A2FB084502FB0955E20942EA456261
:10135000B4184A884FEAE5134FEAC236CA8847EB09
:101360000305CDE90645A2FB084502FB0955220A03
:1013700042EA056216EB020A8A894FEA2523A8FB96
:10138000024502FB09554FEAD4524FF0000742EAEA
:10139000452247EB030B12F5FA664FEAE55343F19A
:1013A0000007CDE90467B6F5FA6F77F10007019001
:1013B00060DAA2FB026702FB03F107EB410705219C
:1013C000A6FB014501FB0755DDE9066769104FEAF9
:1013D0003400361A67EB0107CDE90667DDE9040141
:1013E000A608354C46EA8576AF104FF0FF35BAEBCC
:1013F000060A6BEB070BA042A94128DADDE9066774
:1014000040F6AC5412194FF0000543EB050302FB04
:1014100003F1A2FB02236FF0060403EB41035142E8
:1014200004FB0311A2FB044536190D444FF00B01D8
:1014300047EB0507A2FB014501FB0355CDE9066714
:101440006D104FEA3404BAEB040A6BEB050B08FB92
:1014500009F3DDE90401A8FB088909EB43094FEA18
:10146000D87242EA49024FEAE973801A61EB03013C
:10147000CDE90401114B019E1A68A2FB0A4502FB4B
:101480000B55620D42EAC5226B15DDE90645121BBC
:1014900063EB0503D40B44EA434406B13460BCF16A
:1014A000000F02D0049FCCF8007009B0BDE8F08FA7
:1014B0002C1B0020301E002024FAFFFF301B0020D0
:1014C0002DE9F04F724BDFF8D0811A68B8F8006050
:1014D00089B0C6EB22135B437600C6EBE202B8F993
:1014E00002601B135643B8F90420039153439B1326
:1014F00003EBE62606EB860380331B120593654B50
:10150000B6F5FA3A1B684FEAE67747F1FF3BC8F8B1
:1015100018600493AAFB0A670AFB0BF3B8F81020C3
:1015200007EB43070692B8F80E30B8F90820079386
:10153000D3170AFB03F102FB0B11AAFB022381461E
:10154000B8F90A000B44C1171D0306FB01F300FBA9
:101550000733A6FB00011403194445EA1255020A99
:1015600042EA016212194FEA2123B8F8064043EB20
:1015700005030032A2FB040143F5004304FB031101
:101580004B10CA1700930192DDE900231343B8F80A
:101590000CC06FD0069A002012B2D3177343A6FB7B
:1015A000024502FB0733079A1D4412B2D3170AFB08
:1015B00003F3AAFB026702FB0B331F4472047B0494
:1015C000A41843EAD63345EB0305049B0019C3F581
:1015D00080164FEAE6714FEAC17343EA56034FEAB9
:1015E000C6720FFA8CF64FEAC60141EB0501121ADA
:1015F00063EB010340F63544A2FB040104FB031135
:10160000DDE9002302F0E0FAB8F916404B1304FBC1
:1016100003F6420B42EAC142E51702FB0566A4FB52
:1016200002456343354402FB0535A4FB02232B44EA
:10163000540E44EAC314B8F9142024184FEA636521
:1016400045EB01055143D31700FB0313A2FB000137
:101650001944C20C42EA413212194FEAE143B8F987
:1016600012404FEA122043EB050340EA03602201D7
:10167000024400E00022B9F1000F02D0120AC9F8BA
:101680000020039A0AB1059B136009B0BDE8F08FF2
:10169000341B0020C0320020841E00207047704799
:1016A000324B2DE9F0411C88314B0A265A89B3F997
:1016B0001250A41A1A89ED025443B3F91420E4130A
:1016C000224495FBF2F22244DA615643A2F57A6293
:1016D00002FB02F4B3F90480B3F902C0B3F90E704F
:1016E00002FB0CFC02FB08F2B3F90C8024136743E5
:1016F00004FB08F4241404EB62320232DC889210FA
:1017000002F50042B3F920506243B3F900304FEACA
:10171000EC2404EBE72404EB8304AC40154B0234C7
:101720001B68D20BA3EBA4044CF250332B41634350
:1017300055BF5B00B3FBF2F3B3FBF2F35B001A128D
:10174000524340F6DE3462430B4C08365C432414AB
:1017500004EB224202F6CF62361103EB221300B1F2
:10176000036001B10E60BDE8F08100BF3C1B0020AA
:10177000441E0020381B002043E3FFFF13B50C4B31
:1017800004465B681B20022101AA984770B19DF8AE
:1017900004209DF8053043EA022303F54E5310332D
:1017A0004FF48C7293FBF2F32333238002B010BD0D
:1017B0001C1E0020054B1A7802F0FF0122B1012205
:1017C000027000221A70704701707047B01E00202E
:1017D00037B5104B04465D68187806216A46A8475D
:1017E000A8B19DF800209DF80130012043EA0223B2
:1017F00023809DF802209DF8033043EA0223638092
:101800009DF804209DF8053043EA0223A38003B02D
:1018100030BD00BF1C1E002013B5104B04465B6892
:101820003B2006216A469847A8B19DF800209DF804
:101830000130012043EA022323809DF802209DF815
:10184000033043EA022363809DF804209DF80530AD
:1018500043EA0223A38002B010BD00BF1C1E00207B
:10186000254AF0B52549264D146800232B700B70CE
:101870002CB900234B702F7818461A4615E01A46EB
:101880001846A61876880EB9A75C5FB1360548BF22
:10189000013002F1040203F1010348BFC0B2802A03
:1018A000DBB2EED12B700870E3E7C5B2BD420CD2BB
:1018B00014F8205001302E099E4205F00F05A8BFF4
:1018C000731C9542A8BF6A1CEFE74B708A700D48E5
:1018D00051084C1E047002F001020B4811440170C3
:1018E000C3F347020949501E087003F00103084979
:1018F0001A440A70F0BD00BF181000207C29002097
:101900004C1B0020541B0020561B0020571B00209E
:10191000551B002010B50A4B0A4A1B7842609C18E0
:10192000094A046012789A4204D3D31A0B60002348
:101930004B6010BDC3F180030B604A6010BD00BF57
:1019400079280020F9270020F82700201FB56846D5
:1019500002A9FFF7DFFF044B1868029B1844039BA2
:10196000184405B05DF804FB54140020054A064BEA
:1019700010781B7883422EBFC0EB0300C0F18000BB
:10198000C018704779280020F8270020024A002359
:101990001370024A13707047F8270020792800203E
:1019A0002DE9F041038A87890446BFB20D461F40E6
:1019B000002F36D0B7FA87F34FF00042DA40D24317
:1019C00091B21B3B21821740042BF1D8DFE803F0D2
:1019D000221F1C1903006B6A33B103F1FF38002387
:1019E0001FFA88F86B6203E0B4F82C801FFA88F8BD
:1019F0002E6A002EDCD03368304641469847766820
:101A0000F7E72868A18E08E06868218F05E0A868DC
:101A1000A18F02E0E868B4F84010036889B29847E3
:101A2000C6E7BDE8F0810C4B800A98420CD003D881
:101A3000B0F5801F0ED00BE0084B984206D049331A
:101A4000984205D10020704702207047032070475C
:101A5000FE207047012070470100100002001000B6
:101A600090F83B3210B57BB990F83A3290F83922B1
:101A7000934209D201219940B0F8404201332143F9
:101A8000A0F84012DBB2F3E710BD8379DB0703D582
:101A9000D1F1010138BF0021D0F834315A681B89D7
:101AA00009B11361704753617047044B53F82030FC
:101AB0001BB107289CBF1B6819807047640C00206D
:101AC00001F003039B000F229A40984001F0FC01B3
:101AD00001F1804101F5803110B58C6824EA0202E1
:101AE0008A608A6802438A6010BD2DE9F0410F8840
:101AF000002347FA03F2D2072BD58A7803F00705B3
:101B000012F0100F18BF91F803C002F00F0618BFB3
:101B100046EA0C06AD004FF00F0C0CFA05FC06FA75
:101B200005F5DC0850F82480282A28EA0C0C45EA40
:101B30000C0540F8245005D101229A40C46824EADB
:101B4000020205E0482A04D101229A40C4682243D7
:101B5000C2600133102BCCD1BDE8F0813C4B70B595
:101B6000B3F9004040F2E635241A04F2F316AE420F
:101B700003D8002CB8BF644201E04FF4FA74B3F903
:101B80000230181A00F2F31540F2E6339D4203D8F2
:101B90000028B8BF404201E04FF4FA70A042ACBF49
:101BA000034623462B4C0525C3F5FA7393FBF5F347
:101BB000B4F90200B4F900500028B8BF4042002D2B
:101BC000B8BF6D428542A8BF2846632922DDF929A6
:101BD0003BDCC1F1FA0112254D430A24291A614365
:101BE00095FBF4F491FBF4F16429A8BF6421002A69
:101BF00021EAE17108DD643B6420584390FBF2F078
